:020000040800F2
:100000000080002011E80008ADF400083543000826
:10001000AFF40008B1F40008B3F4000800000000D9
:10002000000000000000000000000000D1330008C4
:10003000B5F400080000000061340008A534000891
:10004000B7F40008B9F40008BBF40008BDF40008D8
:10005000BFF40008C1F4000841F4000847F40008A8
:100060004DF4000853F4000859F40008C3F40008E4
:10007000C5F40008C7F40008C9F40008CBF4000870
:10008000CDF40008CFF40008D1F40008D3F4000840
:10009000D5F40008D7F40008D9F400085FF400088C
:1000A000DBF40008DDF40008DFF40008E1F40008E8
:1000B000E3F40008E5F40008E7F40008E9F40008B8
:1000C000EBF40008EDF40008EFF40008F1F4000888
:1000D000F3F40008E9FC000819010108F5F4000830
:1000E00083F400082DF50008F7F40008F9F400087F
:1000F000FBF4000800000000000000000000000009
:1001000000000000000000005FF808F110B5054C89
:10011000237833B9044B13B10448AFF300800123B3
:10012000237010BD280500200000000060F20108C7
:1001300008B5034B1BB103490348AFF3008008BD6A
:10014000000000002C05002060F2010810B50446F4
:10015000C06910B101210CF06FFD206910B10121BF
:100160000CF06AFD204610BD2DE9F04186B005F087
:1001700001FE054600F03EFF0027044606AE06F8E5
:10018000097D284605F08EF9324604F180012846A3
:1001900000F0FCF904F1080300933246231D3849AE
:1001A000284605F0A9FC04F128030093324604F127
:1001B00024033449284605F09FFC04F148033246E5
:1001C0000093314904F14403284605F095FC2F497A
:1001D000284605F0FDFB2E4B20703246CDE900731A
:1001E0002C4904AB284605F05FFC3C23049A2A49BD
:1001F0005343C4E91A37294B3246CDE900732846E8
:1002000005AB05F051FC059B4FF00108C4E91C3714
:1002100064233246CDE90083214904F1780328465E
:1002200005F022FC4FF47A733246CDE900731D4984
:1002300004F17A03284605F017FCFF233246CDE986
:100240000083194904EB0803284605F0EDFB05235C
:10025000A370164B3246CDE90073154904F17C03B7
:10026000284605F021FC9DF80F3033B111480DF000
:10027000D1FB8E21104803F0CBFF06B0BDE8F08122
:100280008EB8010899B80108A4B80108B0B80108EF
:1002900000F91500BCB80108C5B8010800D68300F4
:1002A000CBB80108D3B80108E3B8010840420F00F9
:1002B000EAB80108FBB801080EB90108F8B5002535
:1002C000C0E901120570C0E90335C0E90555C0E970
:1002D0000755456206990446164600F11C0704F0CE
:1002E0003DFC38B9314607480DF094FB2021064803
:1002F00003F08EFF069A3946204604F0F7FB2046AD
:10030000F8BD00BF12B901080EB90108F8B5002503
:10031000C0E901120570C0E90335C0E90555C0E91F
:100320000755456206990446164600F11C0704F07D
:1003300031FB38B9314607480DF06CFB20210648E7
:1003400003F066FF069A3946204604F00DFB20466E
:10035000F8BD00BF12B901080EB9010830B58DB063
:1003600005F008FD044600F04BFC5B4B5B4A009334
:1003700003215B4B02A8FFF7A1FF02A9204605F06D
:100380009FFD02A8FFF7E2FE564B574A0093032158
:10039000564B02A8FFF792FF02A9204605F090FDF8
:1003A00002A8FFF7D3FE524B524A009303214F4B52
:1003B00002A8FFF783FF02A9204605F081FD02A8ED
:1003C000FFF7C4FEB4234C4A009302214B4B02A812
:1003D000FFF79CFF02A9204605F072FD02A8FFF777
:1003E000B5FE4123464A00930221464B02A8FFF77F
:1003F0008DFF02A9204605F063FD02A8FFF7A6FEC7
:1004000000230121404D414A02A88DF80830039194
:100410000495CDE90523CDE90733CDE909330B93E5
:1004200004F0B8F938B9294639480DF0F3FA20211B
:10043000384803F0EDFE012209A902A804F098F95A
:1004400002A9204605F03CFD02A8FFF77FFE052328
:100450000225314A00930221304B02A8FFF756FFD4
:1004600002A9204605F02CFD02A8FFF76FFE2C4BD9
:100470002C4A2946009502A8FFF748FF02A920460A
:1004800005F01EFD02A8FFF761FE1423264A009323
:100490002946264B02A8FFF739FF02A9204605F09E
:1004A0000FFD02A8FFF752FE6423214A009329465C
:1004B000204B02A8FFF72AFF02A9204605F000FD05
:1004C00002A8FFF743FE01F0F9F9012221460BF0E3
:1004D0001FFC0DB030BD00BF21B701088EB8010868
:1004E000FCB6010845B7010899B801082DB7010805
:1004F00054B70108A4B80108C5B8010863B70108DA
:10050000BCB8010885B70108B0B80108B0B7010848
:1005100012B901080EB90108E3B80108CBB7010808
:10052000DAB70108CBB80108D3B80108F2B701085F
:1005300085B801084FB8010870B515460022C0E91A
:1005400001150270C0E90332C0E90522C0E90722A3
:100550004262DDE90412044600F11C0604F016FBB9
:1005600038B9294607480DF055FA2B21064803F003
:100570004FFEDDE904233146204604F0F4FA20461C
:1005800070BD00BF12B901080EB90108F7B50C46DD
:10059000154916460546002705F01AFA07230C22CE
:1005A0002070CDE900322846A31C324667700F49FF
:1005B00005F03AFA0E23E3704FF47A733246CDE930
:1005C00000730B49231D284605F04EFAA388094AFB
:1005D0005A43D317C4E904235B104FEA3202C4E93B
:1005E000022303B0F0BD00BFE7BA0108ECBA01086E
:1005F000EFBA01088051010038B5044600F03CFC18
:10060000054694F9030009F0C5F907F057FBA078F7
:1006100009F08EF907F048FB607807F027FC01F03D
:100620004DF9C36B3C301B6898470023C5E91601A0
:1006300085F83A30207838BDF8B500F01DFC064644
:1006400007F02AFD012871F1000304460D460BDB7B
:1006500007F0A4F906F046F94B492B4622460978E3
:1006600006F07DFE494B39E0494C23680133236095
:1006700001F024F947490BF0F7FA216846480DF0DC
:10068000C9F907F0D1F907F00FFA18B995214348D5
:1006900003F0BEFD4EF6602007F0DCF9054618B900
:1006A00098213E4803F0B4FD6B78042B03D09921C8
:1006B0003A4803F0ADFD2F7E28460DF031FA7FB1A8
:1006C00037480DF0A7F901F0F9F8C36B3C301B680F
:1006D0009847C6E9160107F061F9324B1878F8BD62
:1006E00031480DF097F92368042B0CD905F05CFB19
:1006F000037843B12D480DF08DF94FF47A7001F075
:100700003BFF0FF039FD23681E22013BDBB21E2B9D
:1007100028BF1E23A3F12005C3F1200402FA05F12E
:1007200022FA04F4002521434FF4E14402FA03F0D5
:100730008D4208BF844220D3002908BFB0F5616F05
:1007400006460F461BD2B0F5167F71F1000319DA89
:100750003C2871F10003ACBF11460A2100200DF0C6
:10076000A7FA341847EBE075294620460DF0E8F863
:1007700001460F480DF04EF96CE726462F464FF420
:100780001671EBE73C21E9E749050020AF0B00209B
:1007900044050020CDCC1C403DB901080EB901082C
:1007A00054B90108AC0B002064B9010876B90108FE
:1007B0008FB9010838B5044600F05EFB0546CCB1A0
:1007C0000D480DF027F901F079F8C36B3C301B6838
:1007D0009847C5E91601637F802B06D1227FA16E61
:1007E0002868BDE8384004F0EBBD0448BDE8384057
:1007F0000DF010B938BD00BFBBBA0108D3BA01086B
:100800002DE9F047C6B000F037FB054600F0F2FBDB
:100810000023FC2207A9074603A88DF803300CF03B
:1008200056F901F04DF807F035FAFC28824604D954
:100830004FF496717F4803F0EBFC00F01DFB03685A
:100840005B687BBB90F8283013B190F829305BB31C
:1008500090F8383013B190F839303BB306F0A0FF70
:10086000002800F08B81042495F83A6006B3B7F8AD
:10087000981000200DF01CFAC517294604460DF00B
:100880005FF801466C480DF0C5F806F02BF82246DB
:100890002B466A49097806F062FD694B187846B024
:1008A000BDE8F0870124DFE70224DDE70324DBE76E
:1008B00007F0F2FB8046894658EA09030AD00DF09A
:1008C0003FF801465F480DF0A5F806F00BF84246E8
:1008D0004B46DEE7032C00F0C380042C00F0478178
:1008E000022C4FD058480DF095F80DF103035FFA34
:1008F0008AF207A9286804F0E7FA044600F0DEFF50
:10090000C36B3C301B689847B7F884308BB1D5E98E
:100910001623801A61EB0301D7E92223904271EB81
:10092000030306DB0DF00CF8014648480DF072F8A1
:10093000012600F0C3FF46490BF096F907F074F862
:100940009DF803303246214607A807F093F920B9F5
:100950004FF4B671374803F05BFC07F093F8037867
:10096000044623B140F26F11324803F051FC07F006
:1009700015F8D4F8A000FFF71DFF204608F0CAFDC7
:10098000344B8BE734480DF045F8D5E90423C5E92D
:100990000823012385F8293000F06EFA044603A8E5
:1009A0000CF0CDF803222D4903A80CF09DF8082186
:1009B00003A80CF0B7F8314603A80CF0B3F80521F2
:1009C00003A80CF0AFF800F057FA027F437F62B340
:1009D000002B14BF6721652103A80CF0A3F80FF0CA
:1009E00063FC014603A80CF09DF8002103A80CF05D
:1009F00099F8618B03A80CF0D7F8B4F9181003A884
:100A00000CF0A0F8226E94F8AC30002A0CBF022142
:100A1000002103A819430CF085F8012303A88DF8E1
:100A200003300CF08AF8C4B268E7002B14BF6621CB
:100A30000021D1E70EB90108FABA010849050020E2
:100A40004805002011BB010826BB01088DBB010829
:100A5000CDCC1C40AF0B00203DBB0108C7B701083F
:100A600049480CF0D7FFD5E90423C5E90C2301233D
:100A700085F8393000F000FA044603A80CF05FF85E
:100A800004F1640101A812F065FFDDF80490B4F9E7
:100A9000181003A8DDF808800CF054F8618B03A847
:100AA0000CF082F83949484615F06CFD15F046FF08
:100AB000014603A80CF05FF83449404615F062FD8A
:100AC00015F03CFF014603A80CF055F83049D4F866
:100AD000880015F057FD15F031FF014603A80CF012
:100AE0003EF8236E94F8AC10002B0CBF02230023B9
:100AF00003A819430CF016F894F8681003A80CF03A
:100B000011F8D4F884A02349504615F0F7FE28BB0D
:100B10002149504615F036FD15F036FFC1B203A845
:100B20000CF000F80021484615F0C0FEC0B10021CD
:100B3000404615F0BBFE98B10021D4F8880015F0AE
:100B4000B5FE68B10022002303A80CF021F8D4E917
:100B5000102303A80CF01CF802235FE7FF21DEE757
:100B600004F1700013F0B0FB02460B46ECE70B48B3
:100B70000CF050FF34468DF80360BFE608480CF0D7
:100B800049FF084B8AE600BF4FBB01080050C3472E
:100B90000000C8420000CC41000020415FBB0108BA
:100BA00077BB0108AC0B00202DE9F04100259DF832
:100BB0001860C0E901120570C0E90335C0E90555A8
:100BC000C0E90755456231460446174600F11C0846
:100BD00003F0E0FD38B9394607480CF01BFF20212F
:100BE000064803F015FB32464146204603F0C0FD9F
:100BF0002046BDE8F08100BF12B901080EB9010816
:100C0000F0B5A9B0044600F059FE05460CAE00F15F
:100C100011073946304606F081FD2A4652F84D0F3D
:100C2000213551683346256301256763082703C3CF
:100C3000504A514B2946009502A8FFF7B5FF02A97B
:100C4000204605F03DF902A8FFF780FACDE90067DC
:100C500010264A4B04211A460DEB0700FFF76CFCE7
:100C60000DEB0701204605F02BF90DEB0700FFF710
:100C70006DFA0EAB424A00930197424B04210DEBF3
:100C80000700FFF759FC0DEB0701204605F018F9A6
:100C90000DEB0700FFF75AFA10AB00933A4B0196A1
:100CA0001A4604210DEB0700FFF746FC0DEB070188
:100CB000204605F005F90DEB0700FFF747FA14ABE6
:100CC000324A019600930421314B0DEB0700FFF7E8
:100CD00033FC0DEB0701204605F0F2F80DEB0700A1
:100CE000FFF734FA0C230A262A4A009302212A4BE2
:100CF0000DEB0700FFF70AFB0DEB0701204605F09F
:100D0000DFF80DEB0700FFF721FA244B244A009689
:100D100002210DEB0700FFF7F9FA0DEB0701204662
:100D200005F0CEF80DEB0700FFF710FA1D4B1E4A39
:100D3000294600950DEB0700FFF736FF0DEB070185
:100D4000204605F0BDF80DEB0700FFF7FFF9174B44
:100D5000174A009602210DEB0700FFF7D7FA0DEBBB
:100D60000701204605F0ACF80DEB0700FFF7EEF9A0
:100D700029B0F0BDE7BA0108A5B90108B8B9010862
:100D8000D8B90108BFB90108E0B9010811BA0108D2
:100D9000E7B90108ECBA010818BA010840BA01081D
:100DA00067BA010870BA01085BC301088CBA010870
:100DB000EFBA0108FF23024A1370024A137070470A
:100DC000490500204805002070B50D4606460AF08A
:100DD00087FE044603680121DB6898472368314693
:100DE0001B692046984723680021DB682046984706
:100DF00035B1236829462046BDE870401B69184775
:100E000070BD10B504460AF06BFE2146BDE81040E7
:100E10000AF074BC1FB56E23CDE90131002301A98E
:100E2000039305F07DFC05B05DF804FB1FB561235D
:100E3000CDE9013101A9039205F06EFD05B05DF821
:100E400004FB1FB57023CDE90131002301A98DF802
:100E50000C3005F061FD05B05DF804FB07B58DF8B9
:100E6000041001A98DF805208DF8063005F012FE5A
:100E700003B05DF804FB000038B5194C216811F08F
:100E800001012BD14FF40045164800224FF00043DA
:100E900005830125C0E90223C0E90423C0E9082332
:100EA000C0E90C23C0E91023C0E916230160418387
:100EB0000177417780F8281080F8291080F83810E1
:100EC00080F8391080F83A1080F84810056680F8EC
:100ED000AC104822643016F076F92560014838BD20
:100EE00058050020100600202DE9F04385B0894602
:100EF0008046FFF7C1FF4FF00041D0E90456044699
:100F000000208E4208BF854205D015EB080246EB53
:100F10000903C4E90423D4E908568E4208BF854278
:100F200005D015EB080246EB0903C4E90823D4E910
:100F30000C564FF0004100208E4208BF854205D07C
:100F400015EB080246EB0903C4E90C23D4E910565B
:100F50008E4208BF854205D015EB080246EB090317
:100F6000C4E9102304F1490528460CF08FFC4246E1
:100F70004B4668460CF065FC009BC4F84930019B69
:100F8000C4F84D30BDF80830A4F85130D4E9162328
:100F9000B3F1004F08BF002A05D018EB020649EB59
:100FA0000307C4E9166705B0BDE8F08308B5FFF78D
:100FB00063FF0023493000F8013CBDE808400EF013
:100FC0006FBB000038B50AF08BFD0546FFF754FFF4
:100FD000044628460AF0BCFA608328460AF092FBD1
:100FE000618B20830246BDE8384001480CF012BDF9
:100FF000E6BE0108F8B5144E346814F0010421D19E
:10100000124DA0222146284616F0DDF80127284679
:101010001A22214600F8087B16F0D5F81A2221463C
:1010200005F1280016F0CFF81A22214605F14800F4
:1010300016F0C9F800224FF00043C5E91A23C5E9AC
:101040001C2337600148F8BD5405002070050020BE
:101050002DE9F04F89B0FFF70FFF06460AF040FD7B
:101060000546FFF77BF9FA2001F086FAFFF77CF8D6
:10107000FFF7C0FFB74B427805F168041A70827819
:10108000B54BB0F878101A70B0F87A2020460AF004
:1010900005F9B24B48222B64002106F1640016F0DA
:1010A00092F813F0B1F9C82001F066FA02F0E0FFFF
:1010B00020460AF027F9FFF79DFFA94E0546336841
:1010C000A84C13F0010F06D10AF00AFD0AF054FEF5
:1010D000012320603360A4492068FFF79BFEA34BE7
:1010E000A34918702068FFF795FEA249A24E087028
:1010F000A2492068FFF78EFE307026680A2200237E
:1011000005AF9F4905A805F075FA3946304605F048
:1011100007FB9C4B266818706A6805AF9A4905A8BA
:1011200005F0A4FA3946304605F0FAFA26686A6AEC
:101130008DF8070005AF954905A805F097FA3946DF
:10114000304605F0EDFA26686A6C8DF80B0005ADA7
:101150008F4905A805F08AFA2946304605F0E0FADD
:101160008DF80F0020680AF04DF88A4A8DF80C00BF
:1011700089492068FFF75AFE884A8DF80800884997
:101180002068FFF753FE874982462068FFF759FE23
:10119000854A8DF80D0085492068FFF747FE844A8F
:1011A000054684492068FFF741FE834A8DF809000F
:1011B00082492068FFF73AFE814906462068FFF71A
:1011C00040FE804A8DF80E007F492068FFF72EFE12
:1011D0007E4983462068FFF734FE7D4981462068BA
:1011E000FFF72FFE7B498DF80A002068FFF729FEE4
:1011F0009DF8087080462068774A80F82870394644
:10120000764F53461278FFF729FE33463A789DF819
:1012100008102068FFF722FE6F4A9DF80D305146F6
:1012200020681278FFF71AFE564953460A7820685C
:101230009DF80D10FFF712FE33463A7851462068AC
:10124000FFF70CFE644A3346314620681278FFF7F8
:1012500005FE49489DF80E30027831462068FFF7B8
:10126000FDFD484933460A7820689DF80E10FFF7C7
:10127000F5FD5B463A7831462068FFF7EFFD564AA8
:101280009DF80930594620681278FFF7E7FD9DF870
:1012900009303A7829462068FFF7E0FD33463A786E
:1012A0009DF809102068FFF7D9FD304A4B46594692
:1012B00020681278FFF7D2FD9DF80A309DF80C20C7
:1012C00049462068FFF7CAFD2B469DF8072049468E
:1012D0002068FFF7C3FD2B469DF80B204946206888
:1012E000FFF7BCFD2B469DF807209DF80A102068EB
:1012F000FFF7B4FD2B469DF80B209DF80A102068DF
:10130000FFF7ACFD1B4943460A7820685946FFF7B2
:10131000A5FD2B469DF8072041462068FFF79EFD5E
:101320002B469DF80F2041462068FFF797FD2B467E
:101330009DF80C2041462068FFF790FD01224FF4F4
:10134000A071206805F0FCFC002000F07BFE09B0D5
:10135000BDE8F08F5102002050020020E90E000885
:10136000500500206C05002070BE0108C00600205A
:1013700077BE0108C1060020480500207FBE010895
:1013800087BE01084905002093B801088FBE0108F7
:1013900095BE0108191700089BBE01083906000810
:1013A000A0BE0108A5BE01088D1B0008AFBE010844
:1013B000E1130008B6BE010801080008BBBE010821
:1013C000BFBE010891190008C8BE0108D0BE0108BF
:1013D000D8BE0108DFBE0108AF0B0020AC0B002017
:1013E0002DE9F04F9DB00AF07BFB0746FFF702FEA8
:1013F000AF49814638460AF037FCFFF73DFD054608
:10140000FFF73AFD80460AF06BFB0446FFF7F2FD5A
:101410000021064688F8481020460AF06FF9B17896
:1014200070780DF015F9236864211B6920469847F0
:10143000A04920460AF062F9236864211B6920460E
:1014400098479C4920460AF059F995F83830002B06
:1014500000F00F8195F83940002C40F00A81964841
:1014600007F1680A0CF0D6FA0121504609F072FF24
:10147000FFF7C0FD04900AF033FB00F13C03019339
:10148000804612F0F9FE04704470C474064612F0EF
:10149000F9FED8F83C20019812689047049BCDE9EA
:1014A0000201D3E91C2380185941CDE9060100202F
:1014B0000021CDE90401194610460CF041FA0890CC
:1014C000DDE904010CF03CFA089B024619467B4812
:1014D0000CF0A0FA4FF475711420FFF775FCD8F8E2
:1014E0003C3001981B689847DDE90623DDE902BC22
:1014F000121A63EB0103B0EB0B0B61EB0C0C3178B0
:10150000CDE904BC013469B9022C40F0B7806C48C5
:10151000CDE908230CF07EFA08F1680009F0F2FE2C
:10152000DDE90823717819B9012A73F10001C2DAE3
:10153000642012F0E1FA002800F0AD804822314624
:101540000AA815F01CFE12F0F3FA9DF82A302BB110
:101550009DF8293013B901238DF829309DF82930E1
:10156000BBB10F9B23F07F4323F0FF038BB9109B8C
:1015700033F47F030DD1119B33F47F4409D1002153
:10158000139815F093F920B14E480CF043FA8DF8FA
:1015900029409DF83B305BB10DA812F095FE40A3A9
:1015A000D3E9002382428B4102DB00238DF83B30DC
:1015B00099F800306BB19DF83B3053B1FB6B0DA82F
:1015C0005C6812F081FE07F13C0602460B4630468D
:1015D000A0470021504609F0BDFE9DF82940002C8F
:1015E0007AD039480CF016FAC8214FF49670FFF7FC
:1015F000EBFB00214FF49670FFF7E6FB95F86530A2
:1016000005F164044BB3D9F87C3033B30AA9204602
:1016100012F0E0FE14F046FB0646D9F87C000F46B7
:1016200014F01EFB20A3D3E9002314F093FB024621
:101630000B463046394614F013FE70B10DA812F077
:1016400043FEB1F1004F08BF002806D0D5E91023B2
:1016500082428B4101DAC5E9100148220AA92046DD
:1016600015F08DFD19480CF0D5F99DF8293085F855
:10167000AC30174B18781DB0BDE8F08F052C7FF605
:1016800051AF1448CDE908230CF0C4F9FFF7F4FB7F
:101690000121017744E78DF829008DF83B0087E7A9
:1016A000FFE00B5E00000000FCA9F1D24D62503F4C
:1016B00066663640AD0F000857BC01086ABC0108D9
:1016C00089BC0108CFBC0108E6BC010812BD0108B5
:1016D000AC0B0020AFBC01080E480CF09BF9C821F0
:1016E0004FF49670FFF770FBC8211420FFF76CFBD6
:1016F000C8211420FFF768FBC8211420FFF764FB02
:10170000C8211420FFF760FB21461420FFF75CFB83
:10171000A8E700BFFBBC01082DE9F8430AF0E0F997
:101720000446FFF7A9FB0546FFF764FC4F4F06464A
:101730003B68DB0708D404F037FB802201464C48A5
:1017400003F068FB01233B60494B04F13C002B6034
:101750007278484B01271A70B278474B1A70474A83
:10176000474B1A60E36B1B68984785F82870C5E9FA
:101770000401FFF727FC04F168050AF0B1F94149BB
:101780000AF072FA3946284609F0E4FD322712F0D1
:1017900073FD037833B9236864211B692046984799
:1017A000013FF4D112F068FD03788BB936480CF094
:1017B00031F9284609F0A6FD322712F05DFD0378C5
:1017C00033B9236864211B6920469847013FF4D14F
:1017D0000021284609F0BEFD0A2000F0CDFE0AF0E7
:1017E0007FF9044612F048FD057894F88440002DF6
:1017F00014BFA1464FF00009244FDFF8BC802448F5
:101800000CF008F9002D14BF42463A46214B2249FC
:1018100022480CF0FFF8002C14BF42463A461D4BFC
:101820001F491E480CF0F6F81E491F48B9F1000F79
:1018300008BF39460CF0EEF81C480CF0EBF8FFF747
:101840001BFB85F0010584F001040577447704F063
:10185000ABFA05F0B7FD06F18000FEF7CDFE18B13A
:10186000134B1878BDE8F883124BFAE74C050020BB
:101870005C0500205102002050020020030E0008E9
:10188000900C002066663640D6BB0108CEBB01082E
:10189000FDBB010883C401080DBC010818BC010888
:1018A0002FBC0108D3BB010834BC010849BC0108A6
:1018B000AF0B0020AC0B0020C9BB01080AF010B927
:1018C0002DE93048FFF7D8FA0446FFF793FB0546A9
:1018D00009F0BAFCB1F1004F08BF002806D0D4E9E6
:1018E000102382428B4101DAC4E9100194F8483098
:1018F0007BB104F149000BF0C9FFB1F1004F08BF03
:10190000002806D0D4E9102382428B4101DAC4E9D1
:101910001001D4E91023B3F1004F08BF002A22D0F0
:101920000AF0DEF8C36B3C301B689847D4E91023FB
:10193000821A61EB030393469C46D5E91A2393452B
:101940007CEB0303ACBF01250025236EAB4208D01E
:10195000064B07490748002D18BF19460CF05AF8E6
:101960002566BDE830880125EFE700BFC1BB01084F
:10197000BABB010800BF010810B5FFF77DFA0446A5
:10198000FFF738FB236E0BB9283010BD4830FCE759
:101990002DE9F74F0AF0A4F80646FFF76DFA4FF06D
:1019A000004904464FF00008FFF724FBD4E90C235C
:1019B0004B4508BF4245054607D1012384F838301E
:1019C000644B187803B0BDE8F08FFFF7D5FFF36BD9
:1019D00082461B6806F13C009847461C41F100070F
:1019E000394630460BF096FF01465B480CF012F882
:1019F000D4E904234B4508BF424505F1080B7ED1CD
:101A000056480CF007F8012384F82830D4E9042361
:101A1000B3F1004F08BF002A7AD151480BF0FAFF0A
:101A2000012384F8383094F828301BB194F8293019
:101A3000002B75D094F838301BB194F83930002B56
:101A40006ED0D4E91601B6EB000867EB01090BF084
:101A500061FF4946019040460BF072FF019B024630
:101A6000194640480BF0D6FFB5F88430002B5BD107
:101A7000D4E91001B1F1004F08BF002865D00BF088
:101A800049FF014638480BF0C5FF32463B465846F1
:101A90000BF05AFE0BF03EFF014634480BF0BAFF44
:101AA0003B46324650460BF04FFE0BF033FF0146EB
:101AB0002F480BF0AFFF02F0DBFA0AF011F890F8B4
:101AC0004C3023B12B480BF0A5FF0EF055FBFFF770
:101AD000D3F90AF005F80646FFF78CFA00213046E4
:101AE00009F00CFE0CF04EFDB5F89830003318BF2D
:101AF000012384F83A30236E4BBB1F4B61E75846F5
:101B00000BF022FE864277EB0103FFF67FAF77E70B
:101B100050460BF019FE864277EB010383DB7CE72E
:101B200016480BF077FF4BE7D5E92423904579EB76
:101B300003039DDB494640460BF002FF0146104877
:101B40000BF068FF0EF018FB92E70E499AE70E4B78
:101B500037E700BFAF0B00207DBD01088CBD010839
:101B6000A5BD0108BCBD01080EBE010826BE0108C6
:101B700040BE010857BE0108C0060020DDBD0108B7
:101B8000F0BD010877BD0108C10600202DE9F04134
:101B9000FFF772F90446FFF72DFA804609F0A0FF1F
:101BA000D4E90423C4E90223C36B3C301B68984783
:101BB000C4E90401256EFFF783FED4E90823B3F1DD
:101BC000004F08BF002A3DD0D4E9046708F108009F
:101BD0000BF0BAFD864277EB0103ACBF0123002373
:101BE00084F82830002384F82930FFF7C5FED4E9B3
:101BF0000C23B3F1004F08BF002A25D0D4E90467B5
:101C00000BF0A2FD864277EB0103ACBF012300235A
:101C100084F83830236EAB421CBF012384F838307F
:101C2000002384F83930FFF7CDF994F8282094F890
:101C300038306AB153B109480BF0ECFE084B187804
:101C4000BDE8F0810123CBE70123E1E70548F3E795
:101C50000BB10548F0E70548EEE700BF2BBD0108D2
:101C6000AC0B002045BD010856BD010865BD01084B
:101C700013B509F035FF044603689B68984723684D
:101C80002046DB6801219847236820461B694FF4F2
:101C9000FA71984723682046DB68002198470024A2
:101CA00001234FF49672CDE90034074923460748D3
:101CB00000F0C8F800F0B6FA40F24521044802F0FE
:101CC000A7FA204602B010BD14BF01085110000849
:101CD0000EB90108FF23024A1370024A13707047BD
:101CE000C0060020C1060020064A13681968064B8A
:101CF00019B94FF0FF321A6070471268D268D26883
:101D00005268F8E7C80600207807002010B504469E
:101D100020B940F2F261084802F07AFA6269074B92
:101D20009A4207D1A06A064B984203D0B0FA80F0DD
:101D3000400910BD0020FCE70EB9010898070020FB
:101D400080070020F8B51B4B1B4E1C680546306809
:101D50000F46043001F0E9FA334640B901203168FA
:101D6000164EC96A3268884022EA000232606A1C54
:101D700007D137B1196812480431BDE8F84001F0C5
:101D8000B1BA1A686419546007D30E4A106819680A
:101D9000BDE8F840043101F0B1BA0B4A1068196887
:101DA000043101F0ABFA094B1A68A24288BF1C60EB
:101DB000F8BD00BFC0070020C4060020480700206F
:101DC00098070020CC060020C806002078070020D5
:101DD00080B5DFF86C80164F164D174E2B6863B92F
:101DE000164B1B68012BF8D94FF08053C8F8003010
:101DF000BFF34F8FBFF36F8FEEE701F0FBFAFB6885
:101E0000DC68201D01F091FA3368013B33602B68D8
:101E1000013B2B6001F00EFB04F1540016F07CF83E
:101E2000206B01F029FC204601F026FCD6E700BF1C
:101E3000AC0700203807002034070020D00600201F
:101E400004ED00E02DE9F84F4FEA820A8046504643
:101E50000D4699460B9E01F00DFC0746002800F048
:101E6000B780BC2001F006FC0446002800F0AD80DD
:101E7000076325B94FF458715C4802F0C9F952461E
:101E8000A521206B15F09FF9236BAAF1040A9A444F
:101E90002AF0070A6B1E04F134020F3513F8011FF4
:101EA00002F8011B197809B1AB42F7D10A9D4FF036
:101EB000000B042D28BF0425271DE562C4E9135B30
:101EC000384684F843B001F00AFAC5F1050504F17B
:101ED000180001F004FAC4F8B4B060225946246135
:101EE000A561646284F8B8B004F1540015F06BF990
:101EF0003F4B4A46A3653F4B4146E3653E4B504648
:101F0000236601F051FA206006B1346001F072FAE4
:101F10003A4B3B4E1A68DFF8248101321A6032686E
:101F2000002A58D134601B68012B25D1354801F0B7
:101F3000CBF9354801F0C8F9344801F0C5F9DFF8AC
:101F40000091334801F0C0F9324D334801F0BCF93B
:101F5000484601F0B9F9284601F0B6F92F4801F0DA
:101F6000B3F92F4801F0B0F92E4801F0ADF92E4B2E
:101F7000C3F800902D4B1D6001252D4A2D49136893
:101F8000086801331360E26A636405FA02F30343ED
:101F900014200B601B4B394600FB023001F0A2F904
:101FA00001F048FAD8F8003063B13368DA6AE36ABE
:101FB0009A4207D24FF080521F4B1A60BFF34F8FE7
:101FC000BFF36F8F2846BDE8F88F384601F054FB09
:101FD0004FF0FF35F6E7D8F80030002BCCD133684E
:101FE000DA6AE36A9A4298BF3460C5E70EB901081D
:101FF00044EE010864EE010824EE010834070020D5
:10200000C4060020D0060020E4060020F8060020C8
:102010000C07002060070020200700208007002018
:10202000AC07002098070020C8060020CC0600203E
:10203000440700204807002004ED00E0940700203A
:102040004C07002070B504462A4D01F0D3F904B9BD
:102050002C68261D304601F068F960B91421E06A49
:10206000254B41435B5833B90122244982400B6818
:1020700023EA02030B60A36A1BB104F1180001F00C
:1020800054F91F4A1368013313602B68A34220D10F
:1020900031461C4801F026F91B4A136801331360CE
:1020A00001F0C8F9194B1B6893B12B68A3420FD1FB
:1020B000174B1B6823B140F2B641164802F0A8F84E
:1020C0004FF08052144B1A60BFF34F8FBFF36F8FE6
:1020D00070BD124A04F154001368013B136015F0FF
:1020E0001BFF206B01F0C8FA204601F0C5FAFFF78C
:1020F000FBFDD5E7C4060020D006002048070020DD
:1021000044070020AC070020380700209407002077
:10211000400700200EB9010804ED00E0340700205C
:10212000F8B5054620B940F24C51174802F070F856
:10213000164B1B68AB4220D001F05CF9144B6C6964
:102140001F68144B1E6801F075F9BC4217D0B442E9
:1021500015D0114B9C4208D1AB6A83B995F8B830C1
:10216000012B0CBF02200320F8BD0C4B9C4208D071
:10217000002C0CBF04200120F6E70020F4E7022029
:10218000F2E70420F0E700BF0EB90108C406002002
:10219000C8060020CC06002098070020AC070020CD
:1021A00070B5044620B940F21C71194802F030F8AD
:1021B000184D2B68A34229D044B301F01BF92046E7
:1021C000FFF7A4FDF0B1261D304601F0AEF8012363
:1021D0001149E26A08689340034314200B600F4BD7
:1021E000314600FB023001F07DF82B68E26ADB6AC1
:1021F0009A4207D34FF08052094B1A60BFF34F8FBA
:10220000BFF36F8FBDE8704001F014B970BD00BF1F
:102210000EB90108C406002048070020D00600209F
:1022200004ED00E013B500241A4B009401935022F2
:10223000234619491948FFF705FE01281DD100F072
:10224000BBFE012819D14FF0500383F31188BFF36F
:102250006F8FBFF34F8F124B124A1B6854331360BA
:102260004FF0FF32104B1A60104B1860104B1C607F
:1022700002B0BDE8104001F03DB9013007D140F691
:1022800004010C4802B0BDE8104001F0C1BF02B02B
:1022900010BD00BF740700201DBF0108D11D00083C
:1022A000C4060020D40200207807002094070020F4
:1022B000C00700200EB90108024A136801331360F9
:1022C000704700BF40070020014B1868704700BFEF
:1022D000C007002008B501F067F9014B186808BD78
:1022E000C0070020014B1868704700BF340700206A
:1022F0002DE9F84F3A4B1B68002B6AD1394B1C680B
:1023000001341C609CB9384D2B681B6823B140F622
:102310006221364801F07CFF354B2A681968296034
:102320001A60344A136801331360FFF7DDFC324D45
:102330004FF0000B2B68314FA34211D93A68304B54
:10234000D16A14224A439A58022A28BF4FF0010B3F
:102350002C4A1268002A0CBF58460120BDE8F88FAD
:10236000DFF884A0DFF8A490DAF8002012681AB928
:102370004FF0FF322A60E1E7DAF80020D268D66831
:1023800071688C4201D22960D8E706F10408404602
:1023900000F0CBFFB16A19B106F1180000F0C5FFDB
:1023A00001224FF0140CF06AD9F8003002FA00F163
:1023B0001943134BC9F800100CFB0030414600F0E4
:1023C00091FF3868F16AC26A914228BF4FF0010B51
:1023D000CAE70D4A4FF0000B136801331360B7E7EB
:1023E00040070020C0070020C80600200EB90108E1
:1023F000CC0600207C07002078070020C4060020BF
:10240000D0060020C40700203C0700204807002019
:102410002DE9F8432E4C236823B940F668012D4876
:1024200001F0F6FE00F0E6FF2368013B236024681C
:102430002CB1002400F0FEFF2046BDE8F883264BB7
:102440001B68002BF5D0254D254EDFF8A8801FE036
:10245000EB680127DC6804F1040904F1180000F0BE
:1024600064FF484600F061FF1420E26A316807FA11
:1024700002F30B4300FB02804946336000F032FF59
:10248000184BE26A1B68DB6A9A4201D3164B1F6045
:102490002B68002BDCD10CB1FFF726FC134D2C6808
:1024A00044B10127104EFFF723FF00B13760013C14
:1024B000F9D12C600C4B1B68002BBAD04FF0805226
:1024C0000B4B1A60BFF34F8FBFF36F8F0124B1E73F
:1024D000400700200EB901083407002080070020C3
:1024E00048070020C4060020C40700203C07002045
:1024F00004ED00E0D006002038B50C46054620B9B2
:1025000040F2CA41184801F083FE24B940F2CB41A1
:10251000154801F07DFE154B1B6823B140F2CC41FC
:10252000114801F075FEFFF7C7FE114B2A681868C5
:1025300014192CBF0121002182422C600CD961B9F1
:10254000FFF766FF38B94FF080520A4B1A60BFF3AD
:102550004F8FBFF36F8F38BD09B9A042F0D2002171
:10256000201AFFF7EFFBEBE70EB901084007002048
:10257000C007002004ED00E010B5044640B94FF05C
:1025800080520D4B1A60BFF34F8FBFF36F8F10BD9A
:102590000A4B1B6823B14FF4A461094801F038FECF
:1025A000FFF78AFE00212046FFF7CCFBFFF730FF44
:1025B0000028E4D0EBE700BF04ED00E04007002076
:1025C0000EB90108244B70B51A68244B12B10122D0
:1025D0001A6070BD224E1A6033681B6B1A68B2F124
:1025E000A53F0BD15A68B2F1A53F07D19A68B2F165
:1025F000A53F03D1DB68B3F1A53F04D03068316853
:10260000343101F0D5FD174B1C68B4FA84F414235F
:10261000E4B2C4F11F046343134DEB5823B940F6F1
:102620008831124801F0F4FD142202FB04F3E9188A
:102630004868083340682B44984202FB045408BFA2
:102640004368486008BF4B606368094ADB683360D1
:10265000336854331360BCE740070020C4070020F0
:10266000C406002048070020D00600200EB901084B
:10267000D402002070B504462A4E00F0BBFE04B917
:102680003468251D284600F050FE60B91421E06A28
:10269000254B41435B5833B90122244982400B68E2
:1026A00023EA02030B60A36A1BB104F1180000F0D7
:1026B0003CFE29461E4800F015FE94F8B8301D4D2A
:1026C000012B04BF002384F8B83000F0B3FE2A6861
:1026D0002AB100F08FFEFFF707FB00F0ABFE336876
:1026E000A34211D12B6883B1134B1B6823B14FF464
:1026F000D961124801F08CFD4FF08052104B1A60E6
:10270000BFF34F8FBFF36F8F70BD094A11680D4A39
:102710001268914201D13360F6E7BDE87040FFF7DF
:1027200051BF00BFC4060020D0060020480700208B
:102730009807002094070020400700200EB90108E8
:1027400004ED00E03407002038B50D46044620B9FA
:1027500040F69F31074801F05BFD074B20461968A2
:10276000183100F0CBFD2846BDE838400121FFF7C5
:10277000E9BA00BF0EB90108C406002070B50E46C4
:102780001446054620B940F6CA310A4801F040FD1A
:10279000094B28461968183100F0A4FD002C214689
:1027A00008BF3046BDE8704018BF4FF0FF30FFF75C
:1027B000C9BA00BF0EB90108C406002038B5C36805
:1027C000DC6824B940F6FA31154801F021FD04F126
:1027D0001805284600F0A9FD124B1B68E3B9251D1A
:1027E000284600F0A2FD01230F49E26A08689340E1
:1027F000034314200B6029460C4B00FB023000F011
:1028000071FD0B4BE26A1B68DB6A9A4285BF0120AF
:10281000084B0020186038BD29460748EFE700BF85
:102820000EB901084007002048070020D00600200C
:10283000C4060020C407002080070020034B1B684B
:102840000360034B1B684360704700BF7C07002098
:10285000C007002070B50C46054620B940F665411A
:10286000144801F0D5FC24B940F66641114801F046
:10287000CFFC00F0BFFD104B1A682368591C0FD025
:102880000E482E6800686968864201D091420ED9D0
:10289000521A934209D99B1A23602846FFF7CEFFAC
:1028A000002400F0C7FD204670BD002323600124F2
:1028B000F7E700BF0EB90108C00700207C07002021
:1028C0000122014B1A607047C407002070B50C4606
:1028D0001646054608B91B4A156805F134026260C0
:1028E000EA6A052B22612A6B2560E2616A6CA260AC
:1028F000EA6C62614FF00002A2611BD011490968C5
:10290000A9420BD12273D6B1296B0A46531A12F889
:10291000010BA528FAD09B08238470BD032B2373D9
:10292000F1D1FFF7C9FCAB6A0BB102232373FFF7A8
:102930006FFDE8E72846FFF7F3FB2073E3E7268403
:10294000EBE700BFC40600202DE9F84F0D68814673
:102950000C4692461DB300254FF0240B4B6801F145
:1029600008075B68BB424B6004BFCB684B604B6899
:10297000D3F80C8063680BFB05915B6801229F42D2
:10298000636008BFE36805F1010508BF6360636821
:10299000DE6853463046FFF799FFB045EAD1284636
:1029A000BDE8F88F2DE9F84305461746FFF784FC8C
:1029B0001F4B1B688B4238D84FF000082426444632
:1029C000DFF8809009EB080106FB04500122FFF7B5
:1029D000BBFFA8F1140818F1640F0444F2D1154BA1
:1029E0000222196806FB0450FFF7AEFF124B0444A5
:1029F0001968022206FB0450FFF7A6FF04440422D4
:102A00000E4906FB0450FFF79FFF044406FB0450E9
:102A100003220B49FFF798FF04440FB100233B60EA
:102A2000FFF7F6FC2046BDE8F8830024F8E700BF76
:102A300034070020C8060020CC060020AC07002088
:102A40009807002020070020014B1868704700BF3E
:102A5000C4060020054B1B6833B1054B1B68002BD7
:102A60000CBF02200020704701207047940700200F
:102A7000400700202DE9F0410446002836D0234AC3
:102A8000C36A11681746C96A8B4237D21426826915
:102A90001F4D002AA8BF3A6806FB0353A2BFD26AA3
:102AA000C2F10502826142699A4221D100F1040813
:102AB000404600F03AFC174B48B9E06A4643AA5931
:102AC0002AB901211A68814022EA01021A603A6893
:102AD0001968D26AE262012404FA02F0084318601D
:102AE0001420414600FB025000F0FCFB204603E0AE
:102AF0003B68DB6AC3620120BDE8F0811368C06CEB
:102B0000DC6AA0422CBF00200120F5E7C4060020AB
:102B1000D006002048070020F8B5044608B9002078
:102B2000F8BD1F4B1B68834204D040F67A711D48E4
:102B300001F06EFB236D23B940F67B71194801F05B
:102B400067FB236DE16AE26C013B91422365E6D0AD
:102B5000002BE4D1251D284600F0E7FB124E134A56
:102B600050B91421E76A794373582BB901201368CF
:102B7000B84023EA00031360E36CC3F10501A161CF
:102B8000E3620124116804FA03F008431060142082
:102B9000294600FB036000F0A5FB2046C0E700BF0C
:102BA000C40600200EB90108D00600204807002006
:102BB000F8B50D460446002845D0036D23B940F60C
:102BC000C971214801F024FBE36C9D4238BF1D46CA
:102BD000E36AAB4237D0236D012B34D11B4B1B680A
:102BE000A34204D140F6E471174801F011FB14260A
:102BF000A269E36A002AE562A4BFC5F10505A561E3
:102C0000134D626906FB03539A421CD1271D3846B7
:102C100000F08BFBE26A0F4C40B95643AB592BB91D
:102C200001212368914023EA01032360012314203A
:102C3000216893400B432360394600FB0250BDE8F6
:102C4000F84000F04FBBF8BD0EB90108C4060020E3
:102C5000D006002048070020044B1A681AB11968F2
:102C60000A6D01320A651868704700BFC40600206B
:102C70002DE9F041214C1E4680460F46154600F0D6
:102C8000B9FB236893F8B830022B16D001212368D2
:102C9000D3F8B42022EA0802C3F8B420236883F8EA
:102CA000B81056B13046FFF74DF84FF08052144B34
:102CB0001A60BFF34F8FBFF36F8F00F0BBFB00F0C4
:102CC00099FB1DB12368D3F8B4302B602368002230
:102CD00093F8B830022B09BF012500252368D3F8EB
:102CE000B41004BFB943C3F8B410236883F8B82004
:102CF00000F0A0FB2846BDE8F08100BFC40600201C
:102D000004ED00E0F8B50E4617461D46044620B90E
:102D100041F219212E4801F07BFA00F06BFB15B14E
:102D2000D4F8B4302B60022394F8B85084F8B8304B
:102D3000EDB2042F1AD8DFE807F00E0309061500DC
:102D4000D4F8B4301E43C4F8B46004E0D4F8B4300E
:102D50000133C4F8B430012D12D0012400F06AFB15
:102D60002046F8BD022DEED10024F7E7D4F8B430A8
:102D70000133F0D041F24A21154801F049FAEAE75F
:102D8000261D304600F0D1FA1420124AE36A116879
:102D90009D400D431560104A314600FB032000F0B2
:102DA000A1FAA36A23B141F25921094801F030FA8E
:102DB0000A4BE26A1B68DB6A9A42CED94FF0805216
:102DC000074B1A60BFF34F8FBFF36F8FC5E700BF8C
:102DD0000EB9010848070020D0060020C4060020D4
:102DE00004ED00E02DE9F843DDF820800E46914621
:102DF0001D46044620B941F28C21384801F008FAFA
:102E000000F0D2FBEFF311874FF0500383F31188EA
:102E1000BFF36F8FBFF34F8F15B1D4F8B4302B6071
:102E2000022394F8B85084F8B830EDB2B9F1040F29
:102E30001AD8DFE809F00E0309061500D4F8B430FB
:102E40001E43C4F8B46004E0D4F8B4300133C4F8CD
:102E5000B430012D12D0012087F31188BDE8F8832A
:102E6000022DEED10020F7E7D4F8B4300133F0D0D2
:102E700041F2CF21194801F0CBF9EAE7A36A23B167
:102E800041F2DA21154801F0C3F9154B1B6803BB69
:102E9000251D284600F049FA01231249E26A086814
:102EA0009340034314200B6029460F4B00FB023074
:102EB00000F018FA0D4BE26A1B68DB6A9A42CAD925
:102EC0000123B8F1000F01D0C8F80030084A1360A0
:102ED000C1E704F118010748EAE700BF0EB901088D
:102EE0004007002048070020D0060020C40600202C
:102EF000C40700208007002038B5054608B9084BF4
:102F00001D68002400F076FA95F8B830022B04BF53
:102F100085F8B840012400F08DFA204638BD00BF86
:102F2000C4060020F8B50F4C00F064FA2568ADB96E
:102F30000D4F0E4E384600F0C7F9304600F0C4F988
:102F40000B4B2A461F600B4B0C210A201E6000F021
:102F50006FFC206010B1084901F02EF8BDE8F84080
:102F600000F068BAFC070020D0070020E40700202A
:102F7000C8070020CC07002022BF0108914208B5F5
:102F8000416000610AD8D21A83699A420DD2084B77
:102F9000011D186800F0B2F9002008BD9A4201D264
:102FA000994202D2011D034BF3E70120F5E700BF70
:102FB000CC070020C807002007B5FFF7B3FF0C4B74
:102FC0001B6843B90B484FF4897101F021F90020C7
:102FD00003B05DF804FB084BC822019301230749A5
:102FE000009307480023FEF72DFF0028EAD0EFE703
:102FF000FC0700200EB901080008002027BF0108C7
:103000001D3100082DE9F04180462C200D46174661
:103010001E4600F02FFB044688B125B94FF4B67167
:10302000084801F0F5F8FFF77DFF069BC4F8008023
:10303000C4E9065726626362201D00F050F920465D
:10304000BDE8F0810EB901082DE9FF410D4690461B
:103050001F46064620B94FF4C3710F4801F0D8F857
:103060000E4C206878B1052DCDE9015803960DDC92
:10307000FFF7F0FC002302280CBF0A9A1A4601A9A8
:10308000206800F0F9FB04B0BDE8F08100233A4667
:1030900001A900F0A7FCF6E70EB90108FC07002023
:1030A0002DE9F74300271A4DDFF86C802B681A686A
:1030B00032B9184A11681360296003B0BDE8F08383
:1030C000DB68DC681E6804F10409484600F02DF94D
:1030D000636A20469847E369012BE7D1A36933442B
:1030E0009E4206D2636024614946286800F006F9D2
:1030F000DCE700230097324619462046FFF7A4FF7D
:103100000028D3D140F27231404601F081F8CDE77A
:10311000C8070020CC0700200EB901082DE9F04FA8
:103120004FF00108624D89B0DFF898B1DBF800205C
:10313000136843B30024D368D3F80090FFF7BCF8BA
:10314000FFF7C2F85B4B82461A681F4690425A4E00
:103150001CD31860002C4CD0584B1B681A68B2FA6C
:1031600082F25209A9EB0A01306800F05DFFFFF717
:103170004FF998B94FF08052514B1A60BFF34F8FFF
:10318000BFF36F8F0AE001249946D7E70393FFF757
:1031900087FF039BC3F800A0FFF73AF9002205A9B7
:1031A000306800F0C3FC0028BED0059B002BF5DB87
:1031B000079C636913B1201D00F0B7F8FFF784F88E
:1031C0003B688146984201D2FFF76AFF059BC7F82A
:1031D0000090092BE2D808FA03F313F4047A57D1CC
:1031E00013F0C70F33D19B06D8D5204600F044FA20
:1031F000D4E7814529D8FFF70BF9DBF80030DB680D
:10320000D3F80CB00BF1040000F08FF8DBF81C30A1
:10321000012B15D1DBF818104B465246494458464D
:10322000FFF7ACFE60B1009423464A46214658465B
:10323000FFF70AFF20B94FF4F471284600F0E8FFC9
:10324000DBF8243058469847A8E722468AE7A16968
:10325000069B4A4619442046FFF790FE00289DD061
:10326000636A20469847E369012B97D1A2690699C2
:10327000CDF800A00A44534651462046FFF7E4FE2D
:1032800000288BD140F20131284600F0C1FF85E7CC
:10329000069BA36123B94FF44671284600F0B8FF9E
:1032A000A1694B464A4649442046FFF767FE75E749
:1032B0000EB90108F8070020FC070020CC07002009
:1032C00004ED00E0C80700204FF0FF3200F10803D2
:1032D0004360C0E9022303610023036070470023B9
:1032E0000361704743689A684B608A609A685160CE
:1032F0009960036808610133036070470A6830B55C
:10330000531C0AD103695A684A6091608B60596006
:10331000036808610133036030BD00F108035C6895
:1033200025689542EFD82346F9E70369D0E90112F1
:103330008A60826851605968814208BF5A600022E1
:1033400002611A68013A1A601868704706480068F6
:10335000006880F3088862B661B6BFF34F8FBFF391
:103360006F8F00DF00BF000008ED00E0002307B50D
:1033700001930B4B1B68013303D0CA21094800F0AD
:1033800047FF4FF0500383F31188BFF36F8FBFF3F4
:103390004F8F019B002BFCD003B05DF804FB00BFF6
:1033A000040000200EB901084FF0807340F8043C7F
:1033B000054B21F0010140F8081C40F80C3C40F896
:1033C000202C4038704700BF6D330008000000001B
:1033D000074B19680868B0E8F00F80F30988BFF35D
:1033E0006F8F4FF0000080F311884EF00D0E704784
:1033F000C40600204FF0500383F31188BFF36F8F92
:10340000BFF34F8F084A13680133012B136009D1B2
:10341000064B1B6813F0FF0F04D040F275110448EF
:1034200000F0F6BE704700BF0400002004ED00E08D
:103430000EB9010810B5074C236823B94FF4BE71CB
:10344000054800F0E5FE2368013B23600BB983F3D8
:10345000118810BD040000200EB901080000000012
:10346000EFF30980BFF36F8F0D4B1A6820E9F00F5F
:1034700010602DE908404FF0500080F31188FFF7ED
:10348000A1F84FF0000080F31188BDE808401968EA
:103490000868B0E8F00F80F30988BFF36F8F7047BA
:1034A000C406002008B54FF0500383F31188BFF322
:1034B0006F8FBFF34F8FFEF71BFF18B14FF0805295
:1034C000024B1A60002383F3118808BD04ED00E06D
:1034D0000022054B05491A600A6041F26701044A5F
:1034E000116007221A60704710E000E018E000E069
:1034F00014E000E013B5264B264C1A78D2B20192A4
:10350000FF221A701B78244ADBB28DF803309DF835
:10351000033003F0500313700723002223609DF84B
:103520000310581E090629D402B123602368032B17
:1035300004D04FF49B71194800F06AFE2368144AC6
:103540001B0203F4E06323600024019BDBB21370D1
:10355000134B1A6842F470021A601A6842F0704203
:103560001A60FFF7B5FF0F4B1C60FFF7EFFEFFF788
:1035700029F8FFF7FBFE204602B010BD9DF803308E
:1035800001225B00DBB28DF803300346C7E700BFC2
:1035900000E400E008080020040800200EB901083B
:1035A00020ED00E00400002008B5EFF305830F2BA9
:1035B0000AD90D4A9B5C0D4A12789A4204D940F20E
:1035C000A5210B4800F024FE0A4B0B4A1B68126829
:1035D00003F4E063934206D9BDE8084040F2B52108
:1035E000034800F015BE08BDF0E300E00408002029
:1035F0000EB901080CED00E00808002070B50D467A
:103600000646FEF759FE0D4B0D491C6862198A42A9
:1036100007D90C233360FEF7FBFE4FF0FF34204642
:1036200070BD1A60074A13685B1B1360064A136873
:103630002B441360FEF7ECFEF1E700BF080000200A
:10364000D46800200C0000200C08002008B5EFF31F
:1036500005831BB1C221034800F0DAFDBDE8084034
:10366000FEF72ABE0EB90108FEF7D2BEFEF724BE51
:10367000FEF7CEBE13F044BD13F04ABD00B58BB0CB
:10368000684614F03DF8034B08981B6818440BB0CB
:103690005DF804FB0C00002000207047704710B557
:1036A0000446FFF7A7FEA46BFFF7C4FEB4FA84F04C
:1036B000400910BD70B51546026C0446866B42B9D0
:1036C00005689DB98068FFF727FAA5600136A663F3
:1036D00070BD6DB9406813F052FD6368226C1344ED
:1036E000A2686360934201D3236863600020EDE722
:1036F000C06813F044FD236CE2685B4221681A4401
:103700008A42E2603EBFA2689B18E360022DEDD1C1
:103710000EB1013EEAE73046D8E703461A6C10B412
:10372000084662B1D9689C681144A142D96028BF9B
:10373000196810BC28BFD960D96813F020BD10BC2F
:10374000704770B50446FFF755FE94F8455004F1F4
:1037500024066DB2002D14DCFF2384F84530FFF7FA
:1037600069FEFFF747FE94F8445004F110066DB26D
:10377000002D12DCFF2384F84430BDE87040FFF7D1
:1037800059BE636A002BE7D03046FFF717F808B13F
:10379000FFF796F8013D6DB2DCE72369002BE9D015
:1037A0003046FFF70BF808B1FFF78AF8013D6DB21C
:1037B000DEE7000038B50D46044620B940F203119B
:1037C000194800F025FDFFF715FED4E90F314B43F2
:1037D0002268D0185B1A1344A060E3600020FF2326
:1037E000A063626084F8443084F8453095B9236959
:1037F00063B104F11000FEF7E1FF38B14FF08052E1
:103800000A4B1A60BFF34F8FBFF36F8FFFF712FEA3
:10381000012038BD04F11000FFF756FD04F124002B
:10382000FFF752FDF2E700BF0EB9010804ED00E01A
:10383000F8B50D461746064620B94FF4BB710D4842
:1038400000F0E6FC05FB06F05030FFF713FF0446DE
:1038500048B155B92060C4E90F6501212046FFF742
:10386000A9FF84F84C702046F8BD00F150030360B6
:10387000F1E700BF0EB901082DE9FF478846019224
:103880001E46044620B940F2F1214B4800F0C0FC2E
:10389000B8F1000F06D1236C23B140F2F221464863
:1038A00000F0B6FC022E07D1E36B012B04D040F2EE
:1038B000F321414800F0ACFCFFF7CCF830B9019B94
:1038C00023B140F2F6213C4800F0A2FC0027B946A3
:1038D000DFF8E8A0FFF78EFDA26BE36B9A4201D3FD
:1038E000022E19D1324641462046FFF7E3FE636AB5
:1038F0001BB104F12400FEF761FF38B14FF0805294
:103900002E4B1A60BFF34F8FBFF36F8FFFF792FDFF
:10391000012004B0BDE8F087019D1DB9FFF78AFDC5
:103920000020F6E717B902A8FEF788FFFFF782FD2F
:10393000FEF7C2FCFFF75EFD94F84430FF2B08BF92
:1039400084F8449094F84530FF2B08BF84F84590E4
:10395000FFF770FD01A902A8FEF77CFF28BBFFF767
:1039600049FDA26BE36B9A420ED1FFF763FD01990B
:1039700004F11000FEF7E8FE2046FFF7E2FEFEF736
:1039800047FD48B10127A5E7FFF754FD2046FFF7A3
:10399000D8FEFEF73DFDF5E74FF08053CAF8003042
:1039A000BFF34F8FBFF36F8FECE72046FFF7C9FEE1
:1039B000FEF72EFDB4E700BF0EB9010804ED00E0EC
:1039C00010B5024600210120FFF732FF044638B14E
:1039D000002383600360C3601A461946FFF74CFF5B
:1039E000204610BD2DE9F843894690461F460446FF
:1039F00020B940F2C331274800F00AFCB9F1000FAA
:103A000006D1236C23B14FF47171224800F000FC01
:103A1000022F07D1E36B012B04D040F2C5311D48C2
:103A200000F0F6FBFFF7C0FDEFF311864FF05003F7
:103A300083F31188BFF36F8FBFF34F8FA26BE36BDC
:103A40009A4201D3022F22D194F845503A466DB2E2
:103A500049462046FFF72EFE6B1C13D1636A0BB953
:103A600001200BE004F12400FEF7A8FE0028F7D0A7
:103A7000B8F1000FF4D00120C8F8000086F31188D7
:103A8000BDE8F88301356DB284F84550E8E70020C1
:103A9000F4E700BF0EB9010870B50D46044620B921
:103AA0004FF48C61204800F0B3FB236C23B140F24B
:103AB00064411D4800F0ACFB236833B9A36823B10F
:103AC00040F26941184800F0A3FBFFF76DFDEFF3EA
:103AD00011864FF0500383F31188BFF36F8FBFF34C
:103AE0004F8FA26BE36B93421CD994F8453001329F
:103AF0005BB2A2635A1C10D1636A0BB9012009E0C2
:103B000004F12400FEF75AFE0028F7D0002DF5D06E
:103B10000120286086F3118870BD01335BB284F800
:103B20004530EBE70020F5E70EB901082DE9F04339
:103B300085B00F460192044620B94FF4A061424877
:103B400000F066FB37B9236C23B140F204513E48C4
:103B500000F05EFBFEF77EFF30B9019B23B140F21F
:103B60000951394800F054FB0026B046DFF8DC90DC
:103B7000FFF740FCA56BD5B139462046013DFFF764
:103B8000CCFDA563236963B104F11000FEF716FEB6
:103B900038B14FF080522D4B1A60BFF34F8FBFF3F7
:103BA0006F8FFFF747FC012005B0BDE8F083019D52
:103BB0001DB9FFF73FFC0020F6E716B902A8FEF793
:103BC0003DFEFFF737FCFEF777FBFFF713FC94F899
:103BD0004430FF2B08BF84F8448094F84530FF2B15
:103BE00008BF84F84580FFF725FC01A902A8FEF76D
:103BF00031FEF0B92046FFF752FDA0B1019904F162
:103C00002400FEF7A1FD2046FFF79BFDFEF700FC18
:103C100038B94FF08053C9F80030BFF34F8FBFF36E
:103C20006F8F0126A4E72046FFF78BFDFEF7F0FB20
:103C3000F7E72046FFF785FDFEF7EAFB2046FFF792
:103C40002EFD0028EDD0B6E70EB9010804ED00E026
:103C50002DE9FF410446019120B940F291515248AB
:103C600000F0D6FA236C23B140F295514E4800F093
:103C7000CFFAFEF7EFFE30B9019B23B140F29A5123
:103C8000494800F0C5FA00252F462E46DFF81C8172
:103C9000FFF7B0FBA36BE3B1013BA363236813B948
:103CA000FEF7DAFFA060236963B104F11000FEF7AC
:103CB00085FD38B14FF080523C4B1A60BFF34F8FF7
:103CC000BFF36F8FFFF7B6FB0125284604B0BDE8B0
:103CD000F081019B4BB925B140F2E151324800F02F
:103CE00097FAFFF7A7FB0025EFE717B902A8FEF741
:103CF000A5FDFFF79FFBFEF7DFFAFFF77BFB94F8CC
:103D00004430FF2B08BF84F8446094F84530FF2B03
:103D100008BF84F84560FFF78DFB01A902A8FEF7F4
:103D200099FD40BB2046FFF7BAFCF0B123683BB9D0
:103D3000FFF760FBA068FEF79DFE0546FFF77AFBE4
:103D4000019904F12400FEF7FFFC2046FFF7F9FC7F
:103D5000FEF75EFB38B94FF08053C8F80030BFF370
:103D60004F8FBFF36F8F012792E72046FFF7E9FCE3
:103D7000FEF74EFBF7E72046FFF7E3FCFEF748FBB4
:103D80002046FFF78CFC0028EDD0002D9DD0FFF7DA
:103D900031FB616A19B1236B1968C1F10501A06893
:103DA000FEF706FF9DE700BF0EB9010804ED00E035
:103DB0002DE9F04385B00F460192044620B94FF437
:103DC000CD61424800F024FA37B9236C23B140F2A8
:103DD0006C613E4800F01CFAFEF73CFE30B9019BD6
:103DE00023B140F27161394800F012FA0026B04662
:103DF000DFF8DC90FFF7FEFAA36BD3B1394620461B
:103E0000E568FFF78AFC636AE56063B104F12400AA
:103E1000FEF7D4FC38B14FF080522D4B1A60BFF33F
:103E20004F8FBFF36F8FFFF705FB012005B0BDE893
:103E3000F083019D1DB9FFF7FDFA0020F6E716B9E2
:103E400002A8FEF7FBFCFFF7F5FAFEF735FAFFF7DD
:103E5000D1FA94F84430FF2B08BF84F8448094F8DA
:103E60004530FF2B08BF84F84580FFF7E3FA01A92E
:103E700002A8FEF7EFFCF0B92046FFF710FCA0B156
:103E8000019904F12400FEF75FFC2046FFF759FC7E
:103E9000FEF7BEFA38B94FF08053C9F80030BFF3CF
:103EA0004F8FBFF36F8F0126A4E72046FFF749FC31
:103EB000FEF7AEFAF7E72046FFF743FCFEF7A8FA55
:103EC0002046FFF7ECFB0028EDD0B6E70EB901085D
:103ED00004ED00E02DE9F84389469046054620B9F7
:103EE00040F2FB61204800F093F9B9F1000F06D1D0
:103EF0002B6C23B140F2FC611B4800F089F9FFF7FD
:103F000053FBEFF311874FF0500383F31188BFF396
:103F10006F8FBFF34F8FAC6B1CB395F8446049466D
:103F200076B22846FFF7F9FB013C731CAC6313D152
:103F30002B690BB901200BE005F11000FEF73EFCE8
:103F40000028F7D0B8F1000FF4D00120C8F8000025
:103F500087F31188BDE8F883013676B285F84460AE
:103F6000E8E72046F4E700BF0EB9010810B50446A3
:103F700020B940F28A71054800F04AF9FFF73AFA91
:103F8000A46BFFF757FA204610BD00BF0EB9010819
:103F900038B5054620B940F2A471064800F038F95A
:103FA000FFF728FAA86BEC6B241AFFF743FA2046B8
:103FB00038BD00BF0EB90108002330B5064A52F8DB
:103FC000335002EBC3041DB942F83310606030BDBA
:103FD0000133052BF3D1FAE7E4170020002310B5D5
:103FE000074A02EBC3014C68844204D1002042F826
:103FF0003300486010BD0133052BF2D1FAE700BF52
:10400000E417002010B5044620B94FF4F8610548C4
:1040100000F0FEF82046FFF7E1FF2046BDE8104023
:10402000FFF72ABB0EB9010870B504460D461646C7
:10403000FFF7E0F994F84430FF2B04BF002384F825
:10404000443094F84530FF2B04BF002384F84530FA
:10405000FFF7F0F9A36B2BB93246294604F124008F
:10406000FEF78CFB2046BDE87040FFF76ABB0000FE
:104070002DE9F04741488AB009F0CCFCFEF732F94F
:104080002425079007993E4809F0C4FC0798684327
:1040900009F05CFD04463B4809F0BCFC94B107996B
:1040A0000DEB05022046FEF77DFC0023DFF8F0A0B3
:1040B000354F07900893089A079B9A421DD32046D4
:1040C00009F02EFDFFF7DAFA0446FFF7E5FA21467C
:1040D00002462E4809F09EFC2D4B2E4819889A88DE
:1040E0008B1A09F097FC2C4B1B6803B198472B489F
:1040F00009F090FC0AB0BDE8F087089B05FB03437C
:104100001B7B042B98BF1AF80320099B88BF3F2212
:10411000642B83BF6420B3FBF0F30899002382BFB4
:1041200005FB01418969B1FBF3F308990898DDF8B3
:1041300020C0DDF820E0DDF82080DDF8209005FBD0
:10414000004005FB0949D9F81C6005FB0141CDE998
:10415000033605FB08439B69029305FB0E439B68EE
:10416000019305FB0C431B8C009303694968384697
:1041700009F050FC089B013308939CE734BF010809
:1041800040BF01084BBF010880BF0108B2BF010852
:104190000C180020D1BF01088808002041C6010882
:1041A0002FBF0108014B1860704700BFA408002012
:1041B00073B5124C064623780D46114A1BB9137885
:1041C0000BB172B6FEE70123002113700D48642283
:1041D00012F0F9FF2B4600960B4A6421094813F0B0
:1041E000F7FE0A4B1B6803B198470125054E304680
:1041F00009F054FC72B62570F9E700BF8008002072
:10420000140800201608002008C00108A408002097
:10421000F7B5184C064623780D46174A1BB9137894
:104220000BB172B6FEE7012300211370134864221C
:1042300012F0C9FF2B460096114A64210F4813F073
:10424000C7FE104B1B680BB10C4898470E4B1B6800
:1042500003B198470125094E0C4F304609F01EFC6A
:10426000384609F01BFC72B6094B257000BF013BB4
:10427000FCD1F2E781080020150800201608002074
:1042800030C0010810080020A40800203FC0010829
:10429000FFFF0F00F8B5DFF898C003681A4FCCF89D
:1042A00000304368194E3B608368194D3360C36822
:1042B000184C2B60036918492360436982690B60BD
:1042C000164BC0691A60164A1060DCF800003868A6
:1042D0003068286820681C460968124D1968124E1B
:1042E000126864220021284612F06DFF23683246CE
:1042F0006421284613F06CFE284609F0CFFB0B4BD7
:1043000000BF013BFCD1ECE7940800209C08002092
:10431000A0080020980800207C08002084080020C5
:104320008C08002016080020F5BF0108FFFF0F00D1
:1043300090080020074B1B6803B198471EF0040F3C
:104340000CBFEFF30880EFF309808169004A104742
:1043500095420008A408002010B1012108F06CBCAF
:10436000704708B109F0F2BB704780687047406839
:1043700070474368012B08D1D0E90432934204D03E
:104380001878003018BF01207047002070474B6834
:1043900070B5042B04460E464FF0000304D0C0E96C
:1043A00000338360204670BDD1E90425AD1AC0E911
:1043B000003383602846FFF7D4FFC4E900000544BA
:1043C000A560D6E90453024629468B4205D00AB1BE
:1043D0000E78167001310132F7E75B1B18446060FC
:1043E000E0E742680346022A06D1D3E904031B1A18
:1043F000032B01D909F007BC002070474368032B49
:1044000006D1D0E904329A4208BF0023184670470B
:104410000023FBE7037870B581680446B3B1284AEE
:10442000284809F0F7FA6368022B12D12046FFF7FB
:10443000D8FF0146244809F0EDFAE1680B78002B1B
:104440003CD02248BDE8704009F0E4BA204A214837
:10445000E7E7032B05D12046FFF7D0FF01461E48B2
:10446000E9E7042B0ED100251C4ED4E90431C91A0A
:104470008D4205D2595D304609F0CCFA0135F4E79A
:104480001748D8E7012B08D12046FFF772FF1549DE
:10449000154B002818BF1946E1E700250F4ED4E957
:1044A00004239B1A9D4205D2515D304609F0B2FAB1
:1044B0000135F4E70D4809F0ADFABEE70C48C1E755
:1044C00052B70108E3C00108F7C0010819C101088B
:1044D00083C40108EDC0010867C2010807D50108BF
:1044E00001C10108DDC00108D8C0010807C10108E9
:1044F00082C40108B1F5884F2DE9F84304460F4600
:1045000002D9174808F05CFB066883689B1B994238
:1045100019D9D0F804900846FFF723FF0546034653
:10452000A9EB0608B14505D00BB132781A700136F7
:104530000133F7E72068FFF70FFF05EB080325605D
:104540003D446360A56025683DB92846C4E901552E
:10455000FFF702FF2846BDE8F8830120FBE700BF14
:104560005BC001082DE9F0410368561A9046826845
:104570000446D21A96420D4615D93046FFF7F1FE91
:1045800007460346A84505D02A7803B11A700135BD
:104590000133F7E720683E44FFF7DEFEC4E9016619
:1045A0002760BDE8F0814768481EFF1ABE420ED85A
:1045B0001A469D19A91A002904DD10F8011F02F8F6
:1045C000011BF7E7002EA8BF9B196360E9E73D4494
:1045D0001F44FA1A002A04DD10F8012F03F8012BFA
:1045E000F7E763682E461846B04505D0327800B12B
:1045F000027001360130F7E7A8EB05084344E4E711
:1046000008B509C81B1AC3F58840884202D2104673
:1046100008F0D6FA994238BF1946581805D2B0F5B5
:10462000884F28BF4FF4884008BD4FF48840FBE70F
:104630002DE9F8430C46591C204615461F46FFF746
:1046400059FF064680B14FF00003EA19294620467B
:10465000FFF788FFD4E901539D4208D00DB1002334
:104660002B706368013363603046BDE8F8831B4AF2
:1046700001212046FFF7C4FF23680746A5EB030985
:10468000FFF76FFE10EB090F1CBF002300F8093085
:10469000236880461A460146954205D009B1107834
:1046A000087001320131F7E7D31A01334344104651
:1046B00019466568954207D019B192F800C081F893
:1046C00000C001320131F5E72D1A1D44206847442E
:1046D000FFF742FEC4E90085A760C5E796C0010860
:1046E0002DE9F04105460E4661B1D0E90132D21AFA
:1046F0008A4209D300221E4403B11A700133B34227
:10470000FAD16B60BDE8F081114AFFF779FF80466E
:10471000FFF727FED5E9001407460A4603469442F0
:1047200005D00BB11078187001320133F7E7002380
:10473000641A3C44264404B123700134B442FAD1D3
:104740002868FFF709FEC5E900744744AF60D9E760
:10475000CAC10108D0E90032D21A914210B503D97A
:10476000891AFFF7BDFF10BD3CBF5B184360FAE735
:1047700070B50C46012120461646FFF7BBFE0546E4
:1047800028B101212046FFF7E5FF23681E70284667
:1047900070BD0000426808B5012A06D1BDE8084096
:1047A0000A4600F11001FFF7E3BF8168024809F0F3
:1047B00031F9002008BD00BF59C1010810B50C1A1D
:1047C000134605D001462246184612F0E3FC034684
:1047D000181910BD2DE9F0410446A2EB0108164658
:1047E000A368226808469B1A98450F4615D940468B
:1047F000FFF7B7FD05460346BE4205D00BB13A7838
:104800001A7001370133F7E72068FFF7A5FD25602F
:104810004544C4E90155BDE8F0816568AD1AA84575
:1048200004D83146FFF7CAFF6060F4E70D4429461B
:10483000FFF7C4FF636829461A468E4205D00AB1C5
:104840000878107001310132F7E7751B1D4465606F
:10485000E1E770B50E46D2E900313046C91A144678
:10486000FFF748FE054630B1D4E900124FF00003CF
:104870003046FFF7AFFF284670BD000070B5D0E9A5
:10488000043100F110060446C91A3046FFF732FE23
:10489000054640B1D4E90712914206D1A168064805
:1048A00009F0B8F80025284670BD4FF000033046E7
:1048B000FFF790FFF7E700BFB0C001082DE9F04116
:1048C0008368A2EB01081746026804469B1A9845C4
:1048D0000E4615D94046FFF744FD05460346B7424C
:1048E00005D0327803B11A7001360133F7E720683A
:1048F000FFF732FD25604544C4E90155BDE8F0816C
:104900004568AD1AA84505D839463046FFF756FF29
:104910006060F3E70D4429463046FFF74FFF6368B8
:1049200029461A468F4205D0087802B1107001312D
:104930000132F7E77D1B1D446560DFE737B50D46A3
:1049400001A8114609F080F904212846FFF7D2FD9D
:10495000044630B14FF0000302AA01A92846FFF730
:10496000ADFF204603B030BDFFF7E8BF426808B591
:10497000022A06D1BDE808400A4600F11001FFF7FF
:10498000DDBF8168024809F045F8002008BD00BF7E
:1049900091C10108FFF7EABF2DE9F0410E46002161
:1049A0001C4617468AB00DF108082022C0E9001104
:1049B00081600546404612F006FC1E2C94BF22463C
:1049C0001F223946404612F0DAFB7368013B032B85
:1049D00014D8DFE803F00230404722462F4938461A
:1049E00013F0A9FB28B122462D49384613F0A3FB4A
:1049F00040B9012229463046FFF7BAFE28460AB0E0
:104A0000BDE8F08122462749384613F094FB28B1CF
:104A100022462549384613F08EFB08B90022E9E703
:104A200000220AA941F8242D404614F0E1FA021CA4
:104A300018BF0122DEE700220AA941F8242D4046D2
:104A400014F0D6FA019B02464345D7D0294630469A
:104A5000FFF774FFD2E723463A4629463046FFF770
:104A6000E7FDCBE714F00106C8D1640821462846CB
:104A7000FFF740FD0028C1D021462846FFF76AFE17
:104A8000B442BBD0022107EB460009F0F9F8002838
:104A9000B4DB2B6898550136F2E700BFD8C0010897
:104AA0006BC00108DDC0010870C0010830B51346B5
:104AB000426885B0032A044600F110050A460FD06B
:104AC000014601A8FFF768FF204601AA2946FFF723
:104AD000C0FE04460198FFF73FFC204605B030BDFC
:104AE0002946FFF7A5FD0446F7E70000F0B50446A8
:104AF00085B0104616460F4613F015FB6268034654
:104B0000032A16D03246214601A8FFF745FFDDE90A
:104B1000011291420BD04FF000033846FFF75AFEC6
:104B200001250198FFF718FC284605B0F0BD0025C7
:104B3000F7E7441C21463846FFF7DCFC054618B968
:104B4000054808F067FFEFE74FF0000332193146E0
:104B50003846FFF707FDE7E776C001080A4600F18F
:104B60001001FFF7C3BFF8B50D4619462846164693
:104B70001F46FFF7BFFC044630B14FF00003F219A7
:104B800031462846FFF79AFE2046F8BD1346426894
:104B900010B5042A06D1BDE810400A4600F1100104
:104BA000FFF7E1BF8168024808F034FF002010BD24
:104BB00020C101082DE9F0410C4690461D460646ED
:104BC00040B139B10849184608F034F8074618B919
:104BD00030602060BDE8F0812A46414612F0CFFAED
:104BE00037602560F6E700BFEEE9010870B50546BD
:104BF00010460E46144613F096FA224603463146F6
:104C00002846BDE87040FFF7D5BF000010B50C4640
:104C100031B1044900F016FD231A5842584110BD25
:104C20000846FCE75BC3010810B500B121B906488E
:104C300008F0F0FE002010BD1AB9044AFFF7D6FFB5
:104C4000F8E70120F7E700BFE4C10108F1C101085E
:104C50002DE9F74305460E4617469846FFF7E4FF51
:104C6000C0B10F49222007F0E5FF0446A8B138463D
:104C7000FFF77BFB81463846FFF7C0FB13F053FA82
:104C80004346CDE90090074A2221204613F0A0F9BF
:104C900030602C6003B0BDE8F0833060F9E700BFFE
:104CA000EEE901081EC201082DE9F8430E469846B8
:104CB00016F8013B02F1FF3903704660C0F8089016
:104CC000044615463D214A46304612F03BFA074657
:104CD00068BB4B46182B28BF1823C4F83001A362C9
:104CE00004F10C05A26A3146284612F048FA002267
:104CF000A66AA3191A7337B1D4F83021791C04F1CC
:104D00002C0012F03CFA0022D4F83031234483F80E
:104D10002C202EB12946404600F094FCC4F8340102
:104D2000D4E901120A48BDE8F84308F0E9BE831B44
:104D3000023DED1A182B1A46A8BF1822B5F5807F40
:104D400028BF4FF48075A262C4F83051C8E700BF95
:104D500026C2010830B504460D46084B9DB00093AD
:104D6000074A084B642103A813F032F903AA294625
:104D70002046FFF73BFF1DB030BD00BF18C2010841
:104D800010C2010800C201082DE9F0431646642252
:104D900003F10C048FB00746884620461849ADF849
:104DA000042013F0AEF970B9336B23B1154A3221E8
:104DB00001A813F00DF901AA41463846FFF716FF86
:104DC0000FB0BDE8F08320460F4913F09AF904466E
:104DD000A0B9736B002BEED00125DFF83490736B14
:104DE00001A81B5DC5F1320128444A46013413F085
:104DF000EFF8102C05F10205F1D1DCE7034ADBE7FF
:104E000032C2010837C201083BC2010843C201088F
:104E100007D50108016000210273C0E90111704744
:104E2000F8B5054617460E4639B332B32049182067
:104E300007F0F6FE044608B3C0E9006700261D4BE4
:104E400000F108074361C0E9026606618021384627
:104E500007F0FAFDD4E90012384607F033FE144992
:104E6000082007F0DDFE90B16B68C0E9004603B989
:104E70006860AB6803B15860A860F8BD0E4808F0E0
:104E8000C9FD01213046BDE8F84007F0D5BE0B480A
:104E900008F0C0FD0A4A40F255110A4808F0BAFD70
:104EA0000121206807F0C8FE18212046EBE700BF6B
:104EB000EEE901088081828366D501089EC201085F
:104EC000BAC20108F1C2010870B54468054604B3CE
:104ED000266806F1080007F0BFFDD6E903239A42D1
:104EE000C4B216D16B681BB96A210B48FFF790F961
:104EF0006868082143686B6007F09EFE6B6803B921
:104F0000AB600121306807F097FE1821304607F0AA
:104F100093FE204670BD00BF0EB9010810B50446CF
:104F2000006810B1012107F087FE204610BD7FB553
:104F30000546FFF71AFA13F0F6F80446861C2846D1
:104F4000FFF715FA013803281DD8DFE800F0020644
:104F5000080F0734601C04B070BD0D34FAE7284612
:104F6000FFF74CFA13F0DFF83418F3E701A82946ED
:104F7000FFF70DFADDE9014301A81B1B06EB430413
:104F8000FFF7CCFFE6E70B34E4E700002DE9F0473C
:104F900086B08146884614461D46FFF745FE68B137
:104FA0002046FFF7C4FF4049074607F043FE064688
:104FB000C9F8000028B93D4808F02CFD06B0BDE84E
:104FC000F0872046FFF7D3F90138032864D8DFE8DB
:104FD00000F00214253D2046FFF7C7F98146204620
:104FE000FFF7C7F9324B334A002814BF1846104662
:104FF000CDE900902B46304A0AE02046FFF7B5F98C
:1050000081462046FFF7EDF92B46CDE900902B4A6B
:105010003946304612F0DCFF05463AE0612D204665
:105020000DD1FFF7A2F905462046FFF7E7F92B4619
:10503000234A00903946304612F0CAFFECE7FFF7EA
:1050400094F981462046FFF7D9F9D1E72046FFF7CA
:105050008CF92B4600901B4A3946304612F0B8FFB7
:10506000DFF868902146054603A8FFF790F9DDE9CF
:10507000034AA2450AD0AF4214F8013B06D9791B76
:1050800070194A4612F0A4FF0235F2E703A8FFF7B1
:1050900045FFC8F8005091E72046FFF766F92B4618
:1050A0000090094AC6E700BFEEE9010866D501088D
:1050B000D8C00108DDC0010852C201085AC2010867
:1050C00063C201086AC2010870C2010807D501085D
:1050D0002DE9F0430E4607469046D1B04FF49C723E
:1050E000002102A81D46589C12F06DF831463B463F
:1050F000424602A8FFF7D8FD3678622E00F0F9800C
:1051000029D83F2E54D008D82E2E5BD09DF80810F9
:105110007D4808F07FFC7D4A58E0532E00F0A180C6
:10512000612EF3D10DF1340979484A4605A908F0FA
:1051300071FC4F98002800F0D580FFF718F903287C
:1051400000F0AF802846734A2146FFF74FFD7248B2
:1051500008F060FC33E0722E48D00ED8642E3AD0AE
:10516000672ED3D105A96D4808F054FC33464F9AF9
:1051700021462846FFF70AFF21E0732E51D0772EF3
:10518000C4D1674808F046FC0399002900F0BA80B2
:10519000644812F0B6FF0646002840F0B38062482B
:1051A00008F038FC3146384600F050FF5F4AA4E072
:1051B0005F4808F02FFC21462846FFF7CBFD51B091
:1051C000BDE8F0835B4808F025FC5B4A2146284691
:1051D000FFF70CFDF3E70399584808F01BFC02ABFE
:1051E0003A4621462846FFF7CFFDE8E705A954488F
:1051F00008F010FC0399534812F083FF20B9384699
:1052000000F03AF9504AE1E74F993846FFF7FEFCC3
:1052100008B14E4ADAE74F9808B1FFF72FFB722327
:10522000A5E705A94A480DAA08F0F4FB4F993846AE
:10523000FFF7ECFC0028ECD14F9810B10DA9FFF757
:105240008DFC73234F9A21462846FFF79FFE216865
:10525000404808F0DFFB2868216808F041FC3E4820
:1052600076E705A93D480DAA08F0D4FB4F993846CA
:10527000FFF7CCFC0028CCD14F9810B10DA9FFF757
:105280006DFC2146284673234F9AFFF77FFE0121CC
:10529000384600F0DBFE324808F0BCFB01F03EF976
:1052A0008DE74F98FFF7AAF812F03DFF08F10106CD
:1052B00006442C49304607F0BDFC074690B14F9894
:1052C000FFF79CF8284A03463146CDF8009038464F
:1052D00012F07EFE39464F98FFF740FC0121384618
:1052E00007F0AAFC61234F9A21462846FFF7B0FC3D
:1052F000ADE71E4808F08EFB1D4A21462846FFF701
:1053000075FCC8E701214EE762C4010884C40108A6
:10531000B4C30108CDC30108D9C3010825C30108DE
:1053200015C401083DC4010843C4010860C4010854
:10533000FFC2010809C3010813C3010816C301080D
:1053400036C3010852B7010849C301084CC301081C
:1053500066C301087FC3010882C4010890C3010825
:1053600095C40108EEE90108EBC30108F0C3010888
:1053700013C401082DE9F0410C4680460D4815463E
:105380001E46069F08F046FB04B14DB90A4808F0D6
:1053900041FB39463046BDE8F041084AFFF726BCDC
:1053A000069733462A4621464046BDE8F041FFF7BE
:1053B0008FBE00BFC1C40108D6C40108E9C40108FA
:1053C0007FB504460D4600680C49164600F000FB08
:1053D00078B100F0E9FC03AB00933246294602ABFA
:1053E000FFF7C8FFDDE902122046FFF719FD04B000
:1053F00070BD034808F00EFBF9E700BF5BC301086E
:105400007FC2010810B10C2107F016BC704710B123
:10541000012107F011BC704730B513460D46044614
:10542000AC4207D01BB194E8070083E807000C33B7
:105430000C34F5E7184630BD10B5044638B1FAF71C
:1054400085FE2046BDE81040282107F0F5BB10BDC1
:1054500070B50446406AFFF7D5FFD4E90656AE4260
:1054600004D02846FAF772FE2835F8E7A06908B19B
:10547000FFF7E2FF204670BDF8B505460024282658
:10548000074FD5E906031B1ADB107B439C4205D26C
:1054900006FB0400FFF7F2F90134F2E7F8BD00BFA4
:1054A000CDCCCCCCF8B50446224808F0B3FA22485B
:1054B00008F0B0FAD4E90631994218D0C91A1F4E43
:1054C000C91071431E4808F0A5FA00252827D4E921
:1054D00006031B1ADB1073439D4205D207FB050030
:1054E000FEF798FF0135F2E7164808F093FAD4E981
:1054F0000931154EC91A89107143144808F08AFA07
:1055000000250C27D4E909031B1A9B1073439D4205
:1055100005D207FB050001F013F80135F2E70C484E
:1055200008F078FA0B4808F075FABDE8F8400A4828
:1055300008F070BAA9C501086EDC0108CDCCCCCC4E
:10554000B3C50108C5C50108ABAAAAAAFEC50108D2
:1055500082C401080EC6010827C601082DE9F043E0
:10556000002487B006466846CDE90044029407F05F
:1055700095F8684607F02AF94FF028082F4F304D6C
:10558000D6E906239B1ADB107B439C424ED208FBD4
:1055900004F302EB0309D35C002B43D14846FEF72A
:1055A000E4FE0146684607F003F94846FEF7DFFED1
:1055B000042837D8DFE800F03803101A24004846E2
:1055C000FEF7D7FE0146684607F0A8F850BBC22197
:1055D0002846FEF71DFE25E04846FEF702FF01467D
:1055E000684607F081F8E8B9C621F1E74846FEF7BA
:1055F00005FF0146684607F0DBF898B9CA21E7E7DE
:10560000494603A8FEF7C3FEDDE903126846521AB5
:1056100007F0A6F818B9CF212846FEF7F9FD039840
:10562000FFF7F5FE0134ABE7D321D1E7684607F079
:10563000F5F8029807B0BDE8F08300BFCDCCCCCC24
:105640000EB901082DE9F04305460E4600244FF03F
:1056500028081A4F8DB0D5E906239B1ADB107B432F
:105660009C4224D208FB042931461822684612F0D5
:1056700074FD4846FEF779FE182201460DEB020044
:1056800012F06BFD684608F04AFB684608F059FBCB
:1056900006A808F044FB06A808F053FB1822684649
:1056A0000DEB020112F047FD18B10134D3E74FF0C2
:1056B000000948460DB0BDE8F08300BFCDCCCCCC8E
:1056C0002DE9F04F06460F4600244FF00C09DFF895
:1056D0006C808DB0D6E909535B1B9B1008FB03F36C
:1056E0009C4224D218223946684612F036FD182210
:1056F00009FB04FB0DEB020055F80B1012F02DFD19
:10570000684608F00CFB684608F01BFB06A808F08A
:1057100006FB06A808F015FB182268460DEB0201EF
:1057200005EB0B0A12F007FD18B10134D2E74FF078
:10573000000A50460DB0BDE8F08F00BFABAAAAAA80
:1057400010B51446FFF77EFF20B12146BDE810409A
:10575000FFF704BA10BD0000F8B50C46064640F24B
:1057600001120021224811F02EFD4FF480722146D3
:105770001F4811F004FD1E491E4808F04BF91E4950
:105780001B4813F053FB1C490546002013F04EFB49
:10579000294607463046FFF755FFA0B9294630464F
:1057A000FFF78EFF044600B30168144808F032F991
:1057B000A3683846984701242046F8BD394610486A
:1057C00008F028F9F8E73A4629463046FFF7B8FFCF
:1057D00004460028F2D00B4808F01CF90A4808F0EB
:1057E00019F93046FFF75EFEE6E729460748E7E786
:1057F0002C0A00204DC60108ECE9010853C6010837
:105800007CC6010868C6010882C4010895C6010863
:1058100010B54FF4807204460649043007F0B6F81C
:10582000002805DD2046BDE810400249FFF794BF7F
:1058300010BD00BF2C09002038B514461D46FFF7E7
:1058400001FF28B12A462146BDE83840FFF72EB9AE
:1058500038BD10B51446FFF7F5FE20B12146BDE86E
:105860001040FFF783B810BD10B51446FFF7EAFEED
:1058700010B12146FEF78EFF002010BD38B514464A
:105880001D46FFF7DFFE28B12A462146BDE8384015
:10589000FFF77CB938BD00002DE9F04700248CB03B
:1058A000074603A8CDE90344059406F0F7FE214618
:1058B00003A8009407F00EF80146002834D02146D2
:1058C00003A806F090FF40F2E73304460093002659
:1058D0003546DFF8F890009BB34273D9214603A800
:1058E00006F0B3FF824600286CD1182321460DEB49
:1058F000030203A806F03AFF0444214603A806F079
:10590000B2FF8046B0B10CAA214642F828AD03A8E8
:1059100006F0CAFE029A044406A93846FFF799FF2A
:1059200000B101350136D6E76A4603A806F062FFEA
:105930000446CCE7214603A806F0DFFF70B10CAAAD
:1059400002F8288D214603A806F0D8FE9DF808200D
:10595000044406A93846FFF787FFE1E7214603A87C
:1059600006F09CFF804668B102AB01AA214603A85D
:1059700006F00DFFDDE90123044406A93846FFF7D0
:105980005BFFCDE7214603A806F07AFF90B10CAB90
:1059900043F8288D01AA214603A8CDF8048006F01B
:1059A000CEFE9DF808300444019A06A93846FFF758
:1059B00065FFB5E7039B4846195D01F0E00108F07B
:1059C00029F8AFE728460CB0BDE8F08738C50108D4
:1059D00008B5FFF737FE18B1BDE80840FEF7C9BCAF
:1059E00008BD10B5044608461146FFF72BFE0146D8
:1059F00020B9C4E90000A060204610BD2046FEF793
:105A0000C6FCF9E708B5FFF71DFE18B1BDE8084070
:105A1000FEF7E7BC08BD08B5FFF714FE18B1BDE8F6
:105A20000840FEF7EBBC08BD2DE9F0410E469DF89D
:105A30001840174698469DF81C50FFF7E3FF844234
:105A400005DCA84203DC88F80000BDE8F0810123F2
:105A500022463B70314606902B46BDE8F041014896
:105A600007F0D8BF10C501082DE9F0410E46BDF87A
:105A7000184017469846BDF81C50FFF7C3FF8442F4
:105A800005DCA84203DCA8F80000BDE8F081012392
:105A900022463B70314606902B46BDE8F041014856
:105AA00007F0B8BF10C501082DE9F0479946DDE9B8
:105AB000086788469246FFF7A5FF0023C517B04246
:105AC00075EB0303044607DB00238742AB4103DB8E
:105AD000C9F80000BDE8F0870123CDE908458AF840
:105AE000003032463B464146BDE8F047014807F0EA
:105AF00091BF00BF10C5010873B51C460E46154680
:105B0000FFF789FF002302AA42F8043D20600699AE
:105B100007F05AFD019B33B122683146034807F074
:105B200079FF01232B7002B070BD00BFB8C6010819
:105B3000002370B5D1E90025AD1A0446C0E9003351
:105B400083600E46284601D008F000F8C4E9000042
:105B50000544A560D6E90053024629468B4205D08C
:105B60000AB10E78167001310132F7E75B1B184459
:105B70006060204670BD38B504460D460B78103085
:105B800000F8103C4B68103140F80C3C51F8083CD0
:105B900040F8083C51F8043C40F8043CFFF7C8FFCB
:105BA00005F11C0104F11C00FFF7C2FF204638BDBF
:105BB0002DE9F843D0E90054641B9146A2101F4C14
:105BC00006465443B4F5884F0F4602D11C4806F0F0
:105BD000F7FF002C14BF22460122A418A1EB0505F3
:105BE00026D2B4F5884F23D82CB30C20604307F09D
:105BF000ADFF804618EB05031CBF99E8070083E85A
:105C00000700424639463068FFF706FC716800F12C
:105C10000C023846FFF700FC05463068FFF7F2FB40
:105C20000C2303FB0484C6E90085B460BDE8F88357
:105C30004FF48844D9E7A046DCE700BFABAAAAAA84
:105C400096C001082DE9F043054685B008460C468C
:105C500017461E4612F067FA172803D982212D48ED
:105C6000FEF7D6FACDE90147D5E9097803962A4A25
:105C7000A8EB0706B41054430134B4F5884F02D999
:105C8000264806F09DFFEB6ADB1B9B1053439C42AA
:105C900015D94FF00C0909FB04F91CB1484607F06F
:105CA00055FF0446224641463846FFF7B5FB686A71
:105CB000FFF7A8FB26446C624C44AE62EC62EA6AD1
:105CC000D5E9090314491B1A9B10121A4B43921071
:105CD0004A430133934206D9114807F09BFE8C21B9
:105CE0000C48FEF795FAD5E90A3293420AD023B15F
:105CF00004AA12E9070083E807000C33AB6205B081
:105D0000BDE8F08301AA194605F12400FFF750FF12
:105D1000F5E700BF0EB90108ABAAAAAA5BC001084B
:105D2000F5C4010838B500250346044603F8045BB2
:105D300029461846142211F046FA0A4AC4E90655C3
:105D40006261C4E90855C4E90A55C4E90C558021CB
:105D500006F0E1FD2046044B044A0549FFF772FFB7
:105D6000204638BDAC080020AD5D0008DBC6010848
:105D7000E7C6010810B5084C2368DB0709D40748BB
:105D8000FFF7D0FF0123064A0649044823600EF0BE
:105D900051FB024810BD00BFA8080020300B0020B6
:105DA0000000002051540008FFF7E4BF08B5FFF7DA
:105DB000E1FFBDE80840FFF775BB0022C0E9002203
:105DC000826010B50C6804600A6042684C684460E8
:105DD0004A6082688C6884608A6010BD70B50E4627
:105DE00005461446B54217D09CB12B7805F1100139
:105DF00023706B6804F110006360AB68A360EB680C
:105E0000E360FFF7DAFF05F11C0104F11C00FFF766
:105E1000D4FF28342835E5E7204670BD2DE9F84346
:105E2000D0E90064A41BE310234C05465C43B4F5A1
:105E3000884F0F46914602D1204806F0C1FE002C43
:105E400014BF23460123E418A1EB060623D2B4F5C0
:105E5000884F20D814B32820604307F077FE80468F
:105E600018EB060002D04946FFF785FE3946424648
:105E70002868FFF7B3FF696800F128023846FFF78A
:105E8000ADFFD5E900690746B14509D03046FAF7BC
:105E90005DF92836F8E74FF48844DCE7A046DFE7F1
:105EA000286808B1FFF7C8FA282303FB0484C5E972
:105EB0000087AC60BDE8F883CDCCCCCC96C001089F
:105EC0002DE9F047D0E9065704460E46DFF80C816D
:105ED0008AB0AF421BD029466846FFF74CFE6846A1
:105EE000FEF743FA81463046FEF73FFA0146484640
:105EF00007F056FF30B13046FEF737FA014640460C
:105F000007F088FD6846FAF721F92835E1E7D4E97A
:105F100006892E4AA9EB0807FD1055430135B5F552
:105F2000884F02D92A4806F04BFE236AA3EB0803E8
:105F3000DB1053439D4220D94FF0280A0AFB05FA93
:105F40001DB1504607F002FE0546494640462A4626
:105F5000FFF744FFD4E90689C14505D04046FAF76A
:105F6000F5F808F12808F7E7A06908B1FFF764FA27
:105F70002F44A5615544E7612562226AD4E90603EE
:105F800012491B1ADB10121A4B43D2104A43013339
:105F9000934206D90F4807F03DFD77210E48FEF7E2
:105FA00037F9D4E90703984209D010B13146FFF719
:105FB000E2FDE3692833E3610AB0BDE8F0870146FA
:105FC000324604F11800FFF729FFF5E7CDCCCCCC21
:105FD0005BC001088AC501080EB9010858C501084F
:105FE000002313B502A941F8043D094B0422D3E96B
:105FF0000140084B20445B689847044628B1064896
:1060000007F008FD204602B010BD0448F8E700BFC5
:10601000800B00206C0B0020F2C8010806C90108A3
:1060200008B5084807F0F6FCFFF7A4FEFFF724FACE
:10603000054807F0EFFCFFF79DFEBDE80840FFF7BD
:1060400031BA00BF23C901083BC9010873B5054631
:106050004FF416700C4607F079FD064630B921481A
:1060600007F0D8FC22212048FEF7D2F84FF4167230
:106070000021304611F0A7F8314628464FF4167239
:10608000FFF76CFA194D014601902CB3184807F040
:10609000C1FCD5E901431C44164DEB681BB10199C5
:1060A0002046083198476B680422104920469847DB
:1060B00004226B680DEB0201A01898476B68019AE7
:1060C000314604F1080098470B4807F0A3FC30461E
:1060D00007F026FD02B070BD084807F09BFC6C6815
:1060E000DAE700BF2BD701080EB90108800B0020AA
:1060F000E4C701086C0B00201EC8010803C8010892
:106100002DE9F74FFFF736FE2F4F06462F4807F0D1
:1061100081FCB846DFF8D090DFF8D0A0FCF7D4F8C7
:106120002B4D38602B68AB462A4C002B37D003F53B
:106130006A436033984232D223782BB9264807F05D
:1061400069FC264807F066FC012330462370FFF700
:106150005FFB41F2883352464FF0FF310020FCF7DD
:1061600087FD0190FCF7B0F8019BC8F8000023B947
:10617000237813B13046FFF74BFBDAF80030DA072B
:1061800044BFD8F800202A609B07C7D50023CBF86E
:106190000030D9F80830002BBED09847BCE72378F0
:1061A0006BB100213046FFF751FF0D4807F032FC7C
:1061B0000C4807F02FFCD9F8083003B198470023AA
:1061C00023702B60C5E700BF980B002062C8010850
:1061D000940B00208C0B002077C801089AC8010896
:1061E000BDC80108CFC801086C0B0020900B00202F
:1061F00010B5FFF7BFFD04460021FFF727FF20463B
:10620000FFF750F9BDE810400348002301220221A6
:106210000068FCF777BD00BF680B002010B5FFF7E2
:10622000A9FD04460021FFF711FF2046BDE81040FC
:10623000FFF738B92DE9F743194E074688467568C8
:106240000AB1B3681D440024DFF8609002A941F848
:10625000084D0422D9F80030284698473268009942
:106260008A4204D00F4807F0D5FB204614E00422F0
:10627000D9F800300DEB0201A818984701990A4897
:1062800007F0C8FB019A4245EFD8D9F800303946EB
:1062900005F108009847019803B0BDE8F08300BFFE
:1062A000800B00202DC8010848C801086C0B002095
:1062B00084B0F0B585B00AAC84E80F000B9B23B91D
:1062C00040F229117F48FDF7A3FF0A9B23B94FF441
:1062D00095717C48FDF79CFF7B4C0AAD0FCD0FC438
:1062E0002B682546794C0FAA07CA45F8103984E86F
:1062F000070012B94FF48063A360236823B940F20A
:1063000035117048FDF784FF2368013304D140F252
:1063100037116C48FDF77CFFFFF72CFD06466C4BF0
:106320006C4A6D49FFF78EFC6C4B6D4A6D493046E7
:10633000FFF788FC6C4B6D4A6D493046FFF782FCD5
:106340004FF4167007F002FC074680B9694807F061
:1063500061FB694807F05EFB3046FFF78DF80023CC
:106360003370FFF73DFE654807F054FB2CE04FF417
:106370001672002110F027FFD4E901032D680422D2
:1063800003A91844A847002861D02268039B9A42B9
:106390005DD15B4807F03EFB01224FF41671384691
:1063A000FFF748FF0446574807F034FBFFF718FE95
:1063B000002C48D001233370224639463046FFF77F
:1063C0006BFA384607F0ACFB33783BBB4FF41670E2
:1063D00007F0BCFB044630B9464807F01BFB7F21A1
:1063E0003848FDF715FF4FF416720021204610F0D3
:1063F000EAFE00224FF416712046FFF71BFF074606
:1064000090BB07F08DFB204607F08AFB3E4807F063
:1064100001FBFFF7AFFC0021FFF718FE3B4BFA2210
:10642000019301233A4900933A480023FBF70AFD00
:1064300020B94FF4A8712348FDF7EAFE05B0BDE886
:10644000F04004B07047344807F0E4FA347000229A
:106450004FF416713846FFF7EDFE04460028ABD125
:10646000384607F05DFB74E74FF4167007F06EFBDB
:10647000054630B91F4807F0CDFA8E211148FDF7C7
:10648000C7FE4FF416720021284610F09CFE4FF410
:10649000167229463046FFF761F808B92846B0E77A
:1064A0008742FBD10023E95CE25C9142F6D10133E3
:1064B0009F42F8D1284607F033FB204607F030FB17
:1064C000ACE700BF0EB901086C0B0020800B002068
:1064D0001D620008EBC60108F7C60108216000082C
:1064E000FCC6010817C70108F16100081FC70108B1
:1064F00037C701082BD701089EC701083BC901080F
:106500003CC7010860C70108C2C70108680B00202A
:10651000D9C701080161000875C7010810B5064C0C
:10652000226922B94FF4AA710448FDF771FE23696C
:10653000BDE81040184700BF6C0B00200EB90108E1
:1065400010B504460168074807F064FA616831B184
:106550000B7823B10448BDE8104007F05BBA03484C
:10656000F9E700BF53C9010819C1010882C4010835
:1065700010B50446C06908B107F0D2FA206908B125
:1065800007F0CEFA606808B107F0CAFA204610BDDD
:1065900010B504460068FDF735FD204610BD00002B
:1065A0001FB50B46546801780294127801925A681C
:1065B000009242681B68024807F02CFA04B010BD34
:1065C00058C90108CB210148FDF722BE0EB90108C8
:1065D000FE2307B502A901F8043D054B1868002306
:1065E00000681A46FDF7FEF903B05DF804FB00BF32
:1065F000A80B0020D0B51F467423C0E9003100234A
:10660000044683600820164606F0F8FAC0E90067E1
:10661000A0602046D0BD70B51D466923C0E9003199
:106620000023044683600820164606F0E7FAC0E916
:106630000065A060204670BD036837B5632B044633
:106640000D4601D0FFF7BEFF002302AA42F8043D29
:10665000A168284606F0B8FF019B1BB1382102480B
:10666000FDF7D6FD03B030BD0EB9010870B5632348
:106670000025C0E90031044685601A20164606F060
:10668000BDFA1A22294610F09EFD3146A060204630
:10669000FFF7D2FF204670BD81647047C164704728
:1066A0002DE9F843D0E90173884600254FF00C0925
:1066B000DB1B0A4E9B105E43ECB2B4420BD209FBCB
:1066C00004724146506811F01CFD01350028F3D1D9
:1066D0002046BDE8F8834FF0FF30FAE7ABAAAAAA3C
:1066E0002DE9F843D0E90473884600254FF00C09E2
:1066F000DB1B0A4E9B105E43ECB2B4420BD209FB8B
:1067000004724146506811F0FCFC01350028F3D1B9
:106710002046BDE8F8834FF0FF30FAE7ABAAAAAAFB
:106720002DE9F0410E4649680446FFF7B9FFC0B2B3
:10673000FF2803D07C212948FDF76AFDD4E9012315
:10674000274F9B1A9B107B437E2B03D97F21234825
:10675000FDF75EFDD4E901120C25E068531A9B1089
:10676000121A7B4392107A430133934205FB03F8DC
:106770000ED84144A160D4E9013496E80700E31A39
:1067800004E9070016489B1058430138BDE8F08122
:10679000404607F0DBF9054618B969210F48FDF7B7
:1067A00037FDD4E901C30027A3EB0C039A100C4B6F
:1067B0005343002B09DD05EB070E0CEB070207CA5C
:1067C000013B8EE807000C37F3E7604607F0A8F9B5
:1067D00065604544C4E90255CDE700BF0EB9010824
:1067E000ABAAAAAAFF2270B5002380F828204FF098
:1067F00000424FF0FF31C0E90D23C2636FF07F42CA
:10680000C0E910120522C0E90033C0E91423C0E931
:1068100002330022C0E90433C0E90633C0E908337B
:106820000363C0E9123383654FF000431E4DC0E996
:1068300018232A68044612F0010213D101211B4ECD
:10684000084632607160FCF7F3FF306018B95121DF
:106850001748FDF7DDFC0123164A174913482B6042
:106860000DF0E8FD154B1A680AB9104A1A60144970
:106870002046FAF7CFFA134B134918702046FAF75F
:10688000C9FA124B124918702046FAF7C3FA114B95
:10689000114918702046FAF7BDFAFE220F4B187006
:1068A0000F4B20461A7070BDA40B0020280C00204E
:1068B0000EB901080000002091650008A80B002017
:1068C000C4CA0108B00B0020CCCA0108AE0B0020DE
:1068D000D4CA0108AC0B0020D9CA0108AF0B0020B4
:1068E000AD0B002010B5084C2368DB0709D407481E
:1068F000FFF778FF0123064A0649044823600DF09C
:1069000099FD024810BD00BFA00B0020C00B002065
:1069100000000020716500082DE9F0410E4649682D
:106920000446FFF7DDFEC0B2FF2803D087212948C7
:10693000FDF76EFCD4E90423274F9B1A9B107B4381
:106940007E2B03D98A212348FDF762FCD4E9041287
:106950000C25A069531A9B10121A7B4392107A439C
:106960000133934205FB03F80ED841446161D4E939
:10697000043496E80700E31A04E9070016489B1060
:1069800058430138BDE8F081404607F0DFF805467E
:1069900018B969210F48FDF73BFCD4E904C300276F
:1069A000A3EB0C039A100C4B5343002B09DD05EBB2
:1069B000070E0CEB070207CA013B8EE807000C37F5
:1069C000F3E7604607F0ACF825614544C4E9055596
:1069D000CDE700BF0EB90108ABAAAAAA38B5D0E925
:1069E00001239B1A074A9B105343CDB29D42044694
:1069F00003D3A6210448FDF70BFC0C20636800FBC1
:106A0000053038BDABAAAAAA0EB9010838B5CCB278
:106A1000114905460B6813F0010307D10F4A702096
:106A20001372012310600E480B605060FF2C10D0D1
:106A3000D5E904239B1A0B4A9B1053439C4203D372
:106A4000B2210948FDF7E4FB0C23286903FB04008D
:106A500038BD0248FCE700BF9C0B0020B40B0020AF
:106A600076C90108ABAAAAAA0EB9010810B5D0E9E7
:106A70000730C9B2D2B2834209D01C788C4204D10B
:106A80005C78944201D1987810BD0333F3E74FF05E
:106A9000FF30F9E72DE9F041D0E904239B1A4F4A72
:106AA0009B1053430D4609780446994203D3932122
:106AB0004B48FDF7ADFBD4E901239B1A474A9B10D5
:106AC00053436978994203D394214548FDF7A0FBCD
:106AD000D4E904239B1A414A9B105343A978994255
:106AE00005D3FE2903D095213D48FDF791FB6A7837
:106AF00029782046FFF7BAFFC3B2FF2B064629D0FC
:106B000029782046FFF782FF697807462046FFF77D
:106B100065FF314680462046FFF778FF4146024632
:106B20003846FFF73DFD29782046FFF76FFF69786B
:106B300006462046FFF752FFA97807462046FFF792
:106B400065FF394602463046FFF72AFD9C2124485E
:106B5000FDF75EFBD4E90723204F9B1A7B437E2B76
:106B600003D99F211E48FDF753FBD4E90762616AF0
:106B7000931B7B43521A57430133BB4203EB430839
:106B80000AD8464426622A88236A23F8032CAA7866
:106B900003F8012CBDE8F081404606F0D7FF064619
:106BA00018B969210E48FDF733FBD4E90702131A1F
:106BB0000A4A5A430023002A0ADDC118B1F800C06E
:106BC000F71826F803C08978013AB9700333F2E761
:106BD00006F0A6FFE66146446662D3E7ABAAAAAA1E
:106BE0000EB90108FF2337B58DF804300A4B0D4666
:106BF0001C6823681BB929210848FDF709FB2A46B0
:106C000001A92068FCF792FF012814BF4FF0FF3064
:106C10009DF8040003B030BDA80B00200EB9010898
:106C200038B5816800681D46144607F041F80346F0
:106C3000201845EBE37138BD08682DE9F041722852
:106C40001F461FD074280FD0632820D1886806F013
:106C50007BFD002871F1000304460D460EDADD21AC
:106C60000D48FDF7D5FA09E08B68D3E90045B5F189
:106C7000004F08BF002C01D0A4187D4120462946B2
:106C8000BDE8F0818868BDE8F041FFF7C9BF002486
:106C90004FF00045F2E700BF0EB901082DE9F041C1
:106CA0000F4606460024FFB2FFF7B0FED6E90758AC
:106CB000454511D02B78BB420CD169783046FFF79F
:106CC0008DFE0368692B05D183681B6803B1984763
:106CD0000134E4B20335EBE72046BDE8F0812DE94D
:106CE000F34180460F460025FFF790FED8F81C4080
:106CF000D8F8206003340336FFB2A6421BD02346E7
:106D000033F8032D9B78ADF804208DF8063014F885
:106D1000033C9F420DD19DF805104046FFF75EFEF3
:106D20000368692B05D183685B6803B19847013517
:106D3000EDB20334E1E7284602B0BDE8F08100007F
:106D4000836C73B504460D46164623B94FF48E7115
:106D50000B48FDF75DFACDE9006423462A46094950
:106D60000948FBF76FF8012807D04FF491710448E8
:106D700002B0BDE87040FDF74BBA02B070BD00BF75
:106D80000EB90108A6CA01085173000838B590F879
:106D900047300446032B0D4604D940F2351106480E
:106DA000FDF736FA94F847305A1C84F847201C4403
:106DB00084F8425038BD00BF0EB9010810B590F8F4
:106DC0004730044623B94FF49D710648FDF720FA79
:106DD00094F84730013BDBB284F847301C4494F808
:106DE000420010BD0EB9010838B50546002495F8DB
:106DF0004730A34207DD2B1993F842102846FFF7CE
:106E000005FE0134F3E738BD00232DE9F74FC0E953
:106E1000083388461946D8E907594FF0004304461D
:106E2000C0E90613C0E90013C0E90213C0E9041366
:106E3000FF208A469B46D2B284F8200001924D453D
:106E4000D4E9006720D02B78019A93421AD169784F
:106E50004046FFF7C3FDDDE90C2301464046FFF73E
:106E6000EBFE594508BF50450CD05F4508BF56455D
:106E700003D0B04271EB070304DA6B78C4E9000178
:106E800084F820300335DAE7B7F1004F08BF002E51
:106E900008D0DDE90C23B21A67EB030316461F4640
:106EA000C4E90467204603B0BDE8F08FF8B50D468D
:106EB0000B4B896906464B434FF47A71B3FBF1F1F2
:106EC000FFF790FE0446C7B2B06C03681B68984792
:106ED000FF2FC6E90E010CBF95F820002046F8BD33
:106EE00040420F0038B5C36C04460D461BB9BDE8DF
:106EF0003840FFF7DBBF806C174903685B69984730
:106F0000A06C0368DB689847D5E9020106F002FD32
:106F10000146124806F07EFDA06C03689968D5E929
:106F200002238847A06C03681B699847E36C984765
:106F3000A06C0368DB689847A06C03681B689847DF
:106F4000C4E90E0100212046FFF74CFEC0B2FE2826
:106F500008BF95F8200038BDD1650008B1CA010806
:106F6000F8B5D1E90667B7F1004F08BF002E054616
:106F70000C4608D11AB1BDE8F840FFF797BFBDE84D
:106F8000F840FFF7AFBF012E77F1000302DA91F866
:106F90002000F8BD92B121462846FFF787FF94F8FC
:106FA0002030C0B28342F4D1D5E90E67D4E9002382
:106FB000964277EB0303B8BFFF20EAE7D0E914233A
:106FC000964277EB0303E6DBFFF78CFFE7E7000071
:106FD0002DE9F04F8DB004460D46FFF717FD03680D
:106FE0008046702B04D04FF4A0716B48FDF710F968
:106FF000A06C03681B6898472A46C4E90C01CDE9D8
:107000000001214602A8FFF7FFFE29462046FFF7B0
:1070100045FE9DF828300646FF2B05D120B940F2E9
:107020004B115D48FDF7F4F8D4E90C0106F072FC51
:1070300001465A4806F0EEFC3146594806F0EAFC93
:107040009DF82810FF297ED100224FF00043CDE9A2
:107050000623DDE90223CDE90423DDE90623CDE99A
:107060000823A36D13B39847DDE90223D4E918017F
:10707000B3F1004F08BF002A09D0DDE9062310F163
:107080000B0641F10007964277EB03030EDAD4E9D1
:107090000C23161843EB0107CDE90801CDE904677D
:1070A00006F04EFC01463F4806F0B4FC4FF0000AE3
:1070B0004FF0004BDFF8F89098F8082002A920461E
:1070C000FFF74EFFA36D064603B19847F3B2FF2BBF
:1070D0005AD1DDE90223D4E90E01161A63EB010748
:1070E00039463046CDE90423CDE90667CDE9086786
:1070F00006F026FC0146484606F08CFCA36D002BEA
:10710000DAD0DDE90223D4E918015B4508BF524516
:1071100009D0DDE9062310F10B0641F10007964284
:1071200077EB0303C8DAD4E90E23161843EB010703
:10713000CDE90801CDE9046706F002FC01461948D3
:1071400006F068FCB8E72046FFF748FCD0E9006786
:10715000DDE9020106F0DEFB3A46034631461248FD
:1071600006F058FCD4E90C23DDE90201801A61EB3A
:1071700003010F460646CDE9066706F0E1FB01462E
:107180000A4806F047FC64E729462046FFF7A7FDBA
:1071900030460DB0BDE8F08F0EB9010884C9010872
:1071A000A3C9010800CA0108BEC90108E2C9010853
:1071B00018CA010870B504460D46FFF727FC03689E
:1071C0006D2B11D0702B09D0612B14D1836894F8EA
:1071D000411094F84000BDE8704018472946204609
:1071E000BDE87040FFF7F4BE034840F22F11FDF7F1
:1071F0000FF84FF0FF3070BD0EB901082DE9F047D0
:1072000090F828300446FF2B04D14FF4E5714A482A
:10721000FCF7FEFF94F828102046FFF7F7FB4268C2
:107220000178464806F0F6FB94F82830DFF81C8118
:1072300084F8463094F846102046FFF7E7FB0368D1
:1072400005466D2B204694F846100BD1FFF79EFDA6
:10725000297A204684F84610FFF7D8FB2046FFF72E
:10726000C3FDE7E7FFF7A6FFC3B2FF2B06460BD12E
:1072700040F2DF113048FCF7CBFF40F2DF11304B1A
:10728000304A31480FF05AFD024694F84610204625
:10729000FFF7ECFBC5B2FF2D09D140F2E5112648FE
:1072A000FCF7B6FF264B274A40F2E511E9E794F8D0
:1072B0004610FE2D204621D1FFF780FD07460146EE
:1072C0002046FFF7A3FB324639462046FFF7CEFBA8
:1072D000C5B2FF2D0DD131462046FFF77FFB40F2AE
:1072E000F1111548FCF794FF154B164A40F2F111C5
:1072F000C7E72046FFF778FD3946DAE7FFF786FB58
:10730000314607462046FFF769FB2946814620465D
:10731000FFF77CFB8246404606F07CFB524649461E
:107320003846FFF73DF994F8463084F8416084F818
:10733000403084F846507DE70EB9010840CA010884
:10734000DDC00108E1CA01085ECA010896CA010849
:1073500008B506F0C5FCFFF7C5FAFFF74FFFD0B53B
:107360001F461646FFF73AFB03688468742B01D06A
:10737000FFF728F9C4E90067D0BD0000FF23054AE4
:107380001370054A1370054A1370054A1370054AB5
:1073900013707047B00B0020AE0B0020AC0B002028
:1073A000AF0B0020AD0B002070B50446044E45180D
:1073B00014F8011B304606F02DFBAC42F8D170BD2D
:1073C00007D5010830B504468DB001467A4A6846B3
:1073D000FEF707FB794A214603A8FEF702FB784A2D
:1073E000214606A8FEF7FDFA76492046FEF7F0FA98
:1073F0000546754806F00EFB0123039A02F11001C1
:10740000914205D011F8010D002818BF0023F7E7BD
:10741000002B53D06D4806F0FDFA5DB36C4806F0C2
:10742000F9FA6C4A214609A8FEF7DBFA6A4806F029
:10743000F1FA08210098FFF7B7FF684806F0EAFA6A
:1074400008210998FFF7B0FF654806F0E3FA10211C
:107450000698FFF7A9FF634806F0DCFA0998069A38
:10746000009900F0CDFE09A8FDF758FD5E4806F032
:10747000D1FA61E05D4806F0CDFA5D4806F0CAFA3F
:107480000699009800F01EFE5A4806F0C3FA04213F
:1074900000980844FFF788FF574806F0BBFA102110
:1074A0005648FFF781FF564806F0B4FA10215548B8
:1074B000FFF77AFF4B4806F0ADFAD7E7102206989F
:1074C0000FF04EFE5049514B002808BF1946504856
:1074D00006F0A0FA002D3DD03D4806F09BFA3D4A4B
:1074E000214609A8FEF77DFA4A4806F093FA0821DA
:1074F0000098FFF759FF484806F08CFA08210998D0
:10750000FFF752FF454806F085FA10210398FFF770
:107510004BFF434806F07EFA10210698FFF744FF20
:10752000304806F077FA0998039B069A009900F014
:107530007DFE09A8FDF7F2FC2A4806F06BFA06A8C2
:10754000FDF7ECFC03A8FDF7E9FC6846FDF7E6FC57
:107550000DB030BD254806F05DFA324806F05AFA03
:10756000039A0699009800F0EFFD224806F052FABF
:10757000042100980844FFF717FF2B4806F04AFA49
:1075800010211E48FFF710FF284806F043FA10218B
:107590002748FFF709FF274806F03CFA1021264844
:1075A000FFF702FF254806F035FA16481021FFF7CD
:1075B000FBFE0C485BE700BFB8B9010811BA01082F
:1075C000E0B90108E7BA010874CB01088BCB0108C8
:1075D000A6CB0108D8B90108ACCB0108BDCB010886
:1075E000CFCB010882C4010877CC0108EFCB01089A
:1075F000F4CB010826CC010838CC0108AC010020EE
:1076000064CC0108DC01002083C401085DCB0108C3
:1076100096CC0108B3CC0108C5CC0108D8CC010830
:10762000F8CC010843CD01087DCD0108E9CD010862
:10763000BC01002000CE0108CC01002017CE0108BB
:1076400010B5084CD4F834221AB959210648FCF771
:10765000DFFDD4F834020023BDE8104003222021CE
:10766000FBF750BB100000200EB90108F0B51F4613
:107670001446C7B005460E46F122002109A80FF0B6
:10768000A2FD09AA1021384603F022F8204610F086
:107690004AFD07461022002101A80FF094FD102F8B
:1076A0003A46214628BF102201A80FF068FD09AA1A
:1076B00005A901A803F086F8324605A928460FF06F
:1076C0005EFD47B0F0BD000038B50C4C0C4D94F891
:1076D0002F30022B0ED1082394F8F321D4F8F411A3
:1076E000012002F0ABFF6B6B00209847042384F865
:1076F0002D3038BDEB6A98470123F8E710000020D1
:10770000ACE60108044B5A7F22B993F8330080F0AD
:10771000010070470020704710000020F0B570276E
:107720009DB006460D463A46002168460FF04BFDD7
:1077300008212B460DEB010004AC0B4AFFF796FF26
:107740002B462046094A102108ADFFF78FFF94E829
:107750000F0085E80F003A46694630460FF00FFDEE
:1077600030461DB0F0BD00BFF4CF0108FCCF0108CA
:1077700008B5054806F04EF9044A92F8F83101338D
:1077800082F8F83108BD00BFA6CF01081000002024
:107790000022024B83F8F821704700BF1000002040
:1077A000014B93F8F90170471000002084B070B5C8
:1077B0008AB00EAC84E80F00704C4FF4107225466E
:1077C000002120460EAE0FF0FEFC0FCE0FC596E84E
:1077D000030014AB85E803000FCB04F1180585E81E
:1077E0000F000E9B0BB9664B23600F9B0BB9644BCC
:1077F0002360109B23B94FF4C2716248FCF708FD67
:10780000129B23B94FF4C4715E48FCF701FD119B34
:1078100023B94FF4C6715B48FCF7FAFC139B23B9FC
:107820004FF4C8715748FCF7F3FCA3690BB9032365
:10783000A36101F015FF94F8203013B9012384F8F7
:10784000203001F005FF636A0BB94F4B636201F012
:10785000F3FE09F0C3FFC4F830020138033008D941
:107860004A486368984700200AB0BDE8704004B0F9
:107870007047002204210120FBF7DAFF0322C4F83D
:107880003C0200210120FBF7D3FFC4F8380220B9E5
:107890004FF4DB713B48FCF7BBFC002204210120C4
:1078A000FBF7C6FFC4F83C0120B94FF4DD71354841
:1078B000FCF7AEFC002204210120FBF7B9FFC4F85D
:1078C000400120B940F2BD112E48FCF7A1FC4FF455
:1078D0008163A4F80032002384F83430012384F853
:1078E000043206F0C7FD05AD68B9A36822690593A7
:1078F000236807920893E26863680692009395E80C
:107900000F0006F0D1FD06F0BBFD84F8320001F057
:10791000E7FE23681E4E0793636806F1A0020893F2
:10792000236904960693E368F03605930AAB43F89F
:107930001C2D93E803008DE8030095E80F0002F08A
:1079400007F90196A3694FF4CD7200931149012301
:107950001148FAF777FA012804D04FF4F171094879
:10796000FCF756FC002303220421D4F83402FBF771
:10797000C9F9012084F8310076E700BF100000202B
:107980000DDA00080EB9010808E6D33330CF01083C
:107990005401002063CF0108917E000810B50F4C00
:1079A000D4F8343223B940F2EB110D48FCF730FC27
:1079B000002303220421D4F83402FBF7A3F942F296
:1079C0001071D4F83802FCF743F90023D4F83802D8
:1079D0001A46BDE810401946FBF74EBF10000020C4
:1079E0000EB9010838B50E4DD5F8383223B94FF429
:1079F000FE710C48FCF70CFC0021D5F83802FCF7AE
:107A000027F90128044608D10023D5F838021A4680
:107A10001946FBF731FF204638BD0020FCE700BFC8
:107A2000100000200EB9010810B5FFF7DBFF68B1A8
:107A3000074C0023D4F8340203220821FBF762F933
:107A4000D4F83402BDE81040FAF7AABB10BD00BF5D
:107A500010000020002313B502A941F8043D4EF6A2
:107A60005E224EF66023441E94428CBF02461A46A4
:107A7000034BD3F84001FCF759F8019802B010BD50
:107A80001000002010B50648FFF7E4FF044620B9B7
:107A90004FF40A710348FCF7BBFB204610BD00BF42
:107AA000E09304000EB9010838B5FFF79BFF194BAE
:107AB00020B15B6818489847002038BDD3F83C01D6
:107AC000FCF754FA04460028F6D1014602F03CF9CE
:107AD00005460028F0D0047001F0C2FC044618B935
:107AE000284602F07FF9E7E70C4A13680133136078
:107AF00073B9136801331360636004232046237055
:107B000001F0D2FC10B9204601F0BCFC6068D4E75B
:107B10001368F1E7100000206BCF0108300C002043
:107B2000F0B58BB005460C4617460193FFF75AFF98
:107B300010B100200BB0F0BD4B4ED6F83C01FCF765
:107B400015FA0028F5D1002F5CD1002CF1D1284680
:107B5000214602F0F9F805460028EAD09DF80530E4
:107B6000002B52D004230370FFF702FE0F2206A958
:107B700003A805F063F89DF804303BB10D230AA972
:107B800001F8203D012203A805F066F89DF80630B3
:107B90003BB102230AA901F8203D012203A805F008
:107BA0005BF896F82E2096F82F30934203D196F882
:107BB0003030934217D02023022A18BF00228DF8BC
:107BC000083095F8783002A90BBF43F0040343F066
:107BD00001038DF809208DF8092003A885F8783075
:107BE000022205F039F896F81432059996F8F0015A
:107BF0001944C9B201F0FAFE844209D9284602F0BC
:107C0000F1F896E7E02F94D8A1E702230370ADE7DF
:107C1000059A32B1D2B20399284600F0BFFF00287E
:107C2000ECD06F77284601F01BFC07460028E5D012
:107C300000230E4A836013680133136083B913680D
:107C4000013313607B60022338463B7001F02CFC4B
:107C500040B9384601F016FC73680548984768E754
:107C60001368EFE7786865E710000020300C00200B
:107C7000DACF010813B51C460023ADF804308DF8A7
:107C800006308DF80520019B2246FFF749FF02B020
:107C900010BD0000034B93F8141293F8F00101F0AB
:107CA000A5BE00BF100000200E2808BF0120024B17
:107CB000D87783F8F001704710000020024B83F85A
:107CC000200083F8F10170471000002008B505F08E
:107CD00089FF024BC3F8480108BD00BF1000002017
:107CE000034630B5054C00F1100522461868596866
:107CF000083303C2AB421446F7D130BDCC0100209B
:107D0000034630B5054C00F1100522461868596845
:107D1000083303C2AB421446F7D130BDBC0100208A
:107D2000034630B5054C00F1100522461868596825
:107D3000083303C2AB421446F7D130BDAC0100207A
:107D4000034630B5054C00F1100522461868596805
:107D5000083303C2AB421446F7D130BDDC0100202A
:107D600010B50446FFF7BCFF2046FFF7C9FF2046C9
:107D7000BDE81040FFF7D4BF30B51025C3B0224C8A
:107D8000F122002105A80FF01EFA2A46002101A8C1
:107D90000FF019FA94F85B3105AA8DF8053094F8C4
:107DA0005A3129468DF8063094F8593104F5B670E9
:107DB0008DF8073094F858318DF8083094F8573121
:107DC0008DF8093094F856318DF80A3094F8553111
:107DD0008DF80B3094F854318DF80C3002F078FCAB
:107DE000052305AA04F5C67101A88DF8043002F038
:107DF000E9FC062305AA04F5BE7101A88DF804303C
:107E000002F0E0FC43B030BD100000200246024BFF
:107E10000068516803C370475C0100200246024BB2
:107E20000068516803C3704764010020034630B501
:107E3000054C00F11005224618685968083303C242
:107E4000AB421446F7D130BD6C010020034630B57B
:107E5000054C00F11005224618685968083303C222
:107E6000AB421446F7D130BD7C010020014B98771E
:107E7000704700BF1000002038B5044600680D466A
:107E8000884203D008B101F0FDFA256038BD00003A
:107E90002DE9F04105F024FF0123764CDFF8DC8169
:107EA000754E84F82D300A23744A4FF0FF310020BC
:107EB000FAF7DEFE012866D1D8F8000043071AD58C
:107EC000337833B109F0EAFB002009F03BFC0023D2
:107ED0003370FBF78FFAFBF7ADFA022384F82D30ED
:107EE0000023D4F838021A461946FBF7C5FC0020D7
:107EF000FAF7C0FBD7E710F0080721D033787BB939
:107F000041F2883009F0F6FB18B99A215C48FCF779
:107F10007FF95C4809F016FC01233370FFF7D4FBAE
:107F20000020FAF7E9FF4FF4FA61D4F83802FBF7C2
:107F30008FFE0028B7D1A1215148FCF769F9B2E7BB
:107F400010F020003FD03378D3B194F82D30042BBB
:107F500016D14D4D3A462946D4F83002FBF728FF9A
:107F600001280DD12B78072B2AD03A462946D4F880
:107F70003002FBF7DBFD012802D1284609F0E8FBBF
:107F80000020FAF7B9FF3378002B8CD001F0A0FA6B
:107F90000546002887D00378012B1AD194F82C10BD
:107FA000A26A01B192B9B2FA82F23848520905F0D8
:107FB00031FD284601F0EEFA284601F063FA72E737
:107FC00001F016FADCE7FAF797FF6CE701F05AFACE
:107FD000A56A032384F82D302B78052B46D8DFE8DB
:107FE00003F003450A0A3A3AD4212548FCF710F970
:107FF000FFF76AFB57E729462548FFF73DFFFFF7E4
:1080000081FB68B101F076FA054618B9E0211C48F9
:10801000FCF7FEF8022328462B7001F095FAE7E7FB
:1080200001F068FA074618B9E7211548FCF7F0F89F
:108030003946284600F028F97B7E53B14FF47A7018
:10804000FAF79AFA3946284600F01EF97B68002BA9
:10805000F2D03846E1E70E480021FFF70DFF284631
:1080600000F038FE284601F00DFAC1E763680948C0
:108070009847F7E710000020340C0020440C002043
:108080000EB9010841760008380C0020CCCE01085A
:10809000380000200CCF010813B50024074802ABBC
:1080A00090F8F11143F8044D054A90F8320005F0BC
:1080B000EBFF2146019802B010BD00BF1000002068
:1080C0006182000830B50430C7B00D46FFF7FEFDF1
:1080D0001B4B0DF1050203F10C0153F8040B8B420D
:1080E00042F8040BF9D11B880124138000238DF87A
:1080F0001330022309AA102128468DF8043002F01B
:10810000E7FA09AA05A901A802F05CFB05A8FFF798
:1081100017FE09AA102128468DF8044002F0D8FA6B
:1081200009AA05A901A802F04DFB05A8FFF718FE52
:108130001022044B5C771A7783F8442147B030BD96
:1081400097CF01081000002030B50430C7B00C46AE
:108150001546FFF7BBFD284B0DF1050203F10C019D
:1081600053F8040B8B4242F8040BF9D11B882046CC
:10817000138000238DF813300223012409AA102153
:108180008DF8043002F0A4FA09AA05A901A802F0AA
:1081900019FB05A8FFF7D4FD09AA102128468DF880
:1081A000044002F095FA09AA05A901A802F00AFB09
:1081B00005A8FFF795FD032309AA05A901A88DF8D5
:1081C000043002F0FFFA05A8FFF79AFD042309AA7C
:1081D0000DEB030005A98DF8043002F0F3FA05A8B1
:1081E000FFF79EFD1122054B5C771A7783F8442137
:1081F00083F8FD4147B030BD97CF01081000002043
:1082000038B50D461446FFF701FE2846FFF706FE77
:108210002046FFF70BFE2046FFF718FE0022024B18
:108220005A7710221A7738BD1000002070B50E461C
:1082300015461C46FFF7EAFD3046FFF7EFFD2846DE
:10824000FFF7F4FD2046FFF701FEBDE87040002275
:10825000024B5A7711221A77FFF78EBD10000020CB
:10826000002310B54168074C1A19106C884202D1DE
:1082700092F83C0020B91033B3F5807FF4D1002090
:1082800010BD00BF100000202DE9F04F064689B058
:108290000C4619B918216C48FBF7BAFF16B13378B0
:1082A000022B03D01A216848FBF7B2FF33691BB9D0
:1082B0001B216548FBF7ACFF33691B78042B05D005
:1082C000022B03D01D216048FBF7A2FF00225F4D67
:1082D000337895F8F1716370D5F8F431394603932A
:1082E00008AB43F80C2D95F83200594A95F8F0B1D7
:1082F00095F8F2A195F8F39105F0C6FE804620B9F5
:108300000123237009B0BDE8F08F059B33B101F064
:10831000EFFB03232370059B6360F3E7B36801332E
:10832000012BB36011D1D5F8E42130690132C5F8D1
:10833000E421B5F8FE2185F82C300132A5F8FE21A4
:1083400000F0DEF8306900F049FCD5F848213369C7
:108350005A60D5F8E4215A8195F8F92142B10022FA
:1083600085F8F9211A7A42F004021A72B5F8FA2156
:10837000A3F87A20404601F0D9F9034695F8F02198
:1083800005EB001130694FF0000880F87D3080F86F
:108390007C2095F804224FF47A7312F00F0208BF84
:1083A00001225A4307AB019306AB00933C3102F51F
:1083B0007A73CDF8188000F0F7FE0028A0D0F9F706
:1083C00083FFF060D4F8A00084F8008008B101F0C9
:1083D00009FD069B0798C4F8A030C4F80A0022469D
:1083E00031461C4800F05EF88022316904F120001B
:1083F0000EF0C5FE0021039B0798636195F83330AA
:10840000C4F80A00C4F8881084F810B0677484F8BF
:1084100012A084F8139021702376B26895F8023286
:10842000D4F8A0009A4200D258B1617685F82C1099
:10843000003018BF0120617E0090074805F0EAFA7D
:1084400060E701216176F3E70EB901081000002012
:10845000618200083800002003D0010808B5104AE6
:1084600010B10023A2F8FE31937FBBB1B2F8FE3108
:1084700092F800128B4211D95B1A92F8011293FB09
:10848000F1F201FB12334BB901F0F2F830B901F00F
:10849000FDF818B9BDE8084001F008B908BD00BFF3
:1084A0001000002070B5D2F8A04006461546E4B191
:1084B0000021204601F07CFBFFF76AF92378204673
:1084C000052B01BF012386F8D1316389A6F8D2318B
:1084D000FFF7C4FFD5F80A10204600F0B5FB237A59
:1084E0005B0701D501232B7270BD2046FFF7B6FF55
:1084F000D5F80A102046BDE8704000F0A5BB00008A
:10850000134B10B49A7F02B3027A93F8F01142F041
:1085100001020272DA7F914208D193F83C40A4B183
:1085200093F84C408CB193F85C4074B1B3F8FE41C1
:1085300093F800329C4208D9914206D0037A10BCCD
:1085400043F002030372FFF713B910BC704700BF7A
:1085500010000020431EDBB21F2B96BF0D4A0023E4
:10856000D35C0A280BD8012202FA00F010F4A46FA1
:1085700005D0094A92F814221A440E2A07DC074A49
:10858000107818440E28CCBF00200120704700202E
:10859000704700BF40D0010810000020570C002099
:1085A00070B5057804462846FFF7D4FF88B1094A1C
:1085B000094E1378F5540133137051B1074A2478EA
:1085C00092F81432D01880F805420846013382F838
:1085D000143270BD570C0020480C00201000002001
:1085E0002DE9F04F002593B0CDE907019DF870808B
:1085F000B74E0992059345450AD2059B595D5F190F
:108600000846FFF7A7FF029028B9B24805F002FA22
:1086100013B0BDE8F08F01391F2900F2A682DFE810
:1086200011F02000A4022C0054027D016101C4015C
:1086300042025402EB01A40256022C016D026F02A9
:10864000A402A402A402A402A402A402A402A402FA
:10865000A402A402A402A402A402A402A402A402EA
:108660009102A8EB0503DBB2012B4FF0000400F0F0
:10867000028186F8FD410224FDE0A8EB0503DBB290
:10868000039307238DF8383000231C460193039A87
:10869000231D934202DA3B5D032B10D0019B2BB1CB
:1086A0009DF838306FF300038DF838309DF838307E
:1086B000072B40F0D2800024DFF81C92C6E03B1963
:1086C000D3F8012005345FFA82FB0BF00F034FEA69
:1086D0001B1B0693BBF1060FC2F30F23E4B24FF04E
:1086E00000090F92049303D902F0F003F02B2FD16D
:1086F0004FF6FF73C2F30762049902F07002602A1A
:1087000008BF194600230A469A4611465FFA8AF0C6
:108710000B930A9201F07CF8DDE90A2380B106EBA5
:108720000A11096C61B106EB0A1191F844104FEA85
:10873000111C01F00F01594502D8E34598BF0346CB
:108740000AF1010ABAF1100FDFD10BB14FF00209A3
:10875000069B072B05D99DF83C3003F00F030F2B28
:1087600001D149F004099DF83FA00AF0700ABAF15E
:10877000600F0CD149F00109BAF1000F0FD0DDE90B
:108780000132BAF1600F18BF1346019307E0BAF146
:10879000000FF4D1049801F019F80028EAD19DF8EF
:1087A0003830C9F3400269F3000362F34103C9F3AF
:1087B000800969F382038DF8383068E73B19D3F8F4
:1087C00001A09DF83830053403F00703072BCDF8DE
:1087D00040A0E4B23AD19DF84030C3F30311CAB2CD
:1087E00086F8F0110AF00F010F290BD021B90121F1
:1087F00061F303038DF840309DF84030C3F3030369
:1088000086F8F1319DF84310CAF30F20C1F302112D
:1088100001F004F820B940F275114846FBF7F8FC66
:1088200096F84431102B09D11AF0706F01BF012264
:108830009DF8433062F303038DF843309DF84330D5
:108840001A0703D0C3F3030386F80232039A231DE9
:108850009A4202DD3B5D032BB0D054B1032312A832
:10886000002100F8083DFFF79BFE00210EA8FFF74E
:1088700097FE01F03DF92C444AE0A8EB0503DBB27A
:10888000052B40F27081781C05F0B3F997F905309B
:108890000021002B22DB0CA3D3E9002312184B414B
:1088A000002196F8040210EB020941EB030A099B30
:1088B000022B03D119F101094AF1000A079BC3E910
:1088C0001C9A0624D7E700BF6E3DD51200000000B9
:1088D0001000002060D001080EB90108A8A3D3E958
:1088E0000023DBE7062312A800F8103D0021FFF764
:1088F00057FE089B12AC03F01F0304F8083D00214B
:108900009B48FFF74DFE20460021FFF749FE6C1CF7
:10891000E4B2A5423FF47CAE25466CE6A8EB050325
:10892000DBB2042B4FF00004A5D9D7F801308DF845
:1089300034401093DBB2C3F30212052A9CBF86F8C1
:10894000F221E2B2C3F303039CBF42F004028DF8AC
:108950003420062B9CBF86F8F3319DF834300DF19E
:1089600041009CBF43F002038DF83430642405F0CD
:1089700042F94443204605F063FC9DF8343088B149
:10898000C6F8F44143F00103052412A800F8104D85
:1089900001218DF83430FFF703FE01210DA8FFF708
:1089A000FFFD68E760F30003EEE7A8EB0503DBB229
:1089B000052B40F2D88057F8010F3B7910900DF14C
:1089C00041008DF8443000F0A7FE9DF84420014698
:1089D0009DF8400000F0BEFE8DF8340001F088F8EC
:1089E000072312A800F8103D0021FFF7D9FD002150
:1089F0000DA8FFF7D5FD64E7A8EB0503DBB2042B58
:108A00004FF000047FF637AFD7F801300DF1410089
:108A100010938DF8344000F07FFE044602469DF826
:108A20004010544804F0F6FF204605F009FC28B138
:108A30009DF8343043F001038DF834309DF8403018
:108A40000F2B2ED801331B0103F12C02334493F872
:108A50002C10324439B11B6B2BB19DF8343043F0EC
:108A600002038DF834309DF8343012A803F003036C
:108A7000032B4FF00A0308BFD46000F8103D01211A
:108A8000FFF78EFD01210DA8FFF78AFD9DF8341038
:108A90003948C1F3400201F0010104F0BBFF052495
:108AA000E9E60022DFE7A8EB0503DBB2012B5AD091
:108AB0007B78012103F00F0386F80432082312A803
:108AC00000F8083DFFF76CFDD5E5AC1C20E7A8EBEE
:108AD0000503DBB2012B46D001237A7812A81109D5
:108AE00002F00F0203FA01F1934086F801320C23E1
:108AF00086F8001200F8083D0021E3E7EC1C07E7C8
:108B0000A8EB0503DBB2012B2DD0B3687C78984726
:108B100001221A4B8DF83820C3E9000123090A33DA
:108B200002FA03F3C6F820320F2312A8002104F042
:108B30000F0400F8083DC6F82442FFF731FD00217C
:108B40000EA8BFE7A8EB0503DBB2012B0BD07B78A7
:108B50000BB1022B07D196F830209A423FF48BAD2F
:108B600086F8303087E5002485E62C46D1E600BF44
:108B70001302002097D00108B6D001082802002077
:108B80006F3DD5120000000038B10078032803D0F3
:108B9000431F58425841704701207047037A70B50F
:108BA0001B09D61804460F2E00F10C001546184478
:108BB00009DC0EF0E4FA0120237A05EB131565F3C6
:108BC0000713237270BDC3F10F020EF0D8FA237A97
:108BD000002043F0F0032372F4E7000073B5134D57
:108BE00006462A78124CBAB11249FFF7D7FF0F2276
:108BF000002110480EF0E7FA00232B7094F8FD31A5
:108C000043B140F2011302A921F8043D022230468B
:108C1000FFF7C4FF02B070BD94F81422002AEDD013
:108C200004F20521FFF7BAFFE8E700BF570C002068
:108C300010000020480C0020024B00F00F0083F8C9
:108C40000402704710000020F0B585B0039104467F
:108C500010B3FFF799FFF8B10020144B9DF90E10E7
:108C600083F8050283F81402207A93F81EC09DF859
:108C70000F200609677F257FBCF1000F05D010F09B
:108C8000010018BF012083F8FC013EB1009604F1F9
:108C90000C032046FFF7A4FC05B0F0BD002FFBD16C
:108CA000002DF9D00095A36EF3E700BF100000205F
:108CB000002310B54168064C1A19106C884202D185
:108CC00092F83C0018B91033302BF5D1002010BDBC
:108CD000100000202DE9F04F054689B018B1037847
:108CE000043B012B03D91E21BB48FBF791FA2B69EA
:108CF0000BB11B781BB11F21B748FBF789FAB74CA2
:108D000094F8F33194F8F1810393D4F8F43194F8A2
:108D1000F0B1029394F8F2A100F09AFC00F0A0FCEC
:108D2000002208AB43F80C2D4146AD4A94F83200BE
:108D300005F0AAF928B9284600F02CFC09B0BDE8D6
:108D4000F08F00F0F3FC059B07469BB100F0D0FECE
:108D500000F0D0FB044618B93B219F48FBF758FAB6
:108D60002B782046637003232370059B636000F01B
:108D7000EBFBE3E7AB68227F0133102AAB602ED117
:108D8000012B09D1D4F8E4310133C4F8E431954B17
:108D90005B699847A4F8DC01B4F8DC310133A4F82E
:108DA000DC31002607AB94F8F39184F8F36101936A
:108DB00006AB009304EB071141F2707341F2883265
:108DC0003C312869069600F0EFF9B0B9284600F06A
:108DD000E1FB069801F006F884F8F391AEE7112A5A
:108DE00006D1636904F5A6709847A4F8DC01D8E7BA
:108DF0004E217948FBF70CFAD3E7069A84F8F391F1
:108E000012B11378012B06D0284600F0C3FB069858
:108E100000F0E8FF92E7237F102B40F098801023AA
:108E2000002684F84431069BDA6803F16307C4F82E
:108E3000482103F15302002E00F098801121DFF841
:108E4000B4C184F84411664610685168083203C6FC
:108E5000BA42B446F7D1644F03F1230203F1330C55
:108E60003E4610685168083203C662453746F7D15E
:108E70005E4F03F1330203F1430C3E461068516824
:108E8000083203C662453746F7D1594F03F1430212
:108E900003F1530C3E4610685168083203C6624520
:108EA0003746F7D19A68A2631A7CC2F3030284F8AA
:108EB000F3211A7CC2F3021284F8F221587CFFF7E6
:108EC000BBFE002394F82E20069812F0FD0F00F14F
:108ED000120018BF84F82E30C4F8EC31C4F8E83121
:108EE000C4F8E43184F82F3084F8303000F0D8FC36
:108EF00000F0FEFD012384F8333000F0FBFA064653
:108F000018B9CA213448FBF783F98022296906F190
:108F100020000EF034F90023069A0798C6F8A02026
:108F200094F83320C6F8883032769DF80C203370E0
:108F3000F2742B78029AC6F80A0086F810B086F808
:108F4000118086F812A07261737030460FE7112B02
:108F500007D192F82260002E3FF461AF84F84431CB
:108F600061E77C211C48FBF753F95CE71021DFF82F
:108F700084C084F84411664610685168083203C6FC
:108F8000BA42B446F7D1184F03F1230203F1330C70
:108F90003E4610685168083203C662453746F7D12D
:108FA000124F03F1230203F1330C3E46106851685F
:108FB000083203C662453746F7D10D4F03F123024D
:108FC00003F1330C3E4610685168083203C662450F
:108FD0003746F7D166E700BF0EB901081000002040
:108FE000B18C0008ACE60108CC010020BC010020D7
:108FF000AC010020DC0100202DE9F04385B00746DC
:109000000C468DF80F202BB101220DF10F0100202D
:1090100008F01AFFF9F758F91D4B1E4D1E4E9DF82A
:109020000F1080469B6A2046984741F288322946B5
:10903000D6F83002FAF77AFD40B32B78012B20D115
:109040002846AC6808F084FB4FF47A70A4EB08095A
:1090500009FB00000DF03EFA7968024696F83200EE
:1090600005F0BAF800F044FDCDE900499DF80F1075
:10907000356843467A680948A847204605B0BDE8E8
:10908000F083284608F064FB0024F6E70446F4E782
:10909000ACE60108580C002010000020FBD10108AC
:1090A0002DE9F84F394E9846736B054689461446AC
:1090B0004FF47A7A9847DFF8DCB0354F0AFB05F2B7
:1090C00002F59C328032B2FBFAF23249D7F8300214
:1090D000FAF72CFD20B9336B98474FF0FF302FE0A3
:1090E0009BF80030072B07D1584608F031FB4FF4AE
:1090F0007A6508F039FEE1E7032B366B22D1DBF805
:10910000045028792968844228BF044648462246EC
:109110000EF035F83F6895F90830B5F90620A988B2
:109120001D48B847B8F1000F05D0EB88A8F800300B
:109130002B7A88F80230174808F00AFBB04720461F
:10914000BDE8F88F042B0BD1124808F001FBB047A3
:109150003C68F9F7B9F801461048A0470020EFE74E
:10916000052B09D10B4808F0F3FAB0473C68F9F732
:10917000ABF801460A48F0E7F2210A48FBF748F845
:10918000044808F0E5FAB047A7E700BFACE60108DD
:1091900010000020640C0020A3D10108CDD10108EB
:1091A000E5D101080EB901082DE9F04F8A4CC9B08C
:1091B0000F4691469846FF2294F8443108A982460A
:1091C000539E00F027FE029018B9002049B0BDE878
:1091D000F08F94F8F01194F8F2517A688D4298BFAC
:1091E0004D1B084694BFEDB20025D4F800B005929F
:1091F000049100F0A7FB039094F8F10100F0B8FB94
:10920000DDE90412039B00907448D847FA682846A9
:10921000D4F800B0039200F095FB039A0346294668
:109220006F48D84794F8F311D4F8F4210846D4F8DD
:1092300000B00492039100F085FBDDE903120346C0
:109240006848D847236842464946674898470121FD
:10925000504600F0ADFC94F8F13194F8F0217968B3
:10926000002001F0EBF90023029A08A93846FFF725
:10927000C3FE04460028A8D09AF8783013F0050FF2
:109280000BD013F0040F0CBF00220222524B93F8B4
:109290002F10914218BF83F82F20FF22002108A829
:1092A0000DF091FF2A460823F968012001F0C6F964
:1092B000A9F114000CF0D4FC43A3D3E900230CF073
:1092C00049FD0CF0E1FF054609F2AB200CF0C8FCAB
:1092D0003FA3D3E900230CF03DFD0CF0D5FF07467A
:1092E000A8F114000CF0BCFC37A3D3E900230CF068
:1092F00031FD0CF0C9FF4FF47A79A0F11403BB42A1
:1093000094BFC5EB0307C5EB070709FB05F18246D0
:10931000B1FBF9F107A80794F9F7EEF8FF223346FD
:1093200008A93846FFF7BCFE421C05463FF44DAF86
:109330000028294F1ADDD7F80080F8F7C5FF23462B
:10934000024629462948C0470EB10123F370002385
:10935000529A9D42136007DD97F84421E9B208A8AC
:1093600001F0FEF8529B186001202FE7082397F8C0
:10937000F321D7F8F411012001F060F909FB0AF19B
:1093800007A8B1FBF9F10794F9F7B6F808F2AB209A
:109390000CF066FC0EA3D3E900230CF0DBFC0CF010
:1093A00073FF3346FF2208A9A0EB0A00FFF778FEFF
:1093B000431C05463FF409AF0028C8DD002EC6D087
:1093C0000223C3E7AFF300800AD7A3703D0AEF3F43
:1093D000A4703D0AD7A3F03F10000020DFD00108A1
:1093E00011D1010837D101085DD1010878D10108F8
:1093F00030B5C3B06B46FF2202A94FF47A60FFF785
:109400004FFE051E24DD0023144C0193D4F848219F
:1094100094F84431E9B202A800F044FE03460190FA
:10942000B0B10278052A01D0032A14D118460021D0
:1094300000F0BEFB0198FFF711F8DDE90010FFF71F
:1094400003FC0023012201A9D4F83C02FAF714FA24
:10945000284643B030BD00F0C5FCF9E710000020FD
:1094600038B5074B0546DB6814209847044620B101
:10947000102200210DF0A7FE2561204638BD00BF57
:109480001000002010B5044650B1006900F0AAFC9D
:1094900000232361034B2046BDE810401B69184799
:1094A00010BD00BF10000020002307B502A941F83D
:1094B000040D06481A46D0F83C01FAF7DDF9431EC0
:1094C0005842584103B05DF804FB00BF1000002073
:1094D000002307B50193064B93F8342022B901A964
:1094E000D3F83C01FAF722FB019803B05DF804FBC6
:1094F00010000020064B10B5DB68A82098470446F2
:1095000018B1A82200210DF05EFE204610BD00BF5C
:109510001000002010B5044698B1D0F8883013B17F
:10952000203000F049FCD4F8A00020B100F05AFC33
:109530000023C4F8A030034B2046BDE810401B694F
:10954000184710BD100000201FB5104C0190D4F832
:109550004001FAF71DFD024640B903A9D4F84001C5
:10956000FAF7E4FA10B10398FFF7D4FF002301A93A
:109570001A46D4F84001FAF77FF920B940F2751184
:109580000348FAF745FE04B010BD00BF10000020EC
:109590000EB9010838B50546FFF7ACFF044620B9FF
:1095A0004FF4BD710548FAF733FE012323702B7881
:1095B00020466370BDE83840FFF7C6BF0EB901080A
:1095C00010B50D4C031D04EB031319719A600123B0
:1095D000013004EB0010026380F82C30114694F83F
:1095E000320004F035FE28B9BDE810400B210348D5
:1095F000FAF70EBE10BD00BF100000200EB9010822
:10960000002301460B4870B41A4606461D1895F80B
:109610003C401CB12D6C8D4208BF22461033B3F57F
:10962000807FF3D122B996F8320070BC04F0A2BE5C
:1096300070BC704710000020044B93F8212083F881
:10964000F3215A6AC3F8F421704700BF10000020CC
:10965000024B93F8202083F8F1217047100000207E
:10966000024BDA7F83F8F021704700BF1000002022
:10967000054B93F8202093F8F11191423ABF012055
:1096800083F8F1210020704710000020064A92F86C
:10969000F031D17F99423DBF03F1FF33012082F8C1
:1096A000F0310020704700BF1000002010B550249A
:1096B000084A21460020FFF783FF2146064A012081
:1096C000FFF77EFF2146BDE81040044A0220FFF765
:1096D00077BF00BFA027BE33E034C1332042C4337C
:1096E00010B50C4CFFF7A8FF94F8320004F06EFEA2
:1096F000FFF7DCFF5021002204F1740304F5A2748B
:10970000197043F8042C5A6003F8082C1033A34254
:10971000F6D110BD10000020437882781B0200783B
:1097200043EA02430343642058437047002330B5A3
:109730004168074C04EB0312156CD8B28D4202D17C
:1097400092F83C201AB90133102BF3D1002030BD20
:1097500010000020C31E0C2B2DE9F04105460E46DB
:1097600090464FF0000401D920460CE069B9164B31
:10977000013503EB0515286B85F82C10FFF740FF2A
:109780004FF003002E63BDE8F081C8F30317062FE6
:109790008CBF00270127084604F052FD67F3000440
:1097A00060F3410404F00303032BDDD1064B28468C
:1097B00003EB05131F6C32464146FFF701FF3846A5
:1097C000FFF71EFFD0E700BF10000020002110B5FA
:1097D0000C460C4BC20709D503EB0112146C24B9DB
:1097E000094804F017F9204610BD01240131102961
:1097F0004FEA5000EED1002CF5D1044804F00AF9EC
:10980000F1E700BF1000002073D201088FD20108D9
:1098100041FA00F000F00100704700004FF6FF73BE
:10982000062914BF0146194600232DE9F0411B4DBE
:1098300017462E461A469E4690B0286CD8B141FA7B
:1098400003F406EB031C9CF844C00CF00F08B84569
:1098500002D8B7EB1C1F10D985F83CE00133102B60
:1098600005F11005E9D1694696F8320004F0D2FD01
:1098700010B0BDE8F0810446E3E704F0010485F888
:109880003C40002CEAD010AC04EB820402F1010C45
:1098900044F8400C5FFA8CF2E0E700BF10000020B3
:1098A00038B50446FFF738FF054604F0C9FC28B177
:1098B0002A464FF050010320FFF782FEE01CFFF71D
:1098C0002BFF054604F0BCFC28B12A464FF050019E
:1098D0000420FFF775FEA01DFFF71EFF054604F0EC
:1098E000AFFC28B12A464FF050010520FFF768FE73
:1098F00004F10900FFF710FF054604F0A1FC28B1B0
:109900002A464FF050010620FFF75AFE04F10C00E2
:10991000FFF702FF044604F093FC38B12246BDE88D
:1099200038404FF050010720FFF74ABE38BD000015
:109930000738C0B205289ABF014B185C0E2070474B
:109940002ED2010807289ABF014B185C00207047EF
:1099500034D20108052804D90628034818BF00207E
:1099600070470248704700BF90D0030048E80100EC
:10997000072810B5044604D940F277110348FAF7D6
:1099800047FC034B13F9240010BD00BF0EB90108BA
:109990003CD20108142810B5044613DD4FF4BE7103
:1099A0001148FAF735FC062C14DD082C14DD0A2CBE
:1099B00014DD0C2C14DD0E2C14DD152CB4BF00208E
:1099C000082010BD022803DD0428ECDC0620F8E79F
:1099D0000720F6E70520F4E70420F2E70320F0E78C
:1099E0000220EEE70120ECE70EB901080F2938B597
:1099F00005460C4604D940F2A7111348FAF708FCB3
:109A00000F2D12D8DFE805F00808080B0E0E0E0E19
:109A10001111111111111D1DC4F1330038BDC4F114
:109A20007300FBE7C4F1F200F8E740F2BF1106480B
:109A3000FAF7EEFB054B064A4FF4E07105480DF0CE
:109A40007DF90020EAE700BF0EB90108DDC001087A
:109A50005CD2010820D301082DE9FF41044600280B
:109A600038D000211D4B03EB011294422DD1CDB211
:109A7000616879B31A4B93F8320004F0D9FA94F87C
:109A80000080DFF868E0064616484FF47A72B8F1B5
:109A9000000F08BF7046217A6768E36801F00F0C79
:109AA0000909CDE90110B3FBF2F3CDF800C0B7FB13
:109AB000F2F229460C4803F0ADFF237853B130464B
:109AC00004B0BDE8F04104F0B1BA01311029CAD1A7
:109AD000FF25CDE704B0BDE8F08100BF4C000020B9
:109AE00010000020E4D20108F5D20108ECD20108F0
:109AF00038B5084803F08EFF0024074D28191034AC
:109B0000FFF7AAFFB4F5807FF8D10448BDE83840DC
:109B100003F080BFB9D201084C00002082C40108C4
:109B20000068704782B0034660B16A4659680068B1
:109B3000013B03C207221DF8021012F1FF3203F8A5
:109B4000011FF8D202B070470FB404B07047000094
:109B500030B585B06D4685E80F00104C95E80F00D4
:109B600084E80F0004F1100208A903C982E8030089
:109B70000BB90B4BE360A3680BB9094BA360636897
:109B80000BB1236833B9A36806489847064B636056
:109B9000064B23600123237605B030BD700C0020F6
:109BA000499B000833D501081171010801710108B2
:109BB0002DE9F34105464E4C4E4A4F48A3680E46E8
:109BC00000290CBF014611464C489847A3684C48F1
:109BD0009847696EA3684B4898472B784A48072BEB
:109BE00096BF4A4A4A4952F82310A7686A78B8478C
:109BF000A36848489847A368697F47489847A3687F
:109C0000297F46489847A368698945489847A368CB
:109C1000696844489847297A0B090193C1F3C00346
:109C20000093002E32D0C1F38003C1F34002A66836
:109C300001F001013C48B0472B7A13F0F00F11D02E
:109C4000A3683A486FF00B079847DFF8F48005F1F6
:109C50000C067F1B297ABA19B2EB111FA36810DB1F
:109C600033489847A368334898472B7F002B3AD155
:109C7000A36831489847A3682D4802B0BDE8F04179
:109C8000184716F8011B40469847E3E7C1F38003E5
:109C9000C1F34002A66801F001012848B0472B7AC1
:109CA00013F0F00FDED0A36820486FF00B07984741
:109CB000DFF88C8005F10C067F1B297ABA19B2EB0C
:109CC000111FA368CCDA16F8011B40469847F4E749
:109CD000AB6E4046995DB84701362A7FB3B29A42CF
:109CE000A768F5D8C7E70026DFF85880F5E700BF7A
:109CF000700C002074D301087BD301088CD30108B9
:109D0000A8D30108BED30108CFD3010854D301085A
:109D100084D30108E3D30108F0D3010806D4010875
:109D200025D401083DD4010858D401089DD4010868
:109D300082C40108EFD40108FED40108ADD40108A3
:109D400007D5010806D501082DE9F041184D8046D8
:109D50002B7E0E461BB9D1211648FAF759FAF22E7E
:109D600003D9D2211348FAF753FA2B688020984779
:109D7000044680B1802200210DF025FAB8F1000FD1
:109D800012D08EB12B6830469847074630B920462E
:109D90006B6898473C462046BDE8F0813246414614
:109DA0000DF0EDF92677A76600236370F3E700BF97
:109DB000700C00200EB9010838B5084D04462A7E03
:109DC0001AB9EC210648FAF723FA34B1A06E20B193
:109DD0006B6898470023A366237738BD700C00207A
:109DE0000EB9010870B5094C0546227E1AB9F72153
:109DF0000748FAF70DFA3DB12846FFF7DDFF636823
:109E00002846BDE87040184770BD00BF700C0020A8
:109E10000EB901082DE9F04F99469F4B17461A7E5F
:109E200093B005460E46984622B94FF485719B487B
:109E3000FAF7EEF9032F01D80024D8E02A786B78DE
:109E400043EA421333702B78022B02D0042B40F0EC
:109E50008D800023042F8DF82630EDD06B68737051
:109E60006B681B0AB370EB88F370EB7933716B6826
:109E7000CDF822309DF82630002B40F0C180052F10
:109E8000DAD006242A7AC2F3400302F001019B01D2
:109E900043EAC11343EA1213C2F3800243EA4213B6
:109EA000737195F808A04FEA1A1A631C9F42C3DD2C
:109EB0006A89DBB232556A890234120AF254D8F840
:109EC00010301A886B899A4204D040F269117348A5
:109ED000FAF79EF9D8F81030B9F1100F1B680A9301
:109EE0000FD9D8F8142002930DF122030193012316
:109EF000297A009358320023090905F10C0000F07B
:109F0000B5FFBAF1000F0BD004EB0A0B5F4593DBF2
:109F10003019524605F10C010DF031F95FFA8BF45E
:109F20002B7F002B77D0BC4286D26B7F04F1010AD5
:109F300033556A7F5FFA8AFAD8F81430002A68D15C
:109F400058330693AB6E06A907932B7F06EB0A00E6
:109F5000ADF8203000F07DFE5044C4B2A7425AD282
:109F600040F297114D48FAF753F965E7032B01D0FA
:109F7000052B01D101236DE7002B3CD1082F7FF683
:109F80005BAFD8F81440701C224652F8083FC6F860
:109F9000013053684360FFF7C5FD102F7FF64CAFCB
:109FA000224652F8103F06F10900C6F809305368FE
:109FB0004360FFF7B7FD122F7FF63EAFB4F898303D
:109FC00006A97374B4F8983005A81B0AB374132358
:109FD0002834CDE90646ADF8203000F004FE162FF7
:109FE0007FF62AAF1724059BC6F813306B66204610
:109FF00013B0BDE8F08FD8F80C30294898471BE71C
:10A0000040F25F112548FAF703F94FF0000A0524E2
:10A010004BE7883395E7E31C9F427FF70DAFB9F11B
:10A02000100F0FD1D8F8143006A9783305A8CDE960
:10A030000636ADF8204000F03DFD059B3351043459
:10A04000E4B2D4E7B9F1110F1FD1D8F814300BA93D
:10A0500003F1780268330B930DF122030F930A9BEF
:10A0600005A81093B5F87A300C92ADF8443095F805
:10A070007C300D968DF8463095F87D30ADF838403F
:10A080008DF8473000F04EFDD7E74FF4DD710348FF
:10A09000FAF7BEF8ABE700BF700C00200EB901085C
:10A0A0000CD501082DE9F04F904D9B462B7EA5B0B5
:10A0B00006460F46904623B940F2C7118C48FAF77E
:10A0C000A7F8022F29D900210846FFF73DFE0446D4
:10A0D00030B9EB6887489847204625B0BDE8F08F37
:10A0E00033785B0903703278072B02F00302427069
:10A0F00003D1EB68804898470CE0B8F1000F00F0FE
:10A100001D82012B40F0F381AB687C48F3E74246A7
:10A110007B4898472046FFF765FE0024DCE70AF1FC
:10A120008801A6E188687346B7E148680023B4E176
:10A1300002EB084806EB09000593CDF83880FFF7DD
:10A14000EFFC0AF168020DF1900A4AF8682D60668A
:10A15000514609A800F0AEFC099A616E059B8A423F
:10A160000FD0EB68674898470E99ED68DDF83230FC
:10A17000BDF830206448A84700212046FFF718FDAD
:10A18000C8E72A6908F10101002B3CD09160227ACE
:10A19000079304F10C03059313091A4606F108010D
:10A1A000059806930CF0EBFFBBF1100F079B0CD941
:10A1B0000DF132016A6901910021CDF8088000910A
:10A1C0005832DDE9050100F051FE237A1B0903F145
:10A1D0000C02974238D903F10D02974215D10023A2
:10A1E0004A482377EB689847667F002E7FF474AF68
:10A1F000237A1B093FF470AF237F002B3FF46CAF31
:10A20000EB68434877E75160C1E70933A9EB0300E6
:10A21000617FC0B220776A6961B958321E440A92E0
:10A220000B96ADF830002B689847A06620B9EB6814
:10A23000384860E78832F1E7514600F00AFD00280F
:10A24000D2DCEB68344856E700232377A366CBE7DC
:10A25000212F01D1012354E1EB6830484BE79DF8F1
:10A260004730043F09EB0700DB09FFF759FC6E6933
:10A270006066A3B30DF1600A0021302250460CF055
:10A28000A2FFFF2332468DF8603052F8083F0DF1EF
:10A290006100CDF8613053683836CDF86530FFF78E
:10A2A00041FCB6F860303A468DF8693049461B0AE1
:10A2B0000DF16B008DF86A300CF061FFCDE90A6A90
:10A2C00008F107080AA909A8ADF8308000F08BFC56
:10A2D000636E099A9A4225D0EB6811480BE728363D
:10A2E000CDE90A69A8F10408ECE700BF700C002072
:10A2F0000EB9010860D501086BD5010896D5010893
:10A30000E5D5010884D60108C3D60108DCD60108CA
:10A3100057D701080DD7010831D701088FD7010899
:10A32000ECD701089DF83F609DF83E30360446EAC0
:10A3300003269DF83D300DF143001E4366609DF8F5
:10A3400042709DF841303F0447EA03279DF84030B2
:10A350001F43A760FFF7E4FBE0609DF84720237CE4
:10A36000D10961F3C713110961F3061362F3030303
:10A3700023749DF84830637494F8213003B324AB00
:10A3800033F8472D9B786282237524AB33F8442D34
:10A390009B78A4F81520E37524AB33F8412D9B7806
:10A3A0002283A37624AB33F83E2D9B78A4F81B20A0
:10A3B000637724AB33F83B2D9B78E28384F820301D
:10A3C0006D6994F9102005F1280C002AB5F8981051
:10A3D00004F1230004F15303CDF860C018AA12DA87
:10A3E00005F11807ADF870100092083504F143022A
:10A3F00004F13301CDE919761B9500F0C5FC01236A
:10A4000084F8223068E6ADF86C101946CDE919677A
:10A4100000F079FC0023F3E7EB684D486BE6701C15
:10A42000FFF77EFB804501466060EB687FF46FAE0E
:10A430004146484898470023052F6377A7F1040950
:10A4400007D9737903F00F0308339945C4BFF35C50
:10A45000637796F80780B279637F42EA082296F81C
:10A4600005C0D5F814A06281002B7FF458AE0AF124
:10A4700058014FF0010ECDE90A166168BBF1100FCB
:10A48000CDF83210ADF830908DF836E029697FF6BE
:10A490004CAE002B7FF446AE4868217A4FEADC1EB2
:10A4A0006EF300014FEA5C1E6EF382014FEA1C1E40
:10A4B0006EF3C3014FEA10486CF3071180B22172AA
:10A4C000411E8A42BCBF08F101081FFA88F8BBF19F
:10A4D0000F0F7FF62DAE111AB1F5804F7FF728AE22
:10A4E0000346ED684FF480411B48A84712E6032B52
:10A4F00095D0052B93D0012B8ED1112F7FF4A8AED0
:10A50000002384F821306B691FFA87F828330A93F7
:10A51000731C0B9308F1FF33ADF8303033780AA980
:10A520000DF13D008DF83C3000F075FB00280DF179
:10A530003C093FF794AEEB680848DCE5032B01D0FB
:10A54000052BD8D1701CFFF7EBFA606073E700BFF2
:10A5500018D80108B8D501081DD60108CCD70108C4
:10A5600013460022FFF79EBD2DE9F0468DB09246BE
:10A5700099462D4A149B074693420C463AD02B4AE3
:10A58000934204D02A4A93422FD1002600E00226AB
:10A59000284DEB6A98472046EB689847012F4FF00B
:10A5A000000429D108230A22CDE90132AB693146E2
:10A5B0000B93CDE90877CDE90644CDE90444039433
:10A5C00000943B464A4602200B9EB0472146FF209E
:10A5D00007F026F9082007F019F9342139202B6CEF
:10A5E0000B930DB0BDE8F0461847AC211248F9F7BF
:10A5F0000FFECAE70126CBE74FF47A630127CDE9C6
:10A6000007430823CDE90173EB69CDE905440B93BA
:10A61000CDE9034722465146CDF80090334602204B
:10A620000B9CA0473946D2E790D0030020A1070039
:10A6300048E80100ACE601080EB901082DE9F34134
:10A640000446104615460E469846FFF783F907461E
:10A650002846FFF777F9C5B21DB9CB210948F9F7AC
:10A66000D7FD64B94046FFF783F9024600972B46B1
:10A6700031462046FFF778FF02B0BDE8F0810022A6
:10A68000F4E700BF0EB901080A680368534003608D
:10A690004A684368534043608A68836853408360D4
:10A6A000CA68C3685340C36070470B6810B514682C
:10A6B0006340036054684B686340436094688B68F0
:10A6C00063408360CB68D2685340C36010BD000014
:10A6D000A1F11003DBB2102B2DE9F0470C46154613
:10A6E00008D84FF0010909FA03F303F0013323F00E
:10A6F00080732BB90023FF2085F8F030BDE8F08788
:10A700000A46014628460CF03AFD04F11C0E4FEAB9
:10A710008E0E5FFA8EFE4FEA1E13013B85F8F03075
:10A7200023462749B3FBF4F204FB1232E81812F077
:10A73000FF0210F804AC10F803CC10F8027C10F8FB
:10A74000016C32D111F80C804FEAD91289EA08085D
:10A7500011F807C08F5D11F80A604FEA420A5244AF
:10A76000C24602EBC20282EA49025FFA82F91A1B70
:10A77000D2B215F802802A448AEA080A05F803A032
:10A7800092F8018004338CEA080C80F801C092F83A
:10A7900002C0DBB287EA0C078770D2789E4586EA52
:10A7A0000206C670BED80020A8E7182CDFD9102AF0
:10A7B00001BF11F80AA011F80CC0CF5D8E5DD6E77D
:10A7C00091DA01082DE9F04F92F8F030A1B01A911A
:10A7D0001892002B00F05D8101461CA8FFF765FF71
:10A7E0004FF00108AC4CAD4DAD4E189B9DF875E097
:10A7F00003EB081319939DF870309DF87AA000932D
:10A80000009A9DF87F90A05C9DF8742014F80A10BF
:10A810000192019F9DF87920E75D02920697029FC1
:10A820009DF87E20E75D03920797A25C9DF8787003
:10A83000049208979DF873209DF87D70059214F896
:10A84000093014F80EC0A25C09979DF872700A973F
:10A85000E75D0B979DF877700C97E75D0D97089F64
:10A86000E75D0E97099FE75D0F979DF87C70109745
:10A870009DF8717011979DF876701297E75D1397A8
:10A880009DF87B701497E75D1597109FE75D16970D
:10A89000119FE75D1797189F97F8F07047453ED8CE
:10A8A0008DF870009DF818008DF872108DF8740006
:10A8B0009DF82C109DF838008DF87A108DF87800EE
:10A8C0009DF810109DF858008DF876108DF87C00DA
:10A8D0009DF84C109DF81C008DF87E108DF87500C9
:10A8E0009DF854109DF83C008DF87F108DF879008C
:10A8F0009DF834109DF85C008DF87B108DF87D007C
:10A900008DF877201A98199A1CA98DF871C08DF8C6
:10A910007330FFF7CAFE002021B0BDE8F08F81EA56
:10A9200003071B97009F434015F807B01B9F80EA61
:10A930000C008BEA070716F80EB081EA0C0187EAD3
:10A940000B078DF8707015F80E707B4016F80A70C2
:10A950007B408DF8713015F80A30584016F80930F0
:10A960005840009B8DF8720016F803C0049B8CEAD7
:10A97000010115F809C0534081EA0C018DF87310EC
:10A9800001991CA8695C4B400299715C4B408DF8A1
:10A990007430069B5A40029BEB5C5A40039BF35C6D
:10A9A0005A408DF87520DDE906325340039AAA5CBF
:10A9B0005340059AB25C53408DF87630079A049B59
:10A9C0005340019AB25C5340059AAA5C53408DF8FB
:10A9D00077300D9A0B9B5340089AAA5C5340099A12
:10A9E000B25C53408DF87830DDE90D325340099A5E
:10A9F000AA5C53400A9AB25C53408DF87930DDE985
:10AA00000E3253400A9AAA5C53400C9AB25C5340EF
:10AA10008DF87A300B9B0F9A5340089AB25C5340E2
:10AA20000C9AAA5C53408DF87B30159A139B5340C7
:10AA3000109AAA5C5340119AB25C53408DF87C3056
:10AA4000DDE915325340119AAA5C5340129AB25C68
:10AA500053408DF87D30DDE916325340129AAA5CDE
:10AA60005340149AB25C53408DF87E30179A139B72
:10AA70005340109AB25C5340149AAA5C19995340FF
:10AA80008DF87F30FFF700FE08F101035FFA83F8CD
:10AA9000ABE6FF2040E700BF91DA010891D801083A
:10AAA00091D901080B0A017043700B0C090E8370D9
:10AAB000C170704770B51025CEB00C462A460646C8
:10AAC000002168460CF07FFB49238DF80030A37B02
:10AAD000D4F80A100DF106008DF80530FFF7E2FFFB
:10AAE00021690DF10A00FFF7DDFF238908A88DF821
:10AAF0000F3000F0FFF9216808A800F00BFA2A4691
:10AB0000694608A800F00CFA2289616808A800F0DC
:10AB100007FA08A90DEB050000F06DFA049B3360FD
:10AB20004EB070BD492370B500250C460646CEB028
:10AB30008DF800300B8BCDE901558DF801301B0AE3
:10AB40008DF802308B7E03958DF80330CB7E0DF1AE
:10AB500006008DF804300B691968FFF7A3FF6169DF
:10AB60000DF10A00FFF79EFFA38908A88DF80F30AA
:10AB70008DF80E5000F0BEF9216808A800F0CAF95F
:10AB8000694608A8102200F0CBF9A289A16808A89C
:10AB900000F0C6F908A904A800F02DFABDF810309D
:10ABA00008A833808DF804508DF803508DF80250BA
:10ABB0008DF8015000F09EF9616808A800F0AAF92C
:10ABC000694608A8102200F0ABF9A289A16808A87C
:10ABD00000F0A6F908A904A800F00DFABDF810309D
:10ABE00073804EB070BD30B50C46CBB0054604A89E
:10ABF00000F080F9216804A800F08CF922896168CE
:10AC000004A800F08DF904A9684600F0F4F9009B4F
:10AC10002B604BB030BD70B50C89BEB006460D46FA
:10AC2000A4B114F00F0411D101AA10212868FFF774
:10AC30004FFD2889A04201DC3EB070BD6868311923
:10AC4000204401AAFFF7BEFD1034F2E74FF0FF30B9
:10AC5000F2E72DE9F0430F89C7B081460D46002F7A
:10AC60004ED0012410224FEA1718002117F00F07C9
:10AC700001A818BF08F101080CF0A5FAAB7BD5F8C4
:10AC80000A100DF10A008DF809308DF80440FFF725
:10AC900009FF29690DF10E00FFF704FF6E68013E00
:10ACA000444503DD288947B0BDE8F08309AA102197
:10ACB00028688DF81340FFF70BFD09AA05A901A824
:10ACC000FFF780FD444510DB002F14BF3B461023E7
:10ACD00030464A464B440DF1130C934207D80134D9
:10ACE000A4B209F110091036DAE71023F0E710F8E2
:10ACF00001EF1CF8011F81EA0E0102F8011BECE7CD
:10AD00004FF0FF30CFE770B5C2B0144606460D468F
:10AD1000F122002105A80CF056FA0023CDE90333F7
:10AD2000636810218DF805301A0A1B0C8DF8073066
:10AD3000A3688DF806208DF808301A0A1B0C8DF8D0
:10AD40000A30A3898DF809208DF80B301B0A8DF885
:10AD50000C30012305AA20688DF80430FFF7B8FCF9
:10AD600005AA314601A8FFF72DFD022305AA1021EF
:10AD700020688DF80430FFF7ABFC05AA294601A82E
:10AD8000FFF720FD42B070BD2DE9F0431025C3B0A0
:10AD90004A9C80460F4616460021F12205A8994696
:10ADA0000CF011FA2A46002101A80CF00CFAA26856
:10ADB00029468DF80520130AEA408DF80720E2683D
:10ADC0008DF80630D37920688DF8083093798DF8A6
:10ADD000093053798DF80A3013798DF80B30D37818
:10ADE0008DF80C3093788DF80D3053788DF80E3047
:10ADF000137805AA8DF80F30238A8DF810301B0ABE
:10AE00008DF8113001238DF80430FFF761FC05AA9D
:10AE1000414601A8FFF7D6FC022305AA294660682F
:10AE20008DF80430FFF754FC05AA494601A8FFF746
:10AE3000C9FC032305AA294620688DF80430FFF7D2
:10AE400047FC05AA394601A8FFF7BCFC042305AA64
:10AE5000294620688DF80430FFF73AFC05AA3146F0
:10AE600001A8FFF7AFFC43B0BDE8F083F0B50F29B0
:10AE7000C7B004460D4616461F4604D94FF4A171CB
:10AE80001B48F9F7C5F90123002F019318BF0223CE
:10AE90008DF808309DF830310DF10A0083F0010380
:10AEA0008DF809304D9B1968FFF7FCFD4E990DF1A7
:10AEB0000E00FFF7F7FD4FF4807309AA102130460A
:10AEC00005AEADF81230FFF703FC09AA314601A820
:10AED000FFF778FC0023601EDAB2954201D847B034
:10AEE000F0BD10F8012FF15C01334A400270F3E726
:10AEF0000EB9010810B5102204460021F1300CF003
:10AF000062F900212046C4F81411F022BDE8104077
:10AF10000CF059B90B46024610211846FFF7D8BB72
:10AF20002DE9FF470446D0F814010E46154604F2F9
:10AF3000011920B3C0F110089045474628BF1746B5
:10AF400048443A460CF01BF9D4F814313B440F2B1B
:10AF5000C4F814311ED9A8451CD204F1F1031946D6
:10AF600013F8012BD87B4B4582EA000203F8012C31
:10AF7000F6D122460846FFF725FC3E44ED1B0DF1B5
:10AF8000100A102D09D82A46314648460CF0F7F829
:10AF9000C4F8145104B0BDE8F08704F1F002731E48
:10AFA00006F10F0013F8017F12F8011F834281EAB6
:10AFB00007011170F6D16A4604F1F103984617466D
:10AFC0009446186859680833ACE803004B4562465C
:10AFD000F6D1224639463846FFF7F4FB43463A4657
:10AFE00003CA524518605960174603F10803F6D1A9
:10AFF0001036103DC5E7F0B50C4689B0102200218F
:10B00000054668460CF0DFF8224669466846FFF7B9
:10B01000D9FB9DF900306A46002B0DF10F0140DA93
:10B02000137812F8010F5B005BB243EAD013914230
:10B0300002F8013CF4D19DF80F305B0083F08703E8
:10B040008DF80F30D4F81431102B39D1002304F2CD
:10B05000011211781DF8030001334140102B02F852
:10B06000011BF6D104F1F102134604F2011712F8A4
:10B07000011BD07B974281EA000102F8011CF6D146
:10B0800004AA9446164618685968083303C6BB429A
:10B090003246F7D1224629466046FFF793FB09B0B6
:10B0A000F0BD137812F8010F5B005BB243EAD013D6
:10B0B0008A4202F8013CF4D19DF80F305B00BFE7F3
:10B0C0009DF900206846002A28DA027810F8016FFE
:10B0D000520052B242EAD612814200F8012CF4D159
:10B0E0009DF80F20520082F0870280218DF80F20FA
:10B0F000E21882F80111002201330F2B1DD9C4F888
:10B100001431002304F2011211781DF803000133F9
:10B110004140102B02F8011BF6D1A3E7027810F88A
:10B12000016F520052B242EAD612814200F8012C5D
:10B13000F4D19DF80F205200D7E7E11881F80121E2
:10B14000DAE7000008B5064802F064FC0020054B71
:10B150001870054B1B689847BDE8084003F012BA09
:10B16000ABDB01088C0C0020900C002010B50D4CBE
:10B170000D4802F04FFC2368002098470B4B1978CC
:10B180000B4B187803F064FA6420F7F7F5F923689D
:10B19000084898476420F7F7EFF90122064B1A7028
:10B1A00010BD00BF900C002091DB01085002002070
:10B1B00051020020BDB100088C0C00200C4B07B5DB
:10B1C0001B788BB101220B4B0B481A7004F068FA04
:10B1D0000A4B02A91B7801F8043D094B18680023AB
:10B1E00000681A46F8F7FEFB03B05DF804FB00BFE9
:10B1F0008C0C0020940C0020950C00209F0C00204B
:10B20000A80B002030B50B4B85B01A7805460A4CC8
:10B2100062B1002209491A7001A8094B094AFBF7DB
:10B22000FAF901A92846FBF77BFA2070207805B0CF
:10B2300030BD00BF520200209F0C00202FBC01082F
:10B2400045B100086DB10008044B1B7813B10448E8
:10B2500002F01CBB00204FF000417047940C00200E
:10B26000950C0020FF22014B1A7070479F0C0020A4
:10B2700009F01CB870B50446074D44F8041B064697
:10B280000FCD0FC42B6830462360002333767376CE
:10B2900001237375B37570BDC8DB0108F0B50646B0
:10B2A00091B014480F46154602F0B4FB0020124A34
:10B2B000CDE907000D92114A09900E92104AADF89F
:10B2C0002450ADF8227007AC02AD0C90CDE90A0015
:10B2D0000F9294E8070085E8070010AA12E903001E
:10B2E0008DE803000AAB0FCB08F092FB01237376C5
:10B2F00011B0F0BDDCDB010815DA00084DDB0008F9
:10B3000021DB000808B5437E1BB92C210E48F8F755
:10B310007FFF0E4802F07EFB08210D4803F094FFEA
:10B32000002308211A460A4803F0DEFE00F0D8FB8D
:10B33000036814211B699847BDE8084001220821D1
:10B34000034803F00FBF00BF0EB90108E9DB010895
:10B3500000000240437E70B504460D461BB93F21F4
:10B360002648F8F755FF267E35B326BB244802F061
:10B3700051FB00F0B5FB234900F076FC0C2122487C
:10B3800003F05CFF324633460C211F4803F0ACFE4D
:10B3900020681E4903685B699847214651F8040BF1
:10B3A00003681B6898471420F7F7E6F82046FFF774
:10B3B000A9FF0123237670BD002EFCD0144802F0B3
:10B3C00029FB02220C21104803F0CCFE3220F7F7B3
:10B3D000D3F820680F2203680E49DB689847642081
:10B3E000F7F7CAF8206803685B6898472068294621
:10B3F00003685B6998472576DDE700BF0EB9010851
:10B40000F5DB0108666636400004024071B20008B0
:10B4100004DC010815DC010810B50446024B03608A
:10B4200002F0C6FC204610BD30DC010810B5044611
:10B43000054B5C3040F85C3C044B40F8043CFFF7A3
:10B44000EBFF204610BD00BF78DF0108DCE00108FB
:10B4500010B50446FFF7E0FF2046082101F0ECFBA1
:10B46000204610BD10B50446FFF7E0FF20468821B6
:10B4700001F0E2FB204610BD07B58DF804108DF8F1
:10B4800005200221024601A803F07EFF03B05DF80B
:10B4900004FB38B505460024A54203DD03F034FC67
:10B4A0000134F9E738BD000081F0010201480E21A6
:10B4B00003F0D0BE0004024004F05EBE37B50023A6
:10B4C000054602A8144600F8011D137001212A4602
:10B4D00003F068FF20B12A460121204603F07EFFD9
:10B4E00003B030BD10B50C46F7F7B4FA022808D106
:10B4F0004FF47A704443B4FBF0F0BDE81040F7F726
:10B500003BB82046BDE8104003F00ABC08B503482C
:10B5100002F080FABDE8084004F02EBE8CDF01087E
:10B5200010B5094C094802F075FA20460F2103F0C6
:10B5300085FE002320461A460F2103F0D5FDBDE805
:10B54000104003F0D3BB00BF0004024032DF01080B
:10B5500008B503F0ADFA03490BF014F80BF014FA38
:10B5600080B208BD00007A447FB5F82300F144059D
:10B5700004AC0646284604F8013D00F019FE0223FB
:10B58000214600930122A023284600F015FE4FF427
:10B5900000430822009306F14D01A02304462846EB
:10B5A00000F034FE0440E4B2284600F003FE2046DA
:10B5B00004B070BD70B50446394D8AB0394802F008
:10B5C00029FA284602F026FA374802F023FA3748CB
:10B5D00002F020FA364802F01DFA364802F01AFA54
:10B5E000354802F017FA354802F014FA344A354962
:10B5F000354802F00FFA3549354802F00BFA354864
:10B6000002F008FA344B354E1B68354A0093354B2F
:10B6100012681B68344930460CF00EFD3146334841
:10B6200002F0F8F994F8540094F84F3094F84E2052
:10B6300094F84D10049094F85300039094F852003D
:10B64000029094F85100019094F85000009028481E
:10B6500002F0E0F907A804F023F807A802F030F997
:10B660000146244802F0D6F940F2E731002002F00A
:10B670001FFB40F2E7310446002002F019FB40F2C4
:10B68000E7310646002002F013FB3246034621460E
:10B69000194802F0BFF9284602F0BCF90AB070BDA3
:10B6A00063DC010881C4010893DC0108A2DC010805
:10B6B000C4DC0108E7DC01080BDD010882C40108D5
:10B6C00018C2010800C201082EDD01083DDD010895
:10B6D00046DD010851DD01086400F81F300D00202F
:10B6E0005000F81F5400F81F71DD010883DD0108C8
:10B6F00064DE01088EDD0108A0DD0108002003F0F2
:10B700008DBE000007B501A807F0F8FF01980AF008
:10B71000C9FA0022044B0AF01DFB0AF0B5FD00B285
:10B7200003B05DF804FB00BF000024402DE9F14F99
:10B7300088460446914603F0BBF9414605460BF0A6
:10B74000BFF800283CD023680121DB6820469847D9
:10B750001D4EDFF87CA0494628460BF0B1F807469D
:10B7600018B3314648460AF00DFF0BF0E7F83146B2
:10B77000834640460AF006FF0BF0E0F831460746E4
:10B7800028460AF0FFFE0BF0D9F83A4601465B4620
:10B79000504602F03FF923684FF47A711B69204646
:10B7A000984703F085F90546D5E7084802F032F9D5
:10B7B000394620462368DB6801B0BDE8F04F1847E2
:10B7C00001B0BDE8F08F00BF00007A44EADD010857
:10B7D000B1DD010870B504463C4B90B019683C4897
:10B7E00002F018F904F1440500F062FC39483A49C6
:10B7F00002F010F9284600F0D5FC30B9374802F0C5
:10B8000009F9B0213648F8F703FD03F06FFA204636
:10B81000FFF7AAFE18B9B5213148F8F7F9FC94F8FA
:10B82000540094F84F30049094F8530094F84E204C
:10B83000039094F8520094F84D10029094F851003F
:10B840000BAE019094F850000090264802F0E2F808
:10B8500000F042FC284600F0DBFB6D46224B84F8EA
:10B8600084000993214B0893214B0793214B0D939F
:10B87000214B0A93214B0C93214B0B93214B0E939D
:10B880000FCE0FC5204B2B6007AB0FCB07F0BAFFD5
:10B890001E4802F0BFF84FF4FA700BF031FC054679
:10B8A00068B91B4802F0B6F82046FFF783FE204631
:10B8B000184A194910B0BDE87040FFF737BF174864
:10B8C00002F0A8F828460BF023FCEDE75402002014
:10B8D00018DE01082EDE0108A086010049DE0108FD
:10B8E0000EB901085FDE010831F300086DF30008AE
:10B8F00089F3000809F30008D1F20008BDB400087C
:10B9000079B4000893B4000815DA000894DE010841
:10B91000C2DE0108CDCC0C4066660640F6DE0108AA
:10B920002DE9FF4100F14405284600F041FC0424C4
:10B930000226284F013C14F0FF0432D0A12301223B
:10B9400039460096284600F037FC4FF40043804605
:10B9500000930422A12302A9284600F057FCB8F165
:10B96000000FE7D00028E5D09DF80830442B1FD108
:10B970009DF809306E2B1BD10DF10A0002F035F94C
:10B98000013084B221460DF109008DF8086002F003
:10B9900056F9002303220093A02302A9284600F0B1
:10B9A0000BFC284600F006FC204604B0BDE8F08100
:10B9B0004FF488430024ADF808306E2300210DF1C8
:10B9C0000B008DF80A3002F03AF90094A02305220A
:10B9D000E3E700BF38DC0108F7B50446002526463A
:10B9E0000FF0C6FD244B25642360244B84F8485097
:10B9F000E363234B84F84C506364224BC4F84D50EE
:10BA0000C4F85150012146F8583F04F15C0002F09F
:10BA100007FA314684F8645084F865501A4E04F1F0
:10BA20006800FFF727FC84F88450184801F0F2FF03
:10BA30003368174F01933B68164D00932B68164AE5
:10BA40001B2104F121000CF0C3FA296804F1110054
:10BA500002F0E5F8396804F1150002F0E0F8316809
:10BA600004F1190002F0DBF8296804F11D0002F06E
:10BA7000D6F8204603B0F0BD78DF010850E0010899
:10BA80000CE00108DCE001086400F81F5ADF01083F
:10BA90005400F81F5000F81F71DD010810B504F0C4
:10BAA000A9FB0A4C0A4B186000F07EFA2368DB07FA
:10BAB00009D40848FFF790FF0123074A07490548C2
:10BAC000236008F0B7FC034810BD00BFA00C0020A5
:10BAD00054020020A80C0020000000202DB4000813
:10BAE00038B5064D064C2B6813F0010F04D1FFF753
:10BAF000D5FF012320602B60206838BDA40C0020F6
:10BB00004C0D002008B5FFF7EBFF012380F84C3007
:10BB100008BD000008B519B1BDE80840FFF700BD39
:10BB2000044801F077FFBDE8084002220F210248D7
:10BB300003F018BB48DF01080004024070B504465A
:10BB4000364801F067FF20460FF01CFD204600211B
:10BB5000FFF7E0FFFBF722FF07F06EFD002104F185
:10BB60006800FFF7F7FB04F1580000F06FFC236852
:10BB70002B4EDB680021204698472A4D03F0EAFB54
:10BB8000304601220D2103F0EDFA304601220E214C
:10BB900003F0E8FA012228460E2103F0E3FA3046CA
:10BBA0000F2103F051FB0321284603F04DFB1E48F3
:10BBB00001F030FF04F06AF803F08AF8002108462B
:10BBC00003F0B2FE002328461A460E2103F08CFA39
:10BBD00028460E2103F032FB30460F2103F02EFBE6
:10BBE0000321284603F02AFB04F1440000F0DAFAAE
:10BBF0004FF4E13004F05CF90C4801F00BFF07F062
:10BC000041FC03F0E3FE2046094A0A49FFF78EFD96
:10BC10002046BDE870400FF0C5BC00BF00DF010842
:10BC2000000002400004024024DF010838BF010880
:10BC3000CDCC0C406666064008B5FFF751FFBDE865
:10BC40000840FFF77BBF000008B50F21054803F04F
:10BC50000FFB28B1BDE808400F21024803F01CBBD0
:10BC600008BD00BF000402402DE9F0410C46064625
:10BC7000234920460AF042FE20B9002120460AF05E
:10BC80001FFE20B14FF413711E48F8F7C1FA304679
:10BC9000FFF7DAFF054650BB02F00AFF1A490746D4
:10BCA00020460AF06FFC0AF049FE174980463846E4
:10BCB0000AF068FC0AF042FE42460146134801F0D1
:10BCC000A9FE394620460AF019FE80B1FFF728FC8C
:10BCD000204609F0E7FF08A3D3E9002309F084FE1A
:10BCE0000AF0F2FA214602463046FFF71FFD2846C9
:10BCF000BDE8F081AFF300807B14AE47E17A843F6A
:10BD0000333353400EB9010800007A44FDDD0108C9
:10BD100030B508468DB014460F4B104A1049F9F75C
:10BD200091FF00210F4A0A9107920F4A069108924B
:10BD30000E490F4A0F4D09920494059104AA01ACD3
:10BD400007CA0B9584E8070007AB00950FCBFAF7FD
:10BD5000AFFA0DB030BD00BFB9B4000839DC01083E
:10BD60005DDC0108DDED000865ED00080000080855
:10BD70000DB5000805BB000838B50546FAF7B2FD59
:10BD8000074B04461A784AB1002205F13C011A70AB
:10BD9000FAF782FC03492046FAF780FC204638BDBA
:10BDA0005802002039BC0008032004F0F5B9000057
:10BDB000024B186803685B68184700BF540D0020E9
:10BDC000024B186803689B68184700BF540D002099
:10BDD0002DE9FF41002315461370022206460D4F40
:10BDE00004AC386804F8011D03680092D3F80C8095
:10BDF000012233462146C04748B14FF4004238681B
:10BE00002946036800921C6901223346A04704B00A
:10BE1000BDE8F081540D002030B585B08DF80D20BF
:10BE20000022074B8DF80C101C6803A923680092B0
:10BE3000DD68022203462046A84705B030BD00BF9A
:10BE4000540D00204FF47A735843B0FBF3F0F6F72B
:10BE500093BB10B50446FFF743FE2146BDE81040F2
:10BE6000FFF75EBD10B53B4C07F038FC20460222C0
:10BE7000002103F077F901222046114603F072F900
:10BE8000002320461A46032103F02EF92046012202
:10BE9000082103F067F9204602220B2103F062F922
:10BEA000204602220C2103F05DF9204602220D21DA
:10BEB00003F058F9204602220E2103F053F9002323
:10BEC00020461A460F2103F00FF920460F2103F0F8
:10BED000B5F9022204F580641146204603F042F9C8
:10BEE000002320461A46032103F0FEF820460321D2
:10BEF00003F0A4F920460022062103F033F920467E
:10BF00000222082103F02EF920460222092103F023
:10BF100029F9204602220C2103F024F920460222AE
:10BF20000D2103F01FF9002320461A460E2103F0CD
:10BF3000DBF820460E2103F081F9002320460F2173
:10BF40001A4603F0D1F82046BDE810400F2103F057
:10BF50007BB900BF0000024008B50D49012003F085
:10BF60005DFA0C490B2003F059FA0B490A2003F043
:10BF700055FA0A49042003F051FA0949072003F051
:10BF80004DFABDE808400749052003F047BA00BF55
:10BF9000592E0108CD3101081D3001081533010863
:10BFA0004D320108E132010808B5022002F016FE08
:10BFB00002F078FEFFF756FF02F08AFEFFF7CCFF93
:10BFC00003F0D6FB0C48F8F7EDF84FF4E13003F03E
:10BFD0006FFF0A4B1A680AB9094A1A60094B1A68B6
:10BFE0000AB9074A1A60084801F014FDBDE8084084
:10BFF000064801F00FBD00BFA9BD0008A80D002034
:10C0000051FD0008AC0D0020AEDF0108C6DF0108BD
:10C010001C4B10B51A6888B0D2075FBF1A4A10606F
:10C0200001221A60194B1A4A04931A4B05931A4BB2
:10C0300003931A4B02931A4B079308AB43F8082D4E
:10C0400093E803008DE8030002AB0FCB02F072FB14
:10C05000044690B1134801F0DDFC0022124811465D
:10C0600003F080F810480F230222002102F01AFF8B
:10C0700002F088FA012008B010BD0C4801F0CAFC9B
:10C080002046F8E7500D0020540D0020B1BD0008F7
:10C0900045BE0008C1BD0008D1BD000819BE00089A
:10C0A00015DA0008DCDF010800000240EDDF0108BE
:10C0B000002307B5ADF804308DF8063001238DF864
:10C0C0000530019807F066FA02F002FE03B05DF851
:10C0D00004EB07F0B1BA00002DE9F0439BB002F089
:10C0E000C9F9DFF8B890254C254FDFF8B48012ADC0
:10C0F00050B9CDE91544CDE91387CDF848900094A7
:10C1000095E80F0002F0D0F91E4B002613931E4B4A
:10C1100006A912931D4B284614931D4BCDE9188791
:10C1200015931C4BCDE916340423CDE9063605F0F2
:10C1300015FD05F007FD01F0C9FD174ACDE90966B7
:10C140001192032208920122CDE90C440B968DF83E
:10C15000262008AB02AC0FCBCDE90F87CDF8389085
:10C1600084E80F0010AB93E803008DE803000CABEC
:10C170000FCBFBF71BFB1BB0BDE8F08315DA000803
:10C1800021DB0008BD35010885340108953301081D
:10C190002D3301084133010853BE00085DF7000844
:10C1A0004DDB0008014803F0C3B800BFA0860100C2
:10C1B00003F08EB803F0A8B82DE9F041069F1E46A3
:10C1C00007F00303032B80460C46154603D11921C3
:10C1D0000D48F8F71DF82046BC07324629460AD517
:10C1E00003F0E0F810B10120BDE8F0810123002048
:10C1F00088F80430F8E7FB0702D503F0E1F8F1E72F
:10C2000003F0C2F8EEE700BF0EB901082DE9F041D6
:10C21000069C0D46E107804616461F4603D536218B
:10C220000D48F7F7F5FFA20703D539210A48F7F7BC
:10C23000EFFF23043A46314628460AD503F0CEF8EC
:10C2400010B10120BDE8F0810123002088F80430FE
:10C25000F8E703F08BF8F3E70EB9010803F07EBAB4
:10C260001FB501A801F0EDFA01A803F057FB05B0D6
:10C270005DF804FB03F0C0BA03F0D8BA084603F037
:10C280004FB9DFB50023CDE90133ADF80C30012300
:10C290008DF807308DF808306FF01D038DF80930E8
:10C2A0000723044601A88DF80A3001F0EFFA23684D
:10C2B00006461B6820460F469847864277EB0103E7
:10C2C000B4BF0120002004B0D0BD70B506461946A9
:10C2D00010461D46144602F021F9736823B120462A
:10C2E0002946BDE87040184770BD00002DE9FF47A2
:10C2F00014461D46824603F031FA80468946261AC6
:10C3000022462B4601A865EB010701F09AFA404648
:10C31000494601F0FFFA29468046204601F0FAFA24
:10C3200039460446304601F00BFB2246034641469F
:10C33000074801F06FFB01A803F0A2F920B13246D3
:10C340003B465046FFF7C1FF04B0BDE8F08700BF91
:10C3500020E00108704770472DE9F043041D85B0C7
:10C36000804620460D4601F04DFD08BB304801F0E7
:10C3700051FBAA7C697C2F4801F04CFB6F684E2F63
:10C3800005D04F2F03D0452F0CBF45270027AE689F
:10C39000082E18D0092E16D0072E14D01F2126489B
:10C3A000F7F736FF254B264A202126480AF0C6FC1F
:10C3B0006421204601F012FD0028DAD135211E4803
:10C3C000F7F726FFD5E7EC680A2C2ED027DC052CE2
:10C3D00008BF052418BF00246B7C73B14FF001091E
:10C3E0000023CDE901932B7C324600933946234646
:10C3F000286803F097FD88F80C90AB7C63B14FF090
:10C400000109114B3246CDE90039394623462868E7
:10C4100003F0F0FA88F80D9005B0BDE8F0830F2C1A
:10C42000DAD0142C08BF0224D4E70124D4E700BFDB
:10C430006CE0010885E001080EB90108DDC00108C3
:10C44000FCE00108A2E001080000024070B5051DF3
:10C450000446284601F0D6FC064678B9237B13B182
:10C4600003F032FD2673637B1BB103F0B1FA0023A6
:10C4700063732846BDE8704001F0C7BC70BD084634
:10C4800003F052BB38B50C468D18AC4204D014F8FA
:10C49000010B03F049FBF8E738BD03F03BBD08464C
:10C4A00003F028BEF0B508B90020F0BD00274668AB
:10C4B0004D1CB5421760F7D803685C185B5C03F04D
:10C4C0001F03A3F1180103298FBF38460D49C9186E
:10C4D00011F8180C0544AE42E6D304280DD8DFE865
:10C4E00000F00403070C0C00637813600130DCE7F4
:10C4F000B4F801305BBA9BB2F7E7D4F801301BBA4D
:10C50000F3E700BF34E10108F7B51F46436816465C
:10C510004A1C9A4205460C4617D803685B5C03F038
:10C52000C003402B11D196B101AAFFF7BBFF50B158
:10C53000019A04446B68A118994206D829681044EE
:10C540000C4434603A6003B0F0BD0020FBE7304695
:10C55000F9E72DE9F7439946436817464A1C9A4282
:10C5600080460D4624D803685B5C03F0C003402B73
:10C570001ED1FFB101AAFFF795FF0446A0B1019EAD
:10C5800009F10109B14513D30544D8F804307219F3
:10C590009A420DD8D8F800103246294438460AF09D
:10C5A000EEFD00233444BB55204603B0BDE8F083C4
:10C5B0000024F9E73C46F7E7F0B5002931D0172A07
:10C5C0001CD8D3B2A3F11804032C8CBF0024164C42
:10C5D0008D689CBFE41814F8184C6F1C4E6804EB6F
:10C5E000070CB4451DD20E6818438F6070550020AB
:10C5F0000130231A5D1C0BD1601CF0BDFF2A05D948
:10C60000B2F5803F2CBF1A231923DBE71823D9E7A3
:10C610008E680D68DB00771C22FA03F38F60AB5540
:10C62000E6E70020E9E700BF34E10108172BF8B581
:10C630000D4616461C4612D8DBB2A3F11802032A97
:10C640008FBF0022144A9B1813F8182CAB680132D4
:10C65000234413446A6893420BD30020F8BDFF2B98
:10C6600005D9B3F5803F34BF19231A23E5E7182312
:10C67000E3E722462946FFF79FFF07460028ECD054
:10C680002868AB68314618440AF079FDAA68E019B9
:10C690002244AA60E2E700BF34E1010818B1002398
:10C6A000C0E9001283607047436873B514464A1CA2
:10C6B0009A4206460D4602D9002002B070BD0368BA
:10C6C0005B5C13F0C00FF7D1002CF5D001AAFFF787
:10C6D000E9FE0028F0D03268019B525D12F0E00FB5
:10C6E00018BFDB432360E8E70A1EABBF01460146E3
:10C6F0000020D243B8BF2020FFF75EBF03685B5C19
:10C7000003F0E001E02907D132B1A3F1F5014B427A
:10C710004B4113700120704700207047836810B5AB
:10C7200044685A1CA24208D2002914BFF524F424FC
:10C73000016882600120CC5410BD0020FCE7F0B4F9
:10C7400046684F1CB74208D805686C5C04F0E004EA
:10C75000402C02D1F0BCFFF7D7BE0020F0BC7047E0
:10C7600013460A4601464020FFF760BFF0B4466812
:10C770004F1CB74208D805686C5C04F0E004602CDC
:10C7800002D1F0BCFFF7E5BE0020F0BC7047F0B46A
:10C7900046684F1CB74208D805686C5C04F0E0049A
:10C7A000602C02D1F0BCFFF7AFBE0020F0BC704798
:10C7B00070B5054608460C460BF0B5FC224603460C
:10C7C0002946BDE870406020FFF730BF83684168AC
:10C7D0005A1C8A423FBF8260BF220168012034BFD9
:10C7E000CA54002070470368585CA0F1BF03584248
:10C7F0005841704713B5036814465B5C03F0E003CF
:10C80000A02B07D142B101AAFFF74CFE019B236088
:10C8100002B010BD0020FBE71046F9E783684168CD
:10C820005A1C8A423FBF8260FF220168012034BF48
:10C83000CA540020704730B18068013888428CBFEC
:10C840000020012070470120704708B50246FFF71D
:10C85000F2FF30B91268505CA0F1FF035842584112
:10C8600008BD0120FCE743688B4207D903685B5C85
:10C8700013F0C00F0CBF012000207047002070474C
:10C8800043688B4208D90368585C00F0E000A0F1CF
:10C8900040035842584170470020704743688B421C
:10C8A00008D90368585C00F0E000A0F1600358422A
:10C8B000584170470020704743688B4208D903688D
:10C8C000585C00F0E000A0F1A003584258417047C6
:10C8D0000020704710B50446FFF7EEFF50B16368C3
:10C8E0008B4208D92368585C00F01F00A0F11F0399
:10C8F0005842584110BD0020FCE743688B4208D9DC
:10C900000368585C0C30C0B201288CBF00200120A5
:10C910007047002070470023C0E9013303690160BC
:10C92000C360704703468068F0B51D68013090FB16
:10C93000F5F405FB14005C68A04224D00026964262
:10C94000304601D11046F0BD8F5DD3E902452F5529
:10C950009C681D68671C97FBF5F405FB14745F6801
:10C960009C60BC4204F1010402BF94FBF5F705FB97
:10C9700017475F6094FBF5F705FB17445D68AC4211
:10C98000E1D00136DBE70020DDE70000F8B5036801
:10C990000446002B0D46164603DC3E212948F7F7D6
:10C9A00037FC3246002128460AF00DFCD4E901701C
:10C9B000B8420CD00021236801EB070C9CFBF3F27A
:10C9C00003FB12C2904205D10020884204D14FF0EF
:10C9D000FF3031E00131EFE7C21992FBF3FE03FBB8
:10C9E0001E2ED4F80CC01CF80EE0BEF10A0F26D1A2
:10C9F00028B3013A92FBF3F103FB1122002106F167
:10CA0000FF3E71450ED2E7686368FB5C6B54676854
:10CA10002668013797FBF6F306FB1377013188424E
:10CA20006760EEDA1CF802300D2B4FF0000304D1E2
:10CA3000054405F8013C0138F8BD2B54FCE70130F2
:10CA4000C3E700BF0EB901084B1C017343738B1C75
:10CA500003318373C17370472DE9F041074688465F
:10CA60001E4615461AB952211548F7F7D1FBD7E9EA
:10CA70000143A34221D2E41ADEB1A3B9A5420ED3E9
:10CA80003B7B3370BB6839682246194440460AF044
:10CA900076FBBB682344BB602046BDE8F0817B7B0E
:10CAA00033702C46EEE7A54201D3FB7BE9E7BB7B65
:10CAB000F6E7AC4228BF2C46E4E70024ECE700BFD1
:10CAC0000EB901080023C0E900128360704710B559
:10CAD00004460846C4E900120021A16021730AF04F
:10CAE00072FB204610BD000038B51546D0E9012381
:10CAF00004465819904202D9257B55B1D51A2068B1
:10CB00002A4618440AF03BFBA3681D44A560012592
:10CB100003E017210248F7F77BFB284638BD00BF2A
:10CB20000EB9010807B502AB03F8011D0122194631
:10CB3000FFF7DAFF03B05DF804FB8068704700235D
:10CB40008360704713B5044689B201A801F077F8F5
:10CB5000022201A92046FFF7C7FF02B010BD13B59E
:10CB6000044601A801F064F8032201A92046FFF75A
:10CB7000BBFF02B010BD13B5044601A801F04FF889
:10CB8000042220460DEB0201FFF7AEFF02B010BDFC
:10CB900013B50446684601F038F805226946204678
:10CBA000FFF7A2FF02B010BD13B5044601A801F0C3
:10CBB00046F8022201A92046FFF796FF02B010BDF9
:10CBC00008B50146044800F025FFBDE808400C21E7
:10CBD0000248F7F71DBB00BF38E101080EB9010894
:10CBE00008B5044800F016FFBDE808401E210248C1
:10CBF000F7F70EBB7DE101080EB9010810B500F092
:10CC0000A5FF044630B9044800F004FF272103487B
:10CC1000F7F7FEFA204610BD6BE101080EB90108D6
:10CC200000F094BF10B9024800F0F4BE00F078BFE5
:10CC300056E1010800F08ABFFFF7F4BF0346002069
:10CC400084B0CDE90112039004AA12E9070083E839
:10CC50000700184604B0704738B51546044660B161
:10CC6000D4E901030344934207D320680AF087FA0A
:10CC70000120A2682A44A26038BD0020FCE7F8B574
:10CC80000E46054680B14F1C384600F05FFF044653
:10CC900040B13A4600210AF096FA3246294620462B
:10CCA0000AF06DFA2046F8BD0446FBE738B50D469C
:10CCB000044628B10BF037FA23462044834201D1C1
:10CCC000002038BD13F8012BAA42F7D10120F8E764
:10CCD00037B504460D460AF061F8002201A902604A
:10CCE00020460CF085F904460AF058F80368222B18
:10CCF00008D0019B1B782BB9002C03DB20462B604E
:10CD000003B030BD012300202B60F9E72DE9F04F7F
:10CD100005464FF0010B002687B0CDE9031206F15E
:10CD20000903122B8CBF0320022000F00FFF00909C
:10CD3000E8B1324636490BF07FF9039B53F8269051
:10CD4000EDB90024009800F0EBFEBBF1000F02D11A
:10CD5000284600F0E5FE84B1049B0136B342254627
:10CD60004FF0000BDBD1204607B0BDE8F08FBBF1E0
:10CD7000000F02D1284600F0D3FE0024F3E7254B34
:10CD80004FF00008B9F1000F08BF994648460BF074
:10CD9000CAF9019000980BF0C6F90290284649465E
:10CDA0000BF0F5F9B8B928460BF0BDF9DDE9012320
:10CDB00001309B1A08FB030000F0C8FE044600285F
:10CDC000BFD003462F4618F1FF3809D2394618461E
:10CDD0000BF0A1F9B6E7019B08F101081844DEE762
:10CDE0004946384605930BF0D2F9059BA0EB070A9C
:10CDF0005246394618460BF0B0F9009950440BF0F2
:10CE00008AF9019A029B9244C3185744DBE700BF9A
:10CE100023C2010883C4010830B580B10346021F54
:10CE200000F1180452F8045F8D4208D0A242F9D1F3
:10CE30001C301A4614680433013401D1116030BD2E
:10CE40008342F6D1FBE770B5044680B1064600EB9D
:10CE50008105AE4204D12046BDE8704000F060BEBE
:10CE600056F8040B0028F4D000F05AFEF1E770BD2C
:10CE70002DE9F74F89460092002838D00027C45D7D
:10CE80008CBB05468346264600EB070AD34538D1BE
:10CE900004B10136002E6FD00137384600F056FE3F
:10CEA0008346002866D03A4600210AF08CF9B0008B
:10CEB00000F04CFE0446002860D04FF000084146C8
:10CEC000AA4532D131B15846FFF7D9FE002855D0D6
:10CED00044F82800584600F023FE009B1E602046C0
:10CEE00003B0BDE8F08F0137B7F5807FC7D10024CC
:10CEF0002646204600243146FFF7A5FF009B1C6014
:10CF0000EDE79BF800304B4505D10CB1002401360C
:10CF10000BF1010BBAE70AF0E5F89BF80030184472
:10CF200043781B0758BF0134F2E72B784B4513D1E8
:10CF300081B15846FFF7A3FE00B308F1010344F89E
:10CF4000280000213A46584601930AF03CF9019B1B
:10CF5000002198460135B3E701910AF0C3F82B7818
:10CF600001991844407810F0080F04BF0BF8013005
:10CF70000131EFE70446BCE73446B0E7584600F01D
:10CF8000CFFDB6E72DE9F743002506460820884681
:10CF900091461F46009500F0D9FD0446002868D050
:10CFA000C0E9005530460BF0BEF801280FD13378A8
:10CFB0002A2B0CD109F1FF33C4F80080636022688A
:10CFC0004A4502D263684B4543D32B4B0EE02D21DB
:10CFD0003046FFF76BFE0546C0B902A941F8040DC3
:10CFE0003046FFF775FE019B63B1244B3B6000990F
:10CFF0002846FFF728FF002C37D0204600F090FD90
:10D00000002432E0C4E900001D46D8E76A462D211D
:10D010003046FFF72DFF009B0546013B012B01D950
:10D02000174BE3E7002302AE46F8043D31460068A3
:10D03000FFF74EFE2060019B0BB1124BD6E7314645
:10D040006868FFF745FE6060019B002BB7D00E4B70
:10D05000CCE7424501D3434501D20C4BC6E70099CA
:10D060002846FFF7F0FE00233B60204603B0BDE8F2
:10D07000F0830546BBE700BF86E2010800E2010835
:10D080001FE2010848E2010867E20108A6E2010880
:10D0900038B590B1451E15F8014F0CB9204638BD82
:10D0A0000AF020F823462044427802F00302022AC4
:10D0B00008BFA4F120032B70EDE70120EFE708B5CE
:10D0C00020B34A1C22D0062920D8DFE801F0040D45
:10D0D000101316191C00002303600AF057F90840CA
:10D0E000431C5842584108BD00234360F5E7002324
:10D0F0008360F2E700238361EFE70123C360ECE77D
:10D1000000230361E9E700234361E6E70120EAE742
:10D1100070B506460D1F01F1180455F8041F4B1C8D
:10D1200003D1A542F9D1002070BD3046FFF7C7FFFB
:10D130000028F6D0F8E708234A4291FBF3F302F007
:10D14000070201F0070158BF51420122DBB2C9B208
:10D1500002FA01F1C25C1143C154704708234A42EC
:10D1600091FBF3F302F0070201F0070158BF5142AF
:10D170000122DBB2C9B28A40C15C21EA0201C1547A
:10D180007047082391FBF3F3DBB2C05C4B4203F022
:10D19000070301F0070158BF5942C9B2084100F026
:10D1A000010070472DE9F047089E8A4690461D46CB
:10D1B000DDF82890074610B11446A24507D875B986
:10D1C000012200240B9B1A602046BDE8F08721460F
:10D1D0003846FFF7D6FF002861D10134EDE7099BFF
:10D1E000023B042B04D8DFE803F0282C2C30340059
:10D1F0006B6801336B6028460AF0C8F8013108BF3C
:10D20000B0F1FF3FDCD031462846FFF758FF002839
:10D21000D6D12FB3044621463846FFF7B2FF002887
:10D2200041D10134A245F6D10446013E042E19D85D
:10D23000DFE806F02B2D2F313300AB680133AB60F4
:10D24000D9E7EB680133EB60D5E72B6901332B613C
:10D25000D1E76B6901336B61CDE7002DE5D1AFE715
:10D260003C46E2E72C6028460AF090F8013108BFFE
:10D27000B0F1FF3FA4D0B9F1000FA1D04946284634
:10D28000FFF746FF00289FD09AE76C60EBE7AC60A1
:10D29000E9E7AC61E7E7EC60E5E72C61E3E7A0458F
:10D2A000DBD1444690E7A045BFD1FAE700232DE942
:10D2B000F04F06468BB01C200C469046099300F0B8
:10D2C00045FC0546002800F0E4801C2000F03EFCF0
:10D2D0000746002800F0DD804FF0FF31021F2B1FB2
:10D2E00005F1180043F8041F984242F8041FF9D1D1
:10D2F00000230121D4F800A00DF12409CDE900316B
:10D30000CDE902793C21234652463046FFF74AFFD9
:10D31000099900296ED1824502D12846FFF77CFD8C
:10D3200002234FF0010AD4F804B0CDE900A3CDE9FF
:10D33000025923465A463C2106F10800FFF732FF06
:10D34000099B002B56D183454CD151462846FFF707
:10D3500063FD03234FF0020AD4F808B0CDE900A31F
:10D36000CDE9025923465A46182106F11000FFF76D
:10D3700019FF099B002B3DD1834546D151462846D4
:10D38000FFF74AFD40F26F1BA3690593E36804931E
:10D3900006F114030693DDF810A006F113030793BA
:10D3A00051460698FFF7EDFE28B105990798FFF75B
:10D3B000E8FE002836D1BBF1010B33D0E3682046EC
:10D3C0000133E36009F0E2FF013108BFB0F1FF3F34
:10D3D00024D0A36929462046D4F80CA00593FFF772
:10D3E00097FEDDE7424621463046FFF75FFF099092
:10D3F0000028AED0284600F093FB17B1384600F065
:10D400008FFB09980BB0BDE8F08F424621463046AD
:10D41000FFF74CFF09900028ECD1B3E701234FF050
:10D42000000A0993099B002BE4D1049B534520D1AA
:10D4300004212846FFF7F0FC05230622D4F810A0AB
:10D44000CDE90032CDE90259234652460C2106F1BE
:10D450001800FFF7A7FE099B002BCBD18245C9D04E
:10D460006369A3EB0803042B0CD94FF0FF33099336
:10D47000C0E7424621463046FFF718FF09900028D2
:10D48000B8D1D9E7424621463046FFF70FFF099051
:10D49000B0E74FF0FF330993002DB2D00027A9E782
:10D4A0002DE9F04F002487B0924606AA894642F83B
:10D4B0000C4D2C219846109DFFF7DAFC074688B9E1
:10D4C0003E4B2B6003993846FFF7BDFC07B0BDE823
:10D4D000F08FD0F800B072685A451CD2304600F088
:10D4E0001FFB0134039BA342ECD957F824602F2182
:10D4F0003046FFF7DBFBA8B92B4630464246514683
:10D50000FFF740FD2B680646002BE2D00028D9D05B
:10D5100000F006FBD6E759464846FFF70CFE0BF134
:10D52000010BD8E700232F21304604AA0493FFF70C
:10D530009FFC049906464B1E012B04D9204B2B60FF
:10D54000FFF781FCBEE742462B4651460068FFF7D5
:10D5500019FD2A6883462AB108B100F0E1FA04995E
:10D560003046EDE72D213068FFF7A0FB18B908F130
:10D57000FF32CBF80420002306A941F8043D70686F
:10D58000FFF7A6FB059A00901AB10E4A58462A608A
:10D59000E3E7DBF80020DBF80410914205D23046C7
:10D5A0000499FFF750FC584699E711464846019206
:10D5B000FFF7C1FDDDE900321A44ECE7CBE20108D8
:10D5C000DDE2010802E301082DE9FF4100230E46D8
:10D5D0000393144602B902AC236048B90546564B82
:10D5E000236003992846FFF72EFC04B0BDE8F081C4
:10D5F00003AA2021FFF73CFC039B0546062B02D023
:10D600004E4B2360EDE71A220021304609F0DBFD86
:10D61000009400223C2331462868FFF741FF22682E
:10D62000002ADED100943C2306F108016868FFF768
:10D6300037FF2268002AD4D10094182306F1100184
:10D64000A868FFF72DFF2368002BCAD16869FFF790
:10D650001FFD07223A496869FFF758FB80460AF028
:10D6600062FD012806F1130706D198F800303F2B20
:10D6700004BF2A2388F80030002208233946404698
:10D680000094FFF70DFF404600F04AFA2268002A96
:10D69000A7D107213846FFF774FD30B1114638464F
:10D6A000FFF749FD0721FFF759FDEF6806F1140860
:10D6B00038460AF038FD012804D13B783F2B04BFDF
:10D6C0002A233B7020230022414638460094FFF76E
:10D6D000E7FE00214046FFF741FD2368002B80D183
:10D6E0002F693846FFF7D4FC00287FF47AAF38461C
:10D6F0000D221449FFF70AFB074600283FF471AFDB
:10D70000183600940D2301223146FFF7C9FE384632
:10D7100000F006FA012421463046FFF732FD30B111
:10D72000611E3046FFF707FD2146FFF717FD013464
:10D730000D2CF0D155E700BFAAE10108C2E10108B4
:10D740005C02002078020020F0B58DB0CDE9002306
:10D75000054628B94FF0FF304FF0FF310DB0F0BD56
:10D760002422002103A809F02EFD03A9684609F030
:10D7700009FC04460028EDD009F008FE4A1C08BF49
:10D78000B0F1FF3F06460F46E4D0626921462846C5
:10D79000FFF78CFD0028DDD1204609F0F7FD4B1C7A
:10D7A00008BFB0F1FF3FD5D08F4208BF864203D0FB
:10D7B000204609F0EBFDD1E72368204601332360C2
:10D7C00009F0E4FD013108BFB0F1FF3FC2D062694A
:10D7D00021462846FFF76AFD0028E9D0BAE770B570
:10D7E0003C258AB0DDE90E64019496FBF5F405FB57
:10D7F00014640294182493FBF4F505FB1433CDE96B
:10D800000330481E0C2190FBF1F301FB13010023B0
:10D81000CDE907339DF84030A2F26C7201A8059162
:10D820000692099309F0B2FD0AB070BD1FB500243D
:10D830000294079C0194069C0094FFF7D0FF04B06B
:10D8400010BDF7B5044602A860E9022309F088FB81
:10D850000269037A551C426990F804C0077B02F202
:10D860006C71067EC2690068A3700033207018BF17
:10D8700001232046013284F801C0E7702571A4F825
:10D880000510E6712272637203B0F0BD30B5457ABF
:10D8900085B0C4788378B0F80520017902950578C1
:10D8A0000195407800902046FFF799FF05B030BD04
:10D8B000904271EB0303B4BF0120002070470000C9
:10D8C000032210B5104986B00B78013393FBF2F2B6
:10D8D00002EB42029B1A0D4A0B7052F82340027869
:10D8E000B0F80530049242781A21039282780292AD
:10D8F000C2780192027920460092054A0AF068FB3C
:10D90000204606B010BD00BFA60D0020ACE3010804
:10D9100071E30108B1F1004F08BF00281FB50246AE
:10D920000B4608D001A8FFF78CFF01A8FFF7C8FF3E
:10D9300005B05DF804FB0148FAE700BFA3E3010866
:10D940002DE9FF4703220D462B4900280B7804469A
:10D9500003F1010393FBF2F202EB4202A3EB020399
:10D96000264A0B7052F8236075F100033EDA4FF03F
:10D97000010A444265EB4505214A00232046294619
:10D9800009F022F81E4A074600232046294609F0DE
:10D990001BF8104619464FF46162002309F014F891
:10D9A0004FF46162804600232046294609F00CF8B6
:10D9B000104619463C22002309F006F83C22814615
:10D9C00000232046294608F0FFFFCDF80080CDE96E
:10D9D00001923B46BAF1000F0BD00A4A1A21304699
:10D9E0000AF0F6FA304604B0BDE8F0874FF0000ABE
:10D9F000C2E7054AF2E700BFA60D0020ACE301082C
:10DA0000805101008FE3010890E301080FB404B0D6
:10DA1000704700000FB437B51B4C256855B9032279
:10DA200029460120F5F704FF2B462A4629462060A7
:10DA3000F5F722FF154D2A68013A03321ED86421FA
:10DA40002068F6F705F980220021114809F0BBFB98
:10DA500007AB069A80210E4801930BF039FD7F2811
:10DA600003DD0C490C480AF056FB2B680848984720
:10DA7000002320681A461946F5F7FEFE03B0BDE8FC
:10DA8000304004B0704700BF300E0020A80D0020C9
:10DA9000B00D002066E101082B0E00200FB410B578
:10DAA0000D4CA2B02268013A033210D825AB249A5B
:10DAB000802102A801930BF00BFD7F2804DD0749AC
:10DAC0000DF183000AF027FB236802A8984722B0D3
:10DAD000BDE8104004B07047AC0D002066E10108BD
:10DAE00070B50446054E4518AC4200D170BD14F81F
:10DAF000011B3046FFF78EFFF6E700BFB8E30108D1
:10DB000038B50C461546FFF785FF20462946FFF736
:10DB1000E7FFBDE838400148FFF77CBF82C4010839
:10DB200010B5044670B1F5F7B9FD2046F5F7A4FD30
:10DB3000F5F760FCBDE81040034A938801339380F9
:10DB4000F5F778BC10BD00BF0C18002070B5214C53
:10DB50008AB0226806460132632A22601E4D0BDD20
:10DB6000F4F772FF0523002201A9F4F7AFFEF4F7E2
:10DB7000ABFB002328602360F4F7A6FB2B6803F5BA
:10DB80007A73984204D9F4F79FFB0023286023603E
:10DB9000124A134C13781BB923606360012313707E
:10DBA000F5F77CFD3046F5F765FD054668B1324670
:10DBB000002109F008FBF5F71DFC238801332380C1
:10DBC000F5F738FC28460AB070BD638801336380DE
:10DBD000F8E700BF380E00203C0E0020340E002075
:10DBE0000C180020006800BA7047008840BA80B264
:10DBF000704700687047837842781B04007843EAD6
:10DC0000022318437047FFF7F4BF0370130E4370ED
:10DC1000130C8370130AC3700271052070470B0E3A
:10DC200003700B0C43700B0A8370C17004207047A3
:10DC30000B0C03700B0A43708170032070470B0AB2
:10DC400003704170022070470B0A017043700B0C87
:10DC5000090E8370C17004207047A0F14103052BA9
:10DC600002D83738C0B27047A0F16103052B01D844
:10DC70005738F7E73038C0B20A2828BFFF2070476E
:10DC80000022013910B50144441E8C4204D014F81E
:10DC9000010F08B1002A01DA104610BDFFF7DDFFC1
:10DCA0000F2802D840EA0212EFE74FF0FF32F3E705
:10DCB00038B505460C460AF0EDF8611B013190FBC2
:10DCC000F1F303FB1100284438BD000010B50446F1
:10DCD0000AF0BCF8014B1C6010BD00BFAC02002074
:10DCE000024B1868013018600AF0B0B8AC0200208E
:10DCF00070B5054608460C460AF015FA0646284651
:10DD00000AF011FA864208D83246294620460AF01F
:10DD100012FAB0FA80F0400970BD0020FCE738B577
:10DD2000451E15F8014F04B938BD09F0DBF923464B
:10DD30002044427802F00302012A08BF20332B70EE
:10DD4000EFE72DE9F04106460AF0EDF930B3002780
:10DD5000341809F0C7F914F8013C354618444378E3
:10DD6000621E19070DD42F463B78A4EB0508013538
:10DD70005BB908F1010239463046BDE8F04109F0CF
:10DD800009BA04F8017C1446E3E709F0ABF915F889
:10DD9000013C184443781B07E5D4EAE7BDE8F0816D
:10DDA00008B50AF0AEF9B0FA80F0400908BD0000ED
:10DDB00010B50446034B03604068F6F723F920468C
:10DDC00010BD00BFC8E3010810B50446FFF7F0FF1F
:10DDD00020460821FEF730FF204610BD38B54368C5
:10DDE00004460D461BB90E210548F6F711FA2946DF
:10DDF0006068F5F72DFF431E5842584138BD00BFFB
:10DE00000EB901084068F6F7B1B808B500234068BC
:10DE10001A461946F5F730FD431E5842584108BDD1
:10DE200038B50D4600210B4B0446416003600322C8
:10DE30000120F5F7FDFC606018B957210648F6F798
:10DE4000E7F92DB1002360681A461946F5F714FD6D
:10DE5000204638BD30DC01080EB90108F8B50F4C7A
:10DE6000D4F880329847234610F5617641F10007D7
:10DE700004F52072D3E90845A04271EB050401DAEC
:10DE8000C3E90801D3E90645A64277EB050401DAA8
:10DE9000C3E9066728339342ECD1F8BD480E002051
:10DEA0002DE9F84F064628B9BDE8F84FDC21344883
:10DEB000F6F7AEB90023334A1C469246D118097AC8
:10DEC0002833B14208BF0134B3F5207FF6D1002CCE
:10DED00054D0062E03D940212948F6F799F92A4B48
:10DEE00053F83650002D47D1E7212548F6F790F931
:10DEF0004FF0000B65430AEB0B04227AB24235D196
:10DF00006268002A32D02269012A03D1D0211C483C
:10DF1000F6F77EF9D4E9062319461343104624D0B8
:10DF2000D4E90889B0EB080061EB090108F0ECFACC
:10DF300007462069013808F0CDFA0146384608F056
:10DF4000D5FB0746284608F0C5FA394608F01AFB03
:10DF5000394608F00DFA08F017FD18EB000249F1F8
:10DF6000000310461946C4E9060125610BF1280B90
:10DF7000BBF5207FBFD101E0012DB9D1BDE8F88FFD
:10DF80000EB90108480E0020D0E301084FF47A735F
:10DF9000B0FBF3F341F65832A3F55223A3F618333E
:10DFA00093422DD81B4B1C4A0344934228D91B4B48
:10DFB0001B4A0344934223D94CF24E32194B03447B
:10DFC00093421DD9184B98421CD903F5371303F51A
:10DFD000D863984218D903F5122303F5F8639842E1
:10DFE00014D903F5122303F5F863984210D903F509
:10DFF000DB2303F5BA63984294BF052006207047DF
:10E0000000207047012070470220704703207047AE
:10E01000042070473F373ACC9E8601007F0F31CCF9
:10E020003E0D0300AF312ACC40DA8E33704700003A
:10E0300070B5134C054694F894320E4623B94FF44C
:10E0400096711048F6F7E4F825B940F22D110D4805
:10E05000F6F7DEF826B94FF497710A48F6F7D8F8C4
:10E060000023282202FB03F0215CA94203D12044B3
:10E070004168B14203D00133102BF3D1002070BDB1
:10E08000480E00200EB901082DE9F04F324F9A4694
:10E0900097F8943293B00191934623B940F241111D
:10E0A0002E48F6F7B5F80026FFF7D8FEB1464FF038
:10E0B000FF383446284DEB68019A934219DBBBF1D7
:10E0C000000F11D1D7F880329847D5E90623904246
:10E0D00071EB030C2EDB12AB03EB890343F8406CAE
:10E0E00009F10109002227E000212846D84700282D
:10E0F000E8D10136102E05F12805DCD1BAF1000F68
:10E1000001D0CAF80080B8F1000F0FD1B9F1010FAA
:10E110000CD909F1FF314046FFF7CAFD12AB03EB02
:10E120008000282350F8404C03FB0474204613B0B1
:10E13000BDE8F08F121ACED042450AD3D9D1D4E926
:10E140000823D5E90801FFF7B3FB002818BF2C46C8
:10E15000CFE790462C46CCE7480E00200EB90108C8
:10E16000F8B50D46044620B94FF4C2711848F6F7C9
:10E170004FF8236923B940F285111548F6F748F89E
:10E18000144BD3F8803298470F4606462069C4E9FD
:10E19000086708F09FF9294608F0F4F9294608F0C5
:10E1A000E7F807F07FFD08A3D3E9002307F0FCFEA2
:10E1B00006F046F908F068F8321847F100031046F7
:10E1C0001946C4E90601F8BD0000000080842E4114
:10E1D0000EB90108480E00202DE9F0410E46174601
:10E1E000054620B94FF4C8711348F6F711F826B95F
:10E1F00040F291111048F6F70BF80021384608F06C
:10E200007DFB20B94FF4C9710B48F6F701F80024E3
:10E21000DFF8288014F80830AB4207D108EB04007F
:10E220004368B34202D13946FFF79AFF2834B4F568
:10E23000207FEFD1BDE8F0810EB90108480E002023
:10E2400008B5FFF7A3FE003018BF012008BD00008D
:10E250002DE9F043344E95B096F8943281460C4641
:10E2600023B94FF4D9713148F5F7D2FF2046FFF7B3
:10E27000E7FF70B121464846FFF7DAFE48B9074686
:10E28000282303FB0768D8F804202AB10137102F90
:10E29000F7D115B0BDE8F08396F894321BB9772119
:10E2A0002248F5F7B5FFB9F1000F03D178211F48D7
:10E2B000F5F7AEFF282200210DEB020008F083FFE6
:10E2C0002046FFF763FE062805468DF8300003D987
:10E2D00040211648F5F79CFF154B0B9403EBC50244
:10E2E00053F835306D4652688DF82890CDE90D23EE
:10E2F0000AAC0FCC0FC50FCC0FC594E80300282340
:10E3000003FB07676E463C4685E803000FCE0FC44B
:10E310000FCE0FC495E8030084E80300387AFFF7B6
:10E32000BFFD4046B5E700BF480E00200EB901080A
:10E33000D0E301080C4B10B593F89432044623B98E
:10E340004FF4EA710948F5F763FF54B1636843B1CC
:10E350000748FFF75FFB0023207A63602372FFF713
:10E360009FFD002010BD00BF480E00200EB901081F
:10E3700008E401082DE9F041124D074695F8943262
:10E38000884623B94FF4F6710F48F5F741FF27B9D6
:10E3900040F2ED110C48F5F73BFF002426462B5DBB
:10E3A000BB4208D128194368434504D1FFF7C2FF97
:10E3B000002818BF06462834B4F5207FEFD1304638
:10E3C000BDE8F081480E00200EB9010870B50F4D70
:10E3D000064695F8943223B94FF4FE710C48F5F7D0
:10E3E00017FF26B940F2FD110948F5F711FF002487
:10E3F0002B5DB34204D1281943680BB1FFF79AFF94
:10E400002834B4F5207FF3D170BD00BF480E002042
:10E410000EB901082DE9F843154D06460F46904602
:10E420000024A946635DB34209D12B195A6832B161
:10E43000002398450DDC09EB0400FFF77BFF28342F
:10E44000B4F5207FEED10024A04508DC0120BDE812
:10E45000F88357F823108A42F1D00133E9E757F8DF
:10E4600024103046FFF7F4FE0028F0D00134EBE72B
:10E47000480E0020014B93F894027047480E00208C
:10E4800010B5074C2378FA2B04D94FF40D710548C9
:10E49000F5F7BEFE20780130C0B2207010BD00BF7D
:10E4A000400E00200EB9010884B070B504AC84E8B9
:10E4B0000F00164C94F8941221BB4FF4267220469C
:10E4C00004F5207504AE08F07EFE0FCE0FC533684C
:10E4D0002B6013B90E4BC4F89032D4F88C3213B9B8
:10E4E0000B4BC4F88C32D4F8883213B1D4F8843290
:10E4F0002BB9084BC4F88832074BC4F88432012387
:10E5000084F89432BDE8704004B07047480E002093
:10E510000DDA000811710108017101082DE93008B8
:10E520000F4B03F52072D3E908BC5BEA0C0405D05D
:10E530001BEB00044CEB0105C3E90845D3E906BC1D
:10E540005BEA0C0405D01BEB00044CEB0105C3E9AE
:10E55000064528339342E6D1BDE83008FFF77EBC7C
:10E56000480E0020024B0A465B68014630201847DF
:10E57000E0100020024B0A461B6801463020184775
:10E58000E01000202F4B10B51B7823B940F2011189
:10E590002D48F5F73DFE2D4CA368984700211F201C
:10E5A000FFF7E8FF20B94FF482712748F5F730FEF6
:10E5B00090211E20FFF7DEFF20B94FF4837122481F
:10E5C000F5F726FE00212020FFF7D4FF20B940F206
:10E5D00007111D48F5F71CFE00212120FFF7CAFF97
:10E5E00020B94FF484711848F5F712FE002122205B
:10E5F000FFF7C0FF20B940F209111348F5F708FEF4
:10E6000000212320FFF7B6FF20B94FF485710E4893
:10E61000F5F7FEFD00212420FFF7ACFF20B940F202
:10E620000B110948F5F7F4FD00212520FFF7A2FFA3
:10E6300020B94FF486710448F5F7EAFDE368BDE8B8
:10E6400010401847F81000200EB90108E010002013
:10E65000354B70B51B7806460D4623B94FF48B71C8
:10E660003248F5F7D5FD324CA36898474721202062
:10E67000FFF780FF20B94FF48E712C48F5F7C8FDE5
:10E6800009212120FFF776FF20B940F22111274808
:10E69000F5F7BEFD40212220FFF76CFF20B94FF4B3
:10E6A00093712248F5F7B4FD00212320FFF762FFA4
:10E6B00020B94FF496711D48F5F7AAFD00212420DA
:10E6C000FFF758FF20B94FF499711848F5F7A0FDEE
:10E6D00000212520FFF74EFF20B940F237111348E3
:10E6E000F5F796FD95213020FFF744FF20B940F261
:10E6F0003B110E48F5F78CFD31463220FFF73AFF0B
:10E7000020B940F23D110948F5F782FD2946332032
:10E71000FFF730FF20B940F23F110448F5F778FDCC
:10E72000E368BDE870401847F81000200EB90108F2
:10E73000E010002084B073B506AC84E80F002C4CC8
:10E7400006AE25460FCE0FC596E8030085E8030008
:10E7500063690BB9274B636163692748984763680E
:10E7600023B940F27D112548F5F752FD236823B9FE
:10E770004FF4BF712148F5F74BFDA36823B940F270
:10E780007F111E48F5F744FDE36823B94FF4C071CB
:10E790001A48F5F73DFD236923B940F28111174866
:10E7A000F5F736FDA36898470DF107010F20FFF735
:10E7B000D9FEE368984763699DF8071010489847A9
:10E7C0009DF80730332B08D00E4863699847002026
:10E7D00002B0BDE8704004B0704701250A4B1D70BF
:10E7E000FFF7D0FE0948636998472846F0E700BF65
:10E7F000E01000200DDA000818E401080EB9010845
:10E800002BE4010850E40108F810002064E401083A
:10E81000002103E00A4B5B584350043109480A4B7E
:10E8200042189A42F6D3094A02E0002342F8043B18
:10E83000074B9A42F9D300F00DF8F3F719FA704735
:10E840006CF20108000000202405002028050020AB
:10E85000D4180020314B82B01A6842F480721A60DA
:10E8600099682F4A0A409A601A6822F0885222F06A
:10E8700001121A601A6822F480221A609A6822F43F
:10E880007D029A600022DA6001921B6813F4007323
:10E8900018BF01230193019B012B37D14FF4805105
:10E8A000204B1A68A3F5806322F00102C3F800240C
:10E8B000D3F8002422F00202C3F80024D3F8002485
:10E8C00022F00402C3F800245A6A42F080525A62CD
:10E8D000154A11605168C906FCD49A689A609A6812
:10E8E0009A609A689A605A6822F460425A605A683C
:10E8F00042F440425A609A6822F003029A609A6891
:10E900009A60064A936813F00C0FFBD14FF0006237
:10E91000064B9A60064ADA6002B07047003802403F
:10E920000CC0FF88003C02400070004000ED00E099
:10E930000003FA0570B5064688B02E4801F0D8FCF1
:10E940002D4B1A680092009A91073CD501214FF493
:10E95000007001F02DFF012001F01AFD274A5368D5
:10E9600043F400335360A2F5374253681B07FCD5CC
:10E970000024012502A801F0F5FC02A91D488DF82C
:10E980000D4006948DF81C508DF80C4001F0C4FC2D
:10E990002A4606233146174801F006FD2946154848
:10E9A00001F0ECFC0221134801F090FD114801F048
:10E9B0007FFD134D01940F4C0221204601F080FD94
:10E9C00058B108B070BD1A6842F001021A60009A8E
:10E9D0009207BBD41A680092F9E7019B01330193B7
:10E9E000019BB3F5805FE7DB38212846F5F710FC83
:10E9F000E2E700BF00240140003802400027014048
:10EA00000EB9010808B5002001F0C2FC002107483A
:10EA100001F0B4FC00214FF4007001F0C9FE044A7B
:10EA2000136823F00103136008BD00BF00240140F8
:10EA30000038024013B5072301220146114801F0B6
:10EA4000B3FC02210F4801F041FD0E4801F030FDFA
:10EA500000230D4C019302210A4801F031FD28B139
:10EA6000084802B0BDE8104001F027BD019B01330A
:10EA70000193019BB3F5805FEDDB4C212046F5F758
:10EA8000C7FBE8E7002401400EB9010870B506464F
:10EA90000825FFF74FFF00243046FFF7CBFF013D6D
:10EAA0000444F9D1FFF7AEFFC4F3CF0070BD0000FE
:10EAB00008B51120FFF7EAFF07F00CFD01460848F2
:10EAC00007F014FE07F0EEF803A3D3E9002307F0E4
:10EAD00041F907F0F9FB08BD2FDD24068195F33FCE
:10EAE00000F07F450F4A536A43F0805353620E4B48
:10EAF0001A465968C906FCD41B68022823F4C0537F
:10EB000006D143F4C05313605368DB06FCD470474E
:10EB1000012802D143F48053F5E70028F3D143F4F0
:10EB20000063F0E7003802400070004010B50C4B65
:10EB30005A68D206FCD41C6814F4C05F0BD114F4DC
:10EB400080500AD114F4006404D106482A21F5F754
:10EB50005FFB204610BD0220FCE70120FAE700BF62
:10EB6000007000400EB9010838B50546012001F0DB
:10EB7000BDFC022D01BF154A136843F00103136069
:10EB8000134B1A6842F480321A601A689203FCD55B
:10EB900042F690529A6099689142FCD19A6842F08C
:10EBA00002029A600A4B9C6814F00804FBD14FF4EF
:10EBB00080321A60074B084A28461A60FFF792FF16
:10EBC0002046BDE8384001F085BC00BF003C024053
:10EBD00000380240B002002000093D0038B505466B
:10EBE000012001F083FC022D01BF144A136843F099
:10EBF00001031360124B1A6842F480721A601A689B
:10EC00009205FCD55A6822F4604242F440425A60B0
:10EC100000229A600A4B9C6814F00C04FBD14FF45C
:10EC200080721A60074B084A28461A60FFF75AFF9D
:10EC30002046BDE8384001F04DBC00BF003C02401A
:10EC400000380240B0020020D0FE3F000C4B5A6B4F
:10EC5000900513D45A6A42F080525A62094A1168E8
:10EC600041F480711160596B41F480715963596BA3
:10EC70008905FCD5136823F480731360704700BFC7
:10EC80000038024000700040054B5A6B910706D4D3
:10EC90005A6B42F001025A635A6B9207FCD57047D7
:10ECA00000380240094B5A6A42F020025A629A69BF
:10ECB00042F020029A619A6922F020029A610022B1
:10ECC000A3F509331A801A855A627047003802404A
:10ECD000002349F6FE7282B00193019B934201DD4D
:10ECE00002B07047019B01330193F6E7002340F621
:10ECF000FE7282B00193019B934201DD02B0704726
:10ED0000019B01330193F6E7002382B00193019B3D
:10ED1000B3F5CC7F01DD02B07047019B0133F5E70D
:10ED2000D0B1012801D1FFF7EFBF0C4B00211A68C9
:10ED30004FF47A73B2FBF3F2094B013A92B21A859F
:10ED400001220138D8629A82596219821A801A8A7D
:10ED5000D207FCD500221A80704700BFB002002005
:10ED60000014004000F1774303F57803B3F5804FBA
:10ED70002DE9F04106460C4617462DD202F1F73335
:10ED800003F608030344B3F5804F25D2FFF7CEFE08
:10ED9000804610B10020FFF7A5FE01F0BFFB012562
:10EDA0002744361BA7420AD101F0C8FBB8F1000F77
:10EDB00002D04046FFF796FE2846BDE8F08141F6B6
:10EDC000027001F0C3FB301914F8011B01F01AFCAA
:10EDD000042818BF0025E5E70025EDE710B50C462F
:10EDE00000F1774101F57801B1F5804F0DD202F1C4
:10EDF000F73303F608030344B3F5804F05D2014609
:10EE0000204608F0BCF9012010BD0020FCE70000FE
:10EE100008B5114B984215D003F58063984213D082
:10EE200003F58063984211D003F5806398420FD0B8
:10EE300003F5006398420DD0084B094A1421094894
:10EE400007F07CFF002008BD0120FCE70220FAE764
:10EE50000320F8E70520F6E700000240CCE40108B3
:10EE600086E40108E5E401080F2808B505D9094B37
:10EE7000094A3B21094807F061FF012303FA00F02A
:10EE8000C043074A51680140516013681840106040
:10EE900008BD00BF24E5010890E40108E5E401088D
:10EEA000000401400F292DE9F84F82460D46934694
:10EEB0001F4605D95A4B5B4A54215B4807F03EFF79
:10EEC0004FF0010909FA05F900F0B8F86FEA0903F3
:10EED000564E032D7268564C02EA03027260326885
:10EEE00003EA0203534A3360136A43F001031362D7
:10EEF0002ED80F22A3684FEA850802FA08F223EA07
:10EF00000203A3605046FFF783FFA36800FA08F0EE
:10EF10001843A0601BF0020F18BFB368464A1CBF1D
:10EF200043EA0903B3601BF0040F1EBFF36843EA12
:10EF30000903F360336843EA090333603B01DBB242
:10EF4000002D45D182F8063340231360BDE8F88FC9
:10EF5000072D13D80F22A5F10408E3684FEA8808AB
:10EF600002FA08F223EA0203E3605046FFF750FF7B
:10EF7000E36800FA08F01843E060CBE70B2D13D8E4
:10EF80000F22A5F1080823694FEA880802FA08F25F
:10EF900023EA020323615046FFF73AFF236900FA90
:10EFA00008F018432061B5E70F22A5F10C0863694A
:10EFB0004FEA880802FA08F223EA02036361504626
:10EFC000FFF726FF636900FA08F018436061A1E7C4
:10EFD000012D03D182F807338023B6E7022D04D137
:10EFE00082F808334FF48073AFE7032D04D182F821
:10EFF00009334FF40073A8E7042D04D182F80A33D3
:10F000004FF48063A1E7092D04D882F817334FF439
:10F0100000039AE782F828334FF48073536095E732
:10F0200030E50108ABE40108E5E401080004014013
:10F03000000001400038024000E100E0144B98421B
:10F0400005D1144AD36943F00103D3617047124BD1
:10F05000984204D10F4AD36943F00203F5E70F4BFE
:10F06000984204D10B4AD36943F00403EDE70C4BFB
:10F07000984204D1074AD36943F00803E5E7094BF6
:10F080009842E3D1034AD36943F02003DDE700BF90
:10F090000000024000380240000402400008024024
:10F0A000000C0240001402400323490010B584689C
:10F0B0008B4024EA030484600124022A04FA01F448
:10F0C00007D0032A0DD0012A07D183682343836028
:10F0D00003E083688A401A43826083681C4384602B
:10F0E00010BD82681343F2E70F29F8B504460F46B6
:10F0F00015461E4603D94B211948F5F789F82046D5
:10F10000FFF79CFF03237A009340DB4321681940FB
:10F1100021600121D4F800C001FA02F04CEA000C91
:10F12000B940C4F800C009B266B1A688314389B2BB
:10F13000A180E168012D03EA0103E36006D0022DFE
:10F1400008D0F8BDA68826EA0101F1E7E368034389
:10F15000E360F6E7E36805FA02F21A43E260F0E7DB
:10F160000EB901080F2970B505460C46164603D99D
:10F170006B210E48F5F74CF82846FFF75FFF032395
:10F1800061008B40DB43EA68012E02EA0302EA6079
:10F1900005D0022E03D02A6813402B6070BDEA68A8
:10F1A00006FA01F11143E960F5E700BF0EB9010865
:10F1B0000F2938B50446154605D987211B4B1C4A33
:10F1C0001C4807F0BBFD0F2A03D91B4B184A8821A6
:10F1D000F6E7FFF733FF07294FF00F0318D8006A4F
:10F1E0008A00934020EA03032362236A05FA02F2AD
:10F1F0001A4322620322236849008A4023EA020359
:10F2000023600223226803FA01F11143216038BD13
:10F21000A1F10802406A9200934020EA030363626E
:10F22000636A95401D436562E4E700BF24E5010879
:10F230003CE501086DE501085AE50108012303FAE0
:10F2400001F189B201837047012303FA01F189B208
:10F2500041837047012303FA01F189B20AB10183A6
:10F26000704741837047008A084100F001007047F1
:10F270000F2938B505460C4603D9B4210548F4F7E3
:10F28000C7FF28686400E04000F00300431E5842B6
:10F29000584138BD0EB90108808A084100F00100CC
:10F2A0007047000010B5084C23681BB90120F4F723
:10F2B00087FB206023682BB9BDE810403621034846
:10F2C000F4F7A6BF10BD00BFFC1000200EB9010866
:10F2D00010B50B4C22681AB93C210A48F4F798FF84
:10F2E000206842F21071F4F7B3FC01280CBF01242E
:10F2F000002403D040210348F4F78AFF204610BDC4
:10F30000FC1000200EB9010810B5074C22681AB98C
:10F3100051210648F4F77CFF002320681A46BDE817
:10F3200010401946F4F7A8BAFC1000200EB90108E5
:10F3300010B50446FFF7B6FFFFF7CAFF21461022BB
:10F34000034801F021FF0446FFF7DEFF204610BD11
:10F350000054004010B5FFF7A5FFFFF7B9FF01F01B
:10F36000CBFE0446FFF7D0FF204610BD08B513467C
:10F370000A460146034801F0FFFA003018BF012099
:10F3800008BD00BF0054004008B513460A460146B8
:10F39000034801F0F1FB003018BF012008BD00BF99
:10F3A0000054004008B513460A460146034801F0E0
:10F3B000BFFC003018BF012008BD00BF0054004052
:10F3C00008B513460A460146034801F041FD0030E6
:10F3D00018BF012008BD00BF0054004008B5134607
:10F3E0000A460146034801F08BFD003018BF01209A
:10F3F00008BD00BF005400400123064A8340516904
:10F40000194205D05361044B53F8203003B118471B
:10F41000704700BF00040140001100200F2838B5DC
:10F4200004460D4603D926210348F4F7F1FE034BA9
:10F4300043F8245038BD00BF0EB901080011002068
:10F440000020FFF7D9BF0120FFF7D6BF0220FFF74A
:10F45000D3BF0320FFF7D0BF0420FFF7CDBF08B50F
:10F460000920FFF7C9FF0820FFF7C6FF0720FFF7B5
:10F47000C3FF0620FFF7C0FFBDE808400520FFF7E7
:10F48000BBBF08B50F20FFF7B7FF0E20FFF7B4FF93
:10F490000D20FFF7B1FF0C20FFF7AEFF0B20FFF7A9
:10F4A000ABFFBDE808400A20FFF7A6BFFEE7FEE776
:10F4B000FEE7FEE7FEE7FEE7FEE7FEE7FEE7FEE724
:10F4C000FEE7FEE7FEE7FEE7FEE7FEE7FEE7FEE714
:10F4D000FEE7FEE7FEE7FEE7FEE7FEE7FEE7FEE704
:10F4E000FEE7FEE7FEE7FEE7FEE7FEE7FEE7FEE7F4
:10F4F000FEE7FEE7FEE7FEE7FEE7FEE70A23B0FBD6
:10F50000F3F203FB120040EA0210C0B270470000A1
:10F51000CA22024B5A6253225A62704700280040A6
:10F52000014B1860704700BF401100204FF40032BB
:10F530000F4B10B50F4C5A61E368DB0503D4302143
:10F540000D48F4F765FEFFF7E3FF4FF40072A36880
:10F5500023F48853A360094BC3F88420FF2363621C
:10F56000074B1B6813B1BDE81040184710BD00BF22
:10F5700000040140002800400EB9010800E100E04D
:10F58000401100202DE9F04F9846374B85B01B788D
:10F59000824691469DF838709DF83C602BB9334BFC
:10F5A000334A8C21334807F0C9FB431E1E2B59D820
:10F5B0000C2957D8A2F5FA63632B53D8B8F1170F6B
:10F5C00050D83B2F4ED83B2E4CD802F13000C0B261
:10F5D000FFF794FF83460846FFF790FF0446504626
:10F5E000FFF78CFF40F400554046FFF787FF45EAE0
:10F5F0000B4545EA042504463846FFF77FFF000225
:10F6000040EA04443046FFF779FF20431A4CFFF7E5
:10F610007FFFE36843F08003E360E3685B06FCD5AB
:10F6200065602060E36823F08003E360124BDA68D2
:10F630009206FCD5FF2204A85A6200F80C6D8DF8E2
:10F6400007A08DF80810ADF809908DF806808DF8A8
:10F650000570FEF71BF9094BC3E90001012005B055
:10F66000BDE8F08F0020FAE744110020DDE5010835
:10F67000D1E50108E6E50108002800404811002016
:10F6800037B50578C4788378B0F8052001790195FD
:10F69000407800902046FFF775FF03B030BD0000B2
:10F6A00038B52B4B04461B781BB9E4212948F4F7E5
:10F6B000AFFD294AD36823F02003D360D3689B06AB
:10F6C000FCD513685268C2F30741080900EB8000BB
:10F6D00001F00F0101EB4001C9B201F5FA61A4F894
:10F6E0000510C2F30721C1F300108500284401F082
:10F6F0000F0101EB4001D2B22171C2F3011101EB04
:10F70000810102F00F0202EB4102E270C3F30742F3
:10F71000C2F3011101EB810102F00F0202EB410281
:10F72000A270C3F30722C2F3021101EB810102F0C0
:10F730000F0202EB4102DBB26270C3F3021202EB72
:10F74000820203F00F0303EB4203237038BD00BFB6
:10F75000441100200EB90108002800401FB501A87F
:10F76000FFF79EFF01A8FEF791F805B05DF804FBD6
:10F7700008B5FFF76BFA1B4A136843F480731360F4
:10F78000FFF7C6FE184A536B23F4403343F4820359
:10F790005363164BDA6842F08002DA60DA68510689
:10F7A000FCD5FF221A611A6942F4FE021A619A68B6
:10F7B00022F040029A609A6822F44C529A60DA6809
:10F7C00022F08002DA60094BDA689206FCD5FF224B
:10F7D0005A620122064B1A70FFF7C0FF054BC3E9BE
:10F7E000000108BD007000400038024000280040C1
:10F7F000441100204811002008B5094B1B7823B99B
:10F8000040F21F110748F4F703FDFFF781FE064B96
:10F810009A6822F480729A60FF225A6208BD00BF83
:10F82000441100200EB901080028004008B5144B0F
:10F830001B7833B9134B144A40F22711134807F0D1
:10F840007DFAFFF765FE124BDA6822F48072DA6007
:10F85000104A916841F400319160116841F400311F
:10F860001160F0210C4A82F829134FF400715160A5
:10F870009A6842F488529A60FF225A6208BD00BF1B
:10F8800044110020DDE50108AAE50108E6E50108CC
:10F89000002800400004014000E100E0F8B51E46E9
:10F8A000194B17461B7833B9184B194A4FF4A571F9
:10F8B000184807F043FA184CFFF72AFEA56825F40C
:10F8C0008075A560E56825F48075E560FFF716FE94
:10F8D00005460846FFF712FE000440EA0561384677
:10F8E000FFF70CFE05463046FFF708FE084340EAE6
:10F8F0000520E368DB07FCD5FF23E0616362BDE818
:10F90000F840FFF793BF00BF44110020DDE5010878
:10F91000BFE50108E6E501080028004003784278C9
:10F920008178C078FFF7BABF38B50D460446F3F7C3
:10F9300061FD1F4A136823F001031360F3F77AFD9A
:10F9400025B11C4A536843F00603536072B6BFF3F7
:10F950004F8FBFF36F8F184A0120136823F0030302
:10F9600043F4007343F00103136000F0CBFD134B2D
:10F970001A6942F004021A6130BF1A6922F00402C7
:10F980001A610F4B0F4A1B6893420AD10220FFF7FE
:10F9900025F9074A136843F00103136004B162B606
:10F9A00038BD094A9342F4D10220FFF7DDF8F0E7B1
:10F9B00010E000E0002004E00070004000ED00E0F6
:10F9C000B0020020D0FE3F0000093D0062B6704743
:10F9D00010B5064C23783BB1054B02221868197903
:10F9E000FFF7C0FB0023237010BD00BF50110020A3
:10F9F000141800202DE9F041069C0646404804609A
:10FA00009DF81C40047181714271C3714379827900
:10FA100001334E2A18BF0133DBB20372C3790446A7
:10FA2000DBB2022B69D05AD8012B61D0354D2B683F
:10FA300043B90120F3F7C4FF286018B96C2132489C
:10FA4000F4F7E6FB0127206821793A4607FA01F12D
:10FA500089B200F03FFE2068002321793A46FFF783
:10FA600043FB2A4B2A4D5A6A42F010025A629A69A5
:10FA700042F010029A619A6922F010029A614FF4E2
:10FA8000807200232B802B85AA816B6284232B80BC
:10FA9000204B186806F01EFD1F4B196806F072FD1A
:10FAA0008046304606F016FD0146404606F01EFE32
:10FAB00006F06AFF3946E8624FF0807000F06CFE95
:10FAC00043F69022154B1A600D225A60144ADA60F0
:10FAD000226818329A60134B1F70BDE8F081052B25
:10FAE00001D00F2BA2D15F210748F4F791FB9DE7CE
:10FAF000037A0133DBB2237298E7037A0233F9E722
:10FB000014180020541100200EB9010800380240DA
:10FB100000100040B0020020B40200201C6002402F
:10FB20002018002050110020F8B54B4B04461B78DC
:10FB30001BB9A7214948F4F76BFB01250027484E64
:10FB40002A463068317905FA01F189B200F0C2FD28
:10FB50003279334605FA02F21204F2603A46FEB2F6
:10FB60005979701CC0B2B14200F1020155D89C799C
:10FB7000452C64D112F0010F4FF00102187902FAFE
:10FB800000F267D003EB8101B01C4A60C0B20122D1
:10FB90001979441C023002FA01F103EB8005696017
:10FBA000D979E4B2022906D11979023403EB84042D
:10FBB0008A406260C4B21B7AA34203D0D321274893
:10FBC000F4F726FB2021274B274A54605960A3F500
:10FBD0001433198821F001010904090C198000214E
:10FBE00019825962596A0029FCD1116841F001015A
:10FBF0001160198841F0010119801A490B689B06B0
:10FC0000FCD5136823F001031360184A138823F00E
:10FC100001031B041B0C1380F8BD1879E60705FAD5
:10FC200000F047BF03EB81010132000403EB8101C7
:10FC300046BF4860D2B24860640801378FE79C79BC
:10FC40004F2CA4D112F0010F4FF00102187902FAE3
:10FC500000F297D0120495E7501100200EB9010868
:10FC600014180020006002401C6002400010004098
:10FC7000054AD36823F4E0631B041B0C43F0BF6305
:10FC800043F40033D360704700ED00E020220021F0
:10FC9000114B10B5C3F88420104B114C1A6A204642
:10FCA00042F480421A625A6942F480425A615A69A7
:10FCB00022F480425A610B4A91811A6A092122F486
:10FCC00080421A620222FFF74DFA2046BDE810403A
:10FCD00002220A21FFF746BA00E100E000380240A4
:10FCE000000002400038014010B50B4C40F2255195
:10FCF000204600F01AFE48B1204600F0F4FD074B04
:10FD0000C0B21B6833B1BDE810401847A388044A4D
:10FD1000DBB2137010BD00BF003801405811002045
:10FD20005418002010B504468021084800F0F7FD63
:10FD30000028F9D02146054800F0D1FD034C4021B0
:10FD4000204600F0ECFD0028F9D010BD003801403D
:10FD500010B5441E14F8010F00B910BDFFF7E2FF03
:10FD6000F8E7000008B5024800F0BDFDC0B208BDCC
:10FD7000003801402DE9F0438846012189B08146D1
:10FD8000084614461D4600F007FD01214FF480404F
:10FD900000F00EFD4FF4C06702230122002602A9E5
:10FDA0003F488DF80C308DF80D308DF80F200297FC
:10FDB0008DF80E6000F04CFC07220921384800F055
:10FDC0008EFC07220A21364800F089FCB8F1450F65
:10FDD000CDF810903CD14FF48063ADF81830072C6B
:10FDE00042D10023ADF81430052D4ED14FF480538D
:10FDF000ADF816300023ADF81C300C2304A92948B7
:10FE0000ADF81A3000F010FD274B1A6802B101223C
:10FE100040F22551234800F06AFD0121214800F0FD
:10FE200053FDFFF79FFF25238DF804309DF84030E8
:10FE30008DF8053000238DF8063001238DF807304A
:10FE4000FFF716FF01A800F037FA09B0BDE8F0830C
:10FE5000B8F14F0F02D1ADF81870C0E7072CADF81C
:10FE600018600DD1592107E0082C02D14FF48053BE
:10FE7000B8E7092CB8D154210C48F4F7C9F9B3E715
:10FE8000082CAED0092CAFD1F0E70F2D02D14FF4E2
:10FE90004053ADE7022D0CBF4FF400530023A7E7FA
:10FEA0000000024000380140581100200EB901083E
:10FEB0000E2307B5082200934E210123FFF75AFFB6
:10FEC00003B05DF804FB0000402200210D4B0E48FA
:10FED000C3F884200D4B5A6A42F400325A629A6980
:10FEE00042F400329A619A6922F400329A61084A17
:10FEF00091815A6A032122F400325A620222FFF7EA
:10FF000031B900BF00E100E00000024000380240CB
:10FF10000044004008B5024800F0E5FCC0B208BD4E
:10FF2000004400402DE9F04F4FF000091F46262302
:10FF300089B09DF848808A4614468DF8043083467F
:10FF40009DF84C509DF850608DF805808DF8069016
:10FF50008DF80790FFF78CFE01A800F0ADF90121A4
:10FF6000084600F019FC01214FF4003000F02CFC91
:10FF7000B5B10823029302238DF80E908DF80C3052
:10FF80004FF00309012302A956488DF80F308DF870
:10FF90000D9000F05DFB07224946524800F09FFBA0
:10FFA000BEB10423029301238DF80F3000234FF0DC
:10FFB00002098DF80E30032302A94A488DF80C90EF
:10FFC0008DF80D3000F044FB07224946454800F00B
:10FFD00086FBBAF1450FCDF810B043D14FF48063E2
:10FFE000072CADF818304BD10023ADF81430052F95
:10FFF00057D14FF480530024ADF81630ADF81C40B3
:020000040801F1
:10000000002E59D1ADF81A6075B1BDF81A3043F021
:100010000403ADF81A30344B1A6802B1012240F2E1
:100020002551324800F063FC04A9304800F0FCFB85
:1000300001212E4800F048FC0DB1FFF76BFF26238D
:100040008DF8043000238DF8063001238DF80580EB
:100050008DF80730FFF70CFE01A800F02DF909B06C
:10006000BDE8F08FBAF14F0F02D14FF4C063B7E78C
:100070000023072CADF818300ED14FF4827107E041
:10008000082C02D14FF48053AFE7092CAFD1FF21E8
:100090001748F4F7BDF8AAE7082CA5D0092CA6D17B
:1000A000F0E70F2F02D14FF44053A4E7022F0CBF0B
:1000B0004FF4005300239EE70823224640F22771A5
:1000C0000A48ADF81A3000F012FC40F226610748E9
:1000D00000F04AFC224640F22661044800F007FC8A
:1000E00092E700BF000002405C1100200044004085
:1000F0000EB9010808B5064B0246186000B101228E
:1001000040F22551034800F0F2FB012008BD00BF7A
:100110005C1100200044004070B5134C40F22551A2
:10012000204600F002FCC0B1104B1D6825B12046EE
:1001300000F0D9FBC0B2A84740F226610A4800F09F
:10014000F4FB78B140F22661074800F00DFC084B43
:100150001B683BB1BDE870401847A388054ADBB275
:100160001370E9E770BD00BF004400405C1100203F
:100170006011002054180020BFF34F8F0449054B35
:10018000CA6802F4E0621343CB60BFF34F8FFEE70F
:1001900000ED00E00400FA0510B5441EE3B2052BA3
:1001A00003D90E211148F4F733F8FEF76DFD45F23F
:1001B00055520F4B1A60DA68D207FCD4052C06D8CA
:1001C000DFE804F003090B0D0F1101225A604CF611
:1001D000CC421A6010BD0222F8E70322F6E704229F
:1001E000F4E70522F2E70622F0E700BF0EB90108A6
:1001F0000030004038B5224C236853B95F2000F02E
:10020000FBFA204D38B1204B236001232B7000F006
:1002100003FB206838BD5E2000F0EEFA18B11B4BDE
:1002200023600223F2E75D2000F0E6FA18B1184BD4
:1002300023600323EAE75C2000F0DEFA18B1154BD7
:1002400023600423E2E75B2000F0D6FA18B1124BDA
:1002500023600523DAE75A2000F0CEFA18B10F4BDD
:1002600023600623D2E7592000F0C6FA18B10C4BE0
:1002700023600723CAE70B4B2360FF23C6E700BFB9
:10028000641100206811002022E6010832E601080E
:1002900048E6010863E6010872E6010881E6010804
:1002A0009AE6010884D3010808B5FFF7A3FF014BC4
:1002B000187808BD6811002030B5012403780A4D74
:1002C00003F01F029440C278590952B1074A2B44E7
:1002D000D26842781201D2B283F8002345F8214057
:1002E00030BD2031FAE700BF00E100E000ED00E0A2
:1002F00008B5084B98420BD101214FF4007000F073
:100300006FFABDE8084000214FF4007000F068BAB1
:1003100008BD00BF0024014043680A7923F0407300
:1003200023F4807343EA02230A6810B51343436041
:10033000D1E9032313438A6884681343084A22409F
:1003400013434A7943EA420383600A7D036B013A0F
:1003500023F0F873D2B243EA0253036310BD00BF27
:10036000FDF7FFC000234FF040720360037143713B
:100370008360C0E90323012303757047836819B1C3
:1003800043F001038360704723F00103FAE70000A4
:10039000044B5A6818B142F400025A60704722F4C4
:1003A0000002FAE7002701401D2970B51BD9072577
:1003B000A1F11E06C46D06EB4606B54024EA05040D
:1003C00003FA06F62643C665062A38D81F24013AE2
:1003D000036C02EB8202944023EA040301FA02F266
:1003E0001A43026470BD13290DD90726A1F1140523
:1003F000C46805EB4505AE4024EA060403FA05F59A
:100400002543C560E0E709290DD90726A1F10A04B3
:10041000056904EB4404A64025EA060503FA04F442
:100420002C430461D0E70726446901EB4105AE4047
:1004300024EA060403FA05F626434661C4E70C2ABB
:100440000CD81F24073AC36B02EB8202944023EAC4
:10045000040301FA02F21A43C263C3E7122A0CD85A
:100460001F240D3A836B02EB8202944023EA0403BB
:1004700001FA02F21A438263B4E7182A0CD81F2447
:10048000133A436B02EB8202944023EA040301FA1D
:1004900002F21A434263A5E71F24193A036B02EBE9
:1004A0008202944023EA040391401943016399E7CF
:1004B000836843F0804383607047806D80B27047EB
:1004C0000368194214BF012000207047C94301602E
:1004D00070470000044B1A6818B142F002021A601B
:1004E000704722F00202FAE7003C0240044B1A680F
:1004F00018B142F004021A60704722F00402FAE7D1
:10050000003C0240044B1A6818B142F008021A601D
:10051000704722F00802FAE7003C0240044B5A6898
:10052000D20741BF034ADA60034ADA60704700BF6E
:10053000003C0240EFCDAB8905040302024A536838
:1005400043F0010353607047003C0240014B986147
:10055000704700BF003C0240084B9A69D10709D49C
:100560009A69D20508D49B6913F4F05F14BF032085
:10057000042070470120704702207047003C024071
:10058000042313B504468DF80730FFF7E5FF8DF817
:1005900007009DF80730012B0AD11CB905238DF8FF
:1005A000073007E0FFF7D8FF013C8DF80700F0E7C0
:1005B000002CF3D09DF8070002B010BD10B5044622
:1005C0004FF40040FFF7DCFF042804BF0023236042
:1005D00010BD000038B504464FF400400D46FFF74B
:1005E000CFFF04280BD1064A4FF40040536823F490
:1005F000807353602560BDE83840FFF7C1BF38BD48
:10060000003C024038B504464FF400400D46FFF769
:10061000B7FF04281BD135B125704FF40040BDE869
:100620003840FFF7ADBFFF2324F0030504F00304B7
:100630002968E40003FA04F421EA04042846FFF7D9
:10064000BDFF21462846BDE83840FFF7C3BF38BD8F
:100650002DE9F0430022012703250E6807FA02F373
:1006600033EA060431D14FEA420C05FA0CF4E443B4
:1006700091F804E0D0F800900EFA0CF804EA0909A9
:100680000EF1FF3E48EA0908BEF1010FC0F80080F4
:1006900011D8D0F808E004EA0E0E4C7904FA0CF4F4
:1006A00044EA0E048460848824EA03048B7993402E
:1006B0009BB223438380C36805FA0CF423EA040445
:1006C000CB7903FA0CF32343C3600132102AC5D15E
:1006D000BDE8F0830AB1018370474183704710B5CC
:1006E0000F2401F00703C90800EB8100016A9B0099
:1006F0009C4021EA04010162016A9A400A430262B5
:1007000010BD0000204B10B59A6802F00C020C2AB4
:1007100030D8DFE802F02F2F2F2F072F2F2F072F92
:100720002F2F2000194B184A036093681849C3F310
:100730000313CC5C0368E34043609468C4F3022471
:100740000C5D23FA04F484609268C2F3C2228A5CCE
:10075000D340C36010BD99680E4CC1F383419A68C1
:10076000615C9B68094BC2F381524B430132B3FB7E
:10077000F2F3D8E74FF400425B68C3F3423301332E
:1007800002FA03F3CFE700BF003802400024F40070
:10079000B8020020C8020020044BDA6911B11043EE
:1007A000D861704722EA0000FAE700BF0038024033
:1007B000044B1A6A11B110431862704722EA000014
:1007C000FAE700BF00380240044B5A6A11B11043E7
:1007D0005862704722EA0000FAE700BF0038024082
:1007E000044B5A6911B110435861704722EA000066
:1007F000FAE700BF003802404309012B054B00F027
:100800001F000CBF1B685B6B23FA00F000F00100B7
:10081000704700BF00380240024A536B43F08073B8
:10082000536370470038024030B50D460446028AD3
:10083000EB8892B222F440521A438989028283895A
:10084000288923F4B052AB8822F00C020343688954
:1008500085B003431343A381A38A68469BB223F464
:1008600040730B43A382FFF74DFFDDE90231154AC8
:10087000944218BF19461923A2894B4329681004D2
:100880004CBF49008900B3FBF1F16425B1FBF5F3DE
:10089000A2891801120405FB13130BD5DA003232BA
:1008A000B2FBF5F202F0070242EA00039BB2238199
:1008B00005B030BD1B013233B3FBF5F303F00F037A
:1008C0000343F3E700380140838919B143F400532F
:1008D0008381704723F400531B041B0CF8E7C1F31A
:1008E0000801818070478088C0F30800704701F0DC
:1008F0001F0310B5C1F342140121012C01FA03F1C9
:1009000005D10C3003683AB11943016010BD022CC7
:100910000CBF10301430F5E723EA0101F5E7038836
:10092000194214BF0120002070470123C1F3421275
:1009300010B5012A01F01F0403FA04F30DD18289D6
:100940001340028892B26BB10123090A03FA01F144
:100950000A4214BF1846002010BD022A0CBF028AAA
:10096000828AEDE71846F7E70B0A01219940C9434F
:1009700089B20180704700002DE9F3411F46002332
:1009800004460D46019316461AB9012002B0BDE88F
:10099000F08140F6FF7301934FF40031204600F0E0
:1009A0004CFD002852D10121204600F016FD4FF2E7
:1009B000FF71204600F02AFD0121204600F0F7FCDF
:1009C00040F6FF73DFF8AC8101934146204600F00A
:1009D00029FD002841D039460122204600F008FDBB
:1009E00040F6FF735F4F01933946204600F025FD26
:1009F000002838D0012E42D10021204600F0EDFC25
:100A0000F2F7F8FC31462046238B00F0DBFCF2F7CE
:100A100011FD40F6FF73544E01933146204600F01D
:100A20000CFD30B3204600F0EEFC287040F6FF735A
:100A30004E4D01932946204600F0FFFC0028A4D02B
:100A4000019B5A1E0192002BF4D104E0019B5A1E17
:100A50000192002BA0D1002098E7019B5A1E019221
:100A6000002BB2D1F7E7019B5A1E0192002BBBD19C
:100A7000F1E7019B5A1E0192002BCED1EBE7022E2B
:100A800025D1F2F7B7FC4FF40061204600F0BEFC20
:100A90000021204600F0A1FC238BF2F7CBFC40F6AE
:100AA000FF73334E01933146204600F0C6FC40B13F
:100AB0000121204600F086FC238A2B70238A6B706C
:100AC000B4E7019B5A1E0192002BECD1C3E740F61C
:100AD000FF77033E238BDFF898802E44B5420197C1
:100AE00028D1234E3146204600F0A7FC70B30021E8
:100AF000204600F072FC204600F085FC40F6FF73B3
:100B00001B4E287001933146204600F096FC18B326
:100B10000121204600F056FC204600F074FC68706D
:100B2000204600F070FCA87080E7019B5A1E0192DD
:100B3000002B90D04146204600F07FFC0028F4D0E6
:100B4000204600F060FC05F8010BC7E7019B5A1E28
:100B50000192002BC6D17EE7019B5A1E0192002B09
:100B6000D1D178E702000010400000101000001002
:100B700004000010010003002DE9F3411E4600238C
:100B8000019340F6FF7304460D4617460193002A71
:100B900000F081804FF40031204600F04EFC002828
:100BA00042D10121204600F002FC40F6FF73DFF83D
:100BB0007C8101934146204600F034FC00283CD063
:100BC00031460022204600F013FC40F6FF73534EDE
:100BD00001933146204600F025FC002833D02978C7
:100BE00020466E1C00F00DFC3D4440F6FF77DFF818
:100BF0003081AE42019731D1494D2946204600F05F
:100C00001CFC002836D02046012100F0DBFB40F61A
:100C1000FF73444D444C01932946204600F00DFCDF
:100C200000282DD1012005E0019B5A1E0192002BC6
:100C3000B0D1002002B0BDE8F081019B5A1E0192A4
:100C4000002BB7D1F5E7019B5A1E0192002BC0D1B2
:100C5000EFE7019B5A1E0192002BEAD04146204645
:100C600000F0EBFB0028F4D016F8011B204600F042
:100C7000C8FBBEE7019B5A1E0192002BBDD1D8E7ED
:100C8000019B5A1E0192002BC6D1D2E7019B5A1E2E
:100C90000192002BCDD04FF40031204600F0CDFB67
:100CA0000028F3D10121204600F081FB40F6FF73BC
:100CB0001E4D01932946204600F0B4FB10B30022DC
:100CC0003146204600F094FB40F6FF73134D01932C
:100CD0002946204600F0A6FBD0B12046012100F0B5
:100CE00071FB40F6FF730F4D0F4C019329462046D0
:100CF00000F0A3FB002895D0019B5A1E0192002B07
:100D0000F4D196E7019B5A1E0192002BD2D190E7B5
:100D1000019B5A1E0192002BDAD18AE7820007005C
:100D200004000010100000100054004001000300F7
:100D30002DE9F3411E46002304460D460193174654
:100D40001AB9012002B0BDE8F08140F6FF730193AB
:100D50004FF40031204600F070FB002837D101210C
:100D6000204600F024FB40F6FF73DFF8E08001939B
:100D70004146204600F056FB002842D03146002272
:100D8000204600F035FB40F6FF732C4E01933146B0
:100D9000204600F047FB002839D0297820466E1CF9
:100DA00000F02FFB3D4440F6FF77DFF89480AE4221
:100DB000019737D1224D2946204600F03EFB0028FE
:100DC000BFD1019B5A1E0192002BF4D104E0019B7C
:100DD0005A1E0192002BBBD12046012100F0F2FAED
:100DE00040F6FF73174D184C01932946204600F03A
:100DF00024FB20B1019B5A1E0192002BF5D100204B
:100E0000A0E7019B5A1E0192002BB1D1E4E7019BA0
:100E10005A1E0192002BBAD1DEE7019B5A1E0192A5
:100E2000002BD9D04146204600F007FB0028F4D023
:100E300016F8011B204600F0E4FAB8E7820007002C
:100E400004000010100000100054004001000300D6
:100E500000232DE9F3410D464FF4003104461746B7
:100E6000019300F0EAFA18B9002002B0BDE8F08161
:100E70000FB90120F9E7297820466E1C00F0C1FA6D
:100E80003D4440F6FF77DFF86C80AE4201971FD1FA
:100E9000184D2946204600F0D0FA28B320460121FB
:100EA00000F090FA40F6FF73134D144C019329465D
:100EB000204600F0C2FA0028DBD0019B5A1E0192A6
:100EC000002BF4D1D0E7019B5A1E0192002BCBD00E
:100ED0004146204600F0B1FA0028F4D016F8011B74
:100EE000204600F08EFAD0E7019B5A1E0192002B9B
:100EF000CFD1B9E7040000101000001000540040EA
:100F00002DE9F3411F46002304460D460193164682
:100F10001AB9012002B0BDE8F0814FF4003100F0B1
:100F20008CFA08B90020F5E70121204600F055FAB7
:100F30004FF2FF71204600F069FA0121204600F0CF
:100F400036FA40F6FF73DFF8AC8101934146204644
:100F500000F068FA00283AD039460122204600F015
:100F600047FA40F6FF735F4F01933946204600F081
:100F700064FA002831D0012E3BD10021204600F038
:100F80002CFAF2F737FA31462046238B00F01AFA92
:100F9000F2F750FA40F6FF73534E01933146204664
:100FA00000F04BFAF8B1204600F02DFA287040F618
:100FB000FF734E4D01932946204600F03EFA00286B
:100FC000A7D0019B5A1E0192002BF4D1AAE7019BE6
:100FD0005A1E0192002BB9D1A4E7019B5A1E01921F
:100FE000002BC2D19EE7019B5A1E0192002BD5D146
:100FF00098E7022E29D14FF40061204600F006FA4E
:10100000F2F7F8F900212046238B00F0E6F9F2F719
:1010100011FA40F6FF73364E01933146204600F038
:101020000CFA60B1F2F7E6F90121204600F0CAF9A6
:10103000238A2B70238A6B70F2F7FCF9B7E7019BC8
:101040005A1E0192002BE8D16CE740F6FF77033E71
:10105000238BDFF89C802E44B542019729D1244E82
:101060003146204600F0E9F978B30021204600F02F
:10107000B4F9204600F0C7F940F6FF731C4E287003
:1010800001933146204600F0D8F920B301212046D3
:1010900000F098F9204600F0B6F96870204600F09C
:1010A000B2F9A87083E7019B5A1E0192002B3FF40E
:1010B00039AF4146204600F0C0F90028F3D0204661
:1010C00000F0A1F905F8010BC6E7019B5A1E019239
:1010D000002BC5D126E7019B5A1E0192002BD0D1CF
:1010E00020E700BF020000104000001010000010B8
:1010F000040000100100030038B5204B08219A6954
:101100001F4842F400129A619A6922F400129A610F
:101110005A6A22F400125A62FEF790F8012308215D
:101120001A461748FDF7E0FF092115480122FEF78E
:1011300019F809211248FEF796F8D8B1012038BDF8
:1011400008212846FEF77AF8FDF7DEFD082128463B
:10115000FEF77AF8FDF7D8FD013CF1D109210848E6
:10116000FEF781F820B940F27D110648F3F750F8F8
:101170002046E4E73324024DEEE700BF003802408A
:10118000000402400EB901082DE9FF41444B054619
:1011900098420E4617467CD103F5F2335A6A08216D
:1011A00042F400125A629A693E4842F400129A616F
:1011B0009A6922F400129A61FEF740F8012308218F
:1011C0001A463848FDF790FF092136480122FDF7FD
:1011D000C9FF09213348FEF746F8002855D00123FE
:1011E00008211A462F48FDF77FFF042208212D48C9
:1011F000FDF7DEFF012309211A462A48FDF774FF97
:10120000042209212748FDF7D3FF274B9A6942F4AE
:1012100000129A619A6922F400129A61684600F0FD
:10122000ADF8224B694601934FF48063ADF80A3064
:101230004FF480432846ADF80C30ADF808700096A6
:1012400000F038F82846012100F0A6F8012019E046
:1012500008214046FDF7F2FFFDF756FD0821404604
:10126000FDF7F2FFFDF750FD013CF1D109210D48DA
:10127000FDF7F9FF0028B2D10D4840F2A511F2F7B1
:10128000C7FF204604B0BDE8F0813324DFF81480A6
:10129000EAE74FF4DA710648F2F7BAFFBEE700BF9B
:1012A0000054004000040240003802400000FFBF2C
:1012B0000EB901087FB50446868868460D46FFF7DB
:1012C00021FA029A2B4926F03F06B2FBF1F13604CF
:1012D000360C88B20643A6802388274E23F00103EC
:1012E0001B041B0C23802B68B3421ED85B00B2FB8F
:1012F000F3F39BB2042B38BF0423013080B2208467
:10130000A3832388AA8843F0010323802388698963
:1013100023F481630A4323F00203134323802A89C1
:10132000AB891343238104B070BD4BF6FF70EE8888
:1013300086421BBF1920434303EB4303B2FBF3F385
:101340000BBFB2FBF3F39BB29BB243F48043C3F3F6
:101350000B020AB943F001034FF496724A434FF46B
:101360007A7192FBF1F2013292B243F4004322848B
:10137000C6E700BF40420F00A086010041F288325C
:10138000044BC0E90023002383604FF48043838132
:10139000704700BF0000FFBF038819B143F001038D
:1013A0000380704723F001031B041B0CF8E703883C
:1013B00019B143F480730380704723F480731B04D6
:1013C0001B0CF8E7038819B143F4007303807047DE
:1013D00023F400731B041B0CF8E7038819B143F4D2
:1013E00080630380704723F480631B041B0CF8E7C1
:1013F00022B141F0010189B20182704701F0FE0182
:10140000F9E701827047008AC0B270470388B1F5DE
:10141000006F1BBF23F400631B0443F400631B0C29
:1014200003807047838A008B43EA004321F07F40AA
:101430001840431A584258417047002382B0009325
:1014400001930B0F01900093009B21F07F4153B15A
:10145000019B14330193019B1B680B4214BF0120B5
:10146000002002B07047019B090C1833F2E70078A6
:10147000013070470FB404B0704700002DE9FF47FA
:101480000F46002104AC254E44F8041D80469246C8
:10149000306822469946F2F71DFD0128039B31D1A1
:1014A0003BB14FF080521E4B1A60BFF34F8FBFF31A
:1014B0006F8FB7F5C87F88BF4FF4C87741463A466B
:1014C000184805F05CFE184D164B21463068AF8079
:1014D0002B60A5F806A085F80890F2F7DDFA039BCB
:1014E0003BB14FF080520E4B1A60BFF34F8FBFF3EA
:1014F0006F8F0E4800940023012204210068F1F749
:1015000071FC039B3BB14FF08052054B1A60BFF357
:101510004F8FBFF36F8F04B0BDE8F08770130020CA
:1015200004ED00E0D4110020C81100207C1300203D
:1015300003480023012202210068F1F7E3BB00BF4A
:101540007C1300201FB5F0F7C5FE0D4B04AA1860F0
:10155000002342F8043D009201220A481146006827
:10156000F1F740FC039B3BB14FF08052064B1A60F1
:10157000BFF34F8FBFF36F8F05B05DF804FB00BF63
:10158000781300207C13002004ED00E01FB5002339
:1015900004AA42F8043D0A48009280210122006812
:1015A000F1F720FC039B3BB14FF08052054B1A60D2
:1015B000BFF34F8FBFF36F8F05B05DF804FB00BF23
:1015C0007C13002004ED00E01FB5104B1C6803469F
:1015D000A8B1002304AA42F8043D00920821012288
:1015E0002046F1F7FFFB039B3BB14FF08052084BC5
:1015F0001A60BFF34F8FBFF36F8F04B010BD01228D
:1016000008212046F1F77EFBF7E700BF7C1300209E
:1016100004ED00E01FB5002304AA42F8043D0A4887
:101620000092102101220068F1F7DCFB039B3BB123
:101630004FF08052054B1A60BFF34F8FBFF36F8F8F
:1016400005B05DF804FB00BF7C13002004ED00E052
:101650001FB500230C4904AA42F8043D08700B484A
:101660000092402101220068F1F7BCFB039B3BB1D3
:101670004FF08052064B1A60BFF34F8FBFF36F8F4E
:1016800005B05DF804FB00BFB81100207C130020FA
:1016900004ED00E000487047B0110020114810B57B
:1016A000002303224FF480710068F1F72BFB4FF009
:1016B00080520D4B1A60BFF34F8FBFF36F8F0B4CEF
:1016C0002068F2F753FC40B1BDE810400023084801
:1016D0001A4619460068F2F7CFB80120F0F74CFF20
:1016E000EEE700BF7C13002004ED00E0741300203F
:1016F0006C130020F8B5104B01461868F2F7A8FAF1
:101700000446B8B14FF080560C4F0D4D0023032214
:101710004FF400713868F1F7F5FA2E60BFF34F8F80
:10172000BFF36F8F3868F0F73BFD2E60BFF34F8F2C
:10173000BFF36F8F2046F8BD6C1300207C13002090
:1017400004ED00E0014B1860704700BF64130020F7
:1017500070B5044678B10378032B0CD1436853B1BC
:101760000025054E1868F26990476068F3690560C6
:1017700098476560257070BD8C11002010B50C482D
:101780000C4C0023052221460068F2F775F8012869
:1017900007D100236360084B1B683BB1BDE81040D4
:1017A00018472046BDE81040FFF7D2BF10BD00BF6C
:1017B00068130020BC110020641300201FB5064CE4
:1017C000002201A92068F2F7B1F908B904B010BDF0
:1017D00001A8FFF7BDFFF3E768130020014B18686D
:1017E000704700BF6813002010B50446064B010A7D
:1017F000A3F84A00202000F045FBE1B22120BDE81B
:10180000104000F03FBB00BF7018002008B5FFF784
:10181000EBFF0122014B83F8522008BD7018002015
:10182000002238B50B4B05461D2083F84E100C46A0
:1018300083F84C2000F080FB20F0060040EA4401D1
:10184000C9B21D2000F01EFB2946BDE83840232008
:1018500000F018BB7018002013B5164C0120A368C7
:101860009847002341F6FE720093009B934218DDD7
:10187000A36802209847002341F6FE720193019B62
:10188000934212DD0C4BB5211C6C4020A047A021D7
:101890004120A04700210120234602B0BDE81040AE
:1018A0001847009B01330093DFE7019B013301934D
:1018B000E5E700BF8C110020ACE60108094B07B535
:1018C0001B6CC2213B209847002341F6FE72019316
:1018D000019B934202DD03B05DF804FB019B0133E1
:1018E0000193F5E7ACE601082DE98748814B824872
:1018F000824E0360824B834C8360834BDFF83492CB
:101900004360824BDFF830B2C360814B0361814B8F
:101910008361814BC36133689847002320681A466E
:101920001946F1F7A9FF7D4B1879F0B94FF0FF3355
:10193000194601AAF1F79CF90028F4D0019BD805BB
:101940001AD500F05DFA002000F0B0FDF36A984768
:10195000FFF734FF0023D9F800001A461946F1F7C3
:101960008BFF0020F0F786FEDDE741F2883301AA05
:101970004FF0FF310020DDE799050DD500F040FA6A
:10198000FFF79CFFF36A9847FFF718FF6421D9F827
:101990000000F2F75DF9C6E7D9F80000F2F7E6FAC1
:1019A0000128C0D0DBF8003023B94FF4B6715C4891
:1019B000F2F72EFC019B1A0604D50722594B1A7028
:1019C000FFF7DCFE019B5B074DD500212068F2F795
:1019D0003FF9012847D1DFF864A10C20DAF818306C
:1019E0009847054668B90346024601462068F1F764
:1019F00043FF002897D140F281114948F2F708FCD3
:101A000091E7DFF83C81DAF81830B8F8040098471D
:101A1000074678B9DAF81C30284698473B463A46DC
:101A200039462068F1F728FF00287FF47CAF40F2A8
:101A30008911E2E708F1040303CB2F606860A96015
:101A40003846D8F80010B8F8042005F098FB0322B7
:101A5000344B1A705D60FFF791FE002320681A4630
:101A60001946F1F709FF019BDF0709D501222D4B2C
:101A70001A7000225A602C4A12689A60FFF77EFEA4
:101A8000019BDD0606D50522264B1A7000225A60FE
:101A9000FFF774FE019B180706D50422214B1A702C
:101AA00000225A60FFF76AFE019B990706D50222C1
:101AB0001C4B1A7000225A60FFF760FE019B9A06C9
:101AC00006D50622174B1A70184A5A60FFF756FEC1
:101AD000019B5B067FF527AF154B1A78114B32B18E
:101AE00008221A7000225A60FFF748FE1BE70922FD
:101AF000F7E700BF451501086C110020ACE60108AE
:101B00007D1401087013002031150108C915010862
:101B100015160108511601088D150108B011002095
:101B20000EB90108BC11002078130020B911002063
:101B3000B811002074130020681300208C110020BD
:101B4000C8110020044B10B55B6998470446FFF7A5
:101B500083FE204610BD00BFACE60108F0B5674C1F
:101B6000054626460F461822002185B0644805F038
:101B70002AFB0FCD0FC695E80F0086E80F0097E807
:101B8000030063695F4D013B033388BF5E4B85E80B
:101B9000030088BF63616368013B033304D94FF4DA
:101BA00031715A48F2F734FB2368013B033304D9FF
:101BB0004FF432715548F2F72BFBA368013B033316
:101BC00004D94FF433715148F2F722FBE368013B2B
:101BD000033304D94FF434714C48F2F719FB2369ED
:101BE000013B033304D94FF435714848F2F710FB39
:101BF000E369013B033304D94FF436714348F2F7EC
